:100000000C944D500C947E500C947E500C947E5069
:100010000C947E500C947E500C947E500C947E5028
:100020000C947E500C947E500C947E500C947E5018
:100030000C947E500D94ABBE0C947E500C947E506C
:100040000C947E500D94923E0C947E500C947E50F5
:100050000C947E500C947E500D94A0510D94DAB601
:100060000C947E500C94A65B0C947E500C947E50A5
:100070000C947E500C947E500C947E500C947E50C8
:100080000C947E500C947E500C947E500C947E50B8
:100090000C947E500C947E500C947E500C947E50A8
:1000A0000C947E500C947E500C947E500C947E5098
:1000B0000C947E500C947E500C947E500C947E5088
:1000C0000C947E500C947E500C947E500C947E5078
:1000D0000C947E500C947E500C947E500C947E5068
:1000E0000C947E50BA014001B40182016401CC013C
:1000F0008401C00174014601AE019001C2014401B6
:1001000052013A01C6017C018C015A013E014801AD
:10011000A2016A019601580134012E01BC0142017D
:100120007801BE014C0196014E0154018E01B601C9
:10013000A0013C0162015E01A801360188017E0137
:10014000AC01A601D0019E01C401A801CE01560157
:100150005001036EDB363D9A9999993DABAAAA2AC4
:100160003E000000803F084AD73B3BCE016E84BC76
:10017000BFFDC12F3D6C74319ABD56833DDA3D0001
:10018000C77F11BED9E4BB4C3E916BAAAABE00004A
:1001900000803F072C7AA5BA6CC590DA3B9365FCCA
:1001A0008BBC53F810FD3C5692834DBD879D3AB6EB
:1001B0003DCBC9BF5BBE73DA0FC93F05A84CCDB2BA
:1001C000D44EB93836A9020C50B9918688083CA69D
:1001D000AAAA2ABE000000803F07634236B79BD818
:1001E000A71A39685618AEBAAB558C1D3CB7CC5718
:1001F00063BD6DEDFD753EF6177231BF00000080E6
:100200003F08000000BE922449123EABAAAA2ABEB3
:10021000CDCCCC4C3E00000080BEABAAAAAA3E00CA
:10022000000000BF000000803F0000000000084107
:1002300078D3BB4387D1133D190E3CC3BD4282AD79
:100240002B3E68EC8276BED98FE1A93E4C80EFFF51
:10025000BE01C4FF7F3F0000000000000D9453B8B2
:100260000D94BE7A0D940C960D944BB80D94DBB89A
:100270000D94147A0D941B7D0D94C6B80D9420B87E
:100280000D94FB510D9467B80D94CD7C0D94715273
:100290000D9425B80D948D780D948AB80D9494B86A
:1002A0000D9409B90D94EC7C0D949EB80D9405B98C
:1002B0000D9443B80D941BB80D940B7A0D94D0B8DF
:1002C0000D9448A70D94CAB80D943F520D9421592E
:1002D0000D94FF6E0D9439B80D94DF860D946D6DFD
:1002E0000D94FC550D9471420D946D520D941D7C2E
:1002F0000D9471B80D9459760D942F7D0D94E5B839
:100300000D9436590D9425520D9467520D94305921
:100310000D94DFB80D9494890D94497D0D94A8B87F
:100320000D94967C0D94829F0D94D4580D94B2B880
:100330000D94825D0D94A16A0D9408920D94F7B806
:100340000D94D7B80D942FB80D949E1B0D94EDB855
:100350000D940EB90D9462AE0D94E9B80D947952D6
:100360000D94F9790D94CC8C0D9417520D94D4B84A
:100370000D94A5B90D94ED510D945DB80D9480B810
:100380000D946B520D94B07C0D94FBB80D94257DAB
:100390000D94885F0D948F940D944D520D9401B976
:1003A0000D94F3B80D945E570D949E5A0D94027AF5
:1003B00048617264636F6465642044656661756C4E
:1003C000742053657474696E6773204C6F61646543
:1003D000640053746F7265642073657474696E672A
:1003E00073207265747269657665640046696C6134
:1003F0006D656E742073657474696E67733A20441A
:10040000697361626C6564002020204D32303020B9
:10041000440046696C616D656E742073657474691F
:100420006E67733A002020204D323039205300414E
:1004300075746F2D526574726163743A20533D3048
:1004400020746F2064697361626C652C20312074A4
:100450006F20696E7465727072657420657874724D
:100460007564652D6F6E6C79206D6F766573206194
:1004700073207265747261637473206F7220726589
:10048000636F766572696573002046002020204DF9
:100490003230382053005265636F7665723A2053CC
:1004A0003D4578747261206C656E67746820286DB4
:1004B0006D2920463A537065656420286D6D2F6D57
:1004C0002900205A002046002020204D32303720BD
:1004D0005300526574726163743A20533D4C656EEB
:1004E00067746820286D6D2920463A5370656564ED
:1004F00020286D6D2F6D29205A3A205A4C69667458
:1005000020286D6D29002044002049002020204D26
:10051000333034205000504944206865617462656E
:10052000642073657474696E67733A002044002018
:1005300049002020204D33303120500050494420C4
:1005400073657474696E67733A00205A002059000D
:1005500020204D323036205800486F6D65206F6680
:100560006673657420286D6D293A00204500205A75
:100570000020590020580020420020540020204D27
:10058000323035205300416476616E6365642076B5
:1005900061726961626C65733A20533D4D696E20EA
:1005A000666565647261746520286D6D2F73292CF2
:1005B00020543D4D696E2074726176656C206665CD
:1005C00065647261746520286D6D2F73292C20423B
:1005D0003D6D696E696D756D207365676D656E74CF
:1005E0002074696D6520286D73292C20583D6D613C
:1005F00078696D756D205859206A65726B20286D79
:100600006D2F73292C20205A3D6D6178696D756DB1
:10061000205A206A65726B20286D6D2F73292C205B
:1006200020453D6D6178696D756D2045206A657264
:100630006B20286D6D2F73290020540020204D322F
:100640003034205300416363656C65726174696F77
:100650006E3A20533D616363656C65726174696FC6
:100660006E2C20543D726574726163742061636303
:10067000656C65726174696F6E00204500205A00D8
:1006800020590020204D3230312058004D617869CA
:100690006D756D20416363656C65726174696F6E21
:1006A00020286D6D2F7332293A00204500205A0012
:1006B00020590020204D3230332058004D61786998
:1006C0006D756D2066656564726174657320286D53
:1006D0006D2F73293A00204500205A002059002030
:1006E000204D393220580053746570732070657244
:1006F00020756E69743A0053657474696E6773206F
:1007000053746F726564007364706F733A00506560
:100710007263656E7420646F6E653A004D323620E8
:10072000532564004D323400506F736974696F6EE5
:1007300020726561642066726F6D20656570726FEE
:100740006D3A004D32332025730020423A00204597
:100750003A00543A005A20736869667420617070D8
:100760006C6965643A000A005A206C6976652061FC
:10077000646A757374206F7574206F662072616E81
:1007800067652E2053657474696E6720746F20301E
:100790002E20436C69636B20746F20636F6E7469E5
:1007A0006E75652E005A206C6976652061646A75E5
:1007B0007374206F7574206F662072616E67652E8A
:1007C0002053657474696E6720746F203000205761
:1007D0003A0020453A00543A004175746F002045B4
:1007E0002F443D00416476616E6365204B3D0022DD
:1007F000005400496E76616C6964205420636F6414
:10080000652E00496E76616C6964204D20636F64CB
:10081000652E004D3232302053256900203A2000E9
:10082000004C414E472053454C20464F52434544CF
:10083000002200205A3A0020593A0020453A002070
:100840005A3A0020593A00583A0020002E0020421F
:100850003A0020453A00543A002042403A002040F5
:100860003A00202F003A00205400202F0020423A66
:1008700000202F006F6B20543A002569206D696EAF
:100880002C2025692073656300496E76616C69646C
:10089000204D20636F6465004D6573682062656458
:1008A000206C6576656C696E67206E6F742061637D
:1008B000746976652E000A002020000A4D65617378
:1008C0007572656420706F696E74733A000A5A20FD
:1008D000736561726368206865696768743A2000AF
:1008E0002C004E756D20582C593A2000476F206817
:1008F0006F6D652066696E6973686564004D657328
:100900006820626564206C6576656C696E6720613D
:10091000637469766174656400557073616D706CA1
:10092000652066696E697368656400426564206C61
:100930006576656C696E6720636F72726563746952
:100940006F6E2066696E697368656400206D696307
:10095000726F6E73004578636573736976652062A4
:100960006564206C6576656C696E6720636F727272
:10097000656374696F6E3A200042656420636F722C
:1009800072656374696F6E2064617461206E6F7448
:100990002076616C69640A0042656420636F72723C
:1009A000656374696F6E20646174612076616C693F
:1009B000640A006261627973746570206170706CA2
:1009C00069656400636C65616E2075702066696E90
:1009D000697368656420004D4553485F484F4D4535
:1009E0005F5A5F5345415243483A20004D65736852
:1009F00020626564206C6576656C696E6720776837
:100A0000696C65206C6F6F702066696E69736865CC
:100A1000642E00006D65736820626564206C6576E5
:100A2000656C696E673A20000A00593A2000005848
:100A30003A20003A206E6F20787920636C616D70E7
:100A4000696E670A003A20787920636C616D706581
:100A5000642E0A00002C2063616C69627261746903
:100A60006F6E207A3A2000426564206C6576656C72
:100A7000696E672C20706F696E743A2000005A20EE
:100A80006A697474657220646174612066726F6D46
:100A9000205A2063616C2E206E6F742076616C6921
:100AA000642E0A005A206A69747465722064617445
:100AB000612066726F6D205A2063616C2E20766112
:100AC0006C69642E0A004E6F20636C616D70696EF4
:100AD0006720666F722066697273742063616C6947
:100AE00062726174696F6E20706F696E742E0A0095
:100AF00046697273742063616C6962726174696FB4
:100B00006E20706F696E7420636C616D7065642E09
:100B10000A0047323820573000473238205730001B
:100B200054656D70657261747572652063616C697E
:100B300062726174696F6E20646F6E652E20436F00
:100B40006E74696E7565207769746820707265735C
:100B500073696E6720746865206B6E6F622E00008B
:100B6000205A20736869667420286D6D293A0054F4
:100B7000656D70657261747572653A2000002F367C
:100B800000537465703A2000005A45524F3A2000D5
:100B90000050494E44412070726F62652063616C61
:100BA0006962726174696F6E207374617274004758
:100BB0003238205730000A00205A3A200020593A93
:100BC000200020583A20004D323230205325690051
:100BD000256920686F757273202569206D696E75AF
:100BE0007465730054494D454F55543A004D3131A9
:100BF000300046756C6C20525820427566666572EE
:100C0000004D3239002055706C6F616420696E2090
:100C100070726F677265737300466163746F727987
:100C2000205245534554004A756C202036203230FE
:100C3000313700436F6D70696C65643A200033444E
:100C40002D677573736E65722C2054657374004A3A
:100C5000756C20203620323031372031303A31392E
:100C60003A34310073746172740025002020202012
:100C70002020002020202020200045524153494EB2
:100C80004720616C6C206461746100466163746F1D
:100C900072792052455345540022206661696C6583
:100CA000643A204275666665722066756C6C210038
:100CB000456E717565696E6720746F207468652074
:100CC00066726F6E743A2022002200456E7175655F
:100CD000696E6720746F207468652066726F6E7429
:100CE0003A20220022206661696C65643A204275D0
:100CF000666665722066756C6C21002200FFFFFF3E
:100D00000000A0400000A0400000004000007A4326
:100D1000333354439AD9514300000000CDCC0CC06A
:100D20009A99193E00007A43000052430000524352
:100D300000000000CDCC0CC09A99193E6563686F25
:100D40003A004572726F723A00000021104220632F
:100D5000308440A550C660E770088129914AA16B94
:100D6000B18CC1ADD1CEE1EFF1311210027332522C
:100D700022B5529442F772D662399318837BB35AE4
:100D8000A3BDD39CC3FFF3DEE362244334200401FC
:100D900014E664C774A44485546AA54BB528850934
:100DA00095EEE5CFF5ACC58DD553367226111630CC
:100DB00006D776F6669556B4465BB77AA719973884
:100DC00087DFF7FEE79DD7BCC7C448E5588668A70C
:100DD000784008611802282338CCC9EDD98EE9AFD4
:100DE000F9488969990AA92BB9F55AD44AB77A966C
:100DF0006A711A500A333A122AFDDBDCCBBFFB9E24
:100E0000EB799B588B3BBB1AABA66C877CE44CC53B
:100E10005C222C033C600C411CAEED8FFDECCDCD73
:100E2000DD2AAD0BBD688D499D977EB66ED55EF40B
:100E30004E133E322E511E700E9FFFBEEFDDDFFCC3
:100E4000CF1BBF3AAF599F788F8891A981CAB1EB68
:100E5000A10CD12DC14EF16FE18010A100C230E391
:100E6000200450254046706760B9839893FBA3DA4D
:100E7000B33DC31CD37FE35EF3B1029012F322D2E1
:100E8000323542145277625672EAB5CBA5A89589DD
:100E9000856EF54FE52CD50DC5E234C324A0148131
:100EA000046674476424540544DBA7FAB79987B8ED
:100EB000975FE77EF71DC73CD7D326F2369106B081
:100EC0001657667676154634564CD96DC90EF92FED
:100ED000E9C899E9898AB9ABA944586548067827D1
:100EE00068C018E1088238A3287DCB5CDB3FEB1E8D
:100EF000FBF98BD89BBBAB9ABB754A545A376A1621
:100F00007AF10AD01AB32A923A2EFD0FED6CDD4D1C
:100F1000CDAABD8BADE89DC98D267C076C645C4570
:100F20004CA23C832CE01CC10C1FEF3EFF5DCF7C2C
:100F3000DF9BAFBABFD98FF89F176E367E554E74C0
:100F40005E932EB23ED10EF01E7C3C3E5E2B3D3FAA
:100F50002F5B5D3B2C2A225C004D383420582059F1
:100F6000205A2045004D3234004D32332025730085
:100F70006175746F25692E67000A002F000A002E24
:100F80000044656C6574696F6E206661696C6564A8
:100F90002C2046696C653A200046696C65206465C2
:100FA0006C657465643A002E002E002E002E004EF3
:100FB0006F772066726573682066696C653A2000F9
:100FC0004E6F7720646F696E672066696C653A20A2
:100FD000002220706F73002220706172656E743A77
:100FE0002200535542524F5554494E452043414CDF
:100FF0004C207461726765743A2200747279696E6C
:101000006720746F2063616C6C207375622D676359
:101010006F64652066696C657320776974682074F5
:101020006F6F206D616E79206C6576656C732E2014
:101030004D4158206C6576656C2069733A0050729A
:10104000757361206933204D4B3220676572656589
:10105000642E005072757361206933204D4B32202D
:101060006265726569742E00507275736120693310
:10107000204D4B3220676F746F776100507275732B
:1010800061206933204D4B3220707265702E005004
:1010900072757361206933204D4B322070726F6E10
:1010A00074612E005072757361206933204D4B328C
:1010B000206F6B005072757361206933204D4B3285
:1010C0002072656164792E007A5F6D696E3A200046
:1010D0007A5F6D61783A20005A204F6666736574B6
:1010E00000795F6D696E3A2000795F6D61783A2012
:1010F000004A61004A610054616B00536900536902
:1011000000416E6F0059657300785F6D696E3A201B
:1011100000785F6D61783A200020576174636864DD
:101120006F6720526573657400496E666F20736344
:101130006865726D00496E666F726D6174696F6E7D
:1011400000496E666F726D61636A65004D6F6E690E
:10115000746F72697A61720053636865726D61744D
:101160006120696E666F00496E666F726D616365BE
:1011700000496E666F2073637265656E0057616328
:101180006874656E206F702061666B6F656C656E4C
:101190002076616E2068656174657220656E2062DC
:1011A00065642E0057617274656E2061756620411A
:1011B000626B7565686C756E6720766F6E2044751E
:1011C00065736520756E6420426574742E004F63EC
:1011D0007A656B6977616E6965206E6120777963E6
:1011E000686C6F647A656E6965206479737A7920BA
:1011F0006920706F646B6C61646B692E004573705D
:101200006572616E646F20656E667269616D696595
:101210006E746F206465206C612063616D6120795C
:101220002064656C206578747275736F722E004946
:101230006E206174746573612064656C20726166F0
:101240006672656464616D656E746F2064656C6C54
:10125000612074657374696E6120652064656C201B
:1012600070696174746F0043656B616E69206E61B3
:10127000207A63686C61646E757469207472797326
:101280006B79206120706F646C6F7A6B792E0057D8
:10129000616974696E6720666F72206E6F7A7A6C0E
:1012A0006520616E642062656420636F6F6C696E97
:1012B00067005761636874656E206F7020676562B0
:1012C0007275696B6572005761727465206175662D
:1012D000204E75747A65722E2E2E004573706572DD
:1012E000616E646F206F7264656E65730041747423
:1012F000656E64656E646F207574656E7465005705
:1013000061697420666F7220757365722E2E2E00CF
:101310004765627275696B742062696A20707269D0
:101320006E740042656E75747A74206265696D2012
:10133000447275636B00557A7974652070727A799E
:10134000206472756B7500557361646F20656E2043
:10135000696D70726573696F6E0055736174692091
:101360006E656C6C61207374616D706100506F7597
:101370007A69746520626568656D207469736B7540
:10138000005573656420647572696E6720707269B8
:101390006E740046696C616D656E74207569746861
:1013A000616C656E0046696C616D656E7420656E7A
:1013B000746E65686D656E0057796A616320666951
:1013C0006C616D656E7400536F6C74617220666938
:1013D0006C616D656E746F00536361726963612047
:1013E00066696C616D656E746F0056796A6D6F75B4
:1013F000742066696C616D656E7400556E6C6F610A
:10140000642066696C616D656E740046696C616D1F
:10141000656E742075697477657270656E004669D3
:101420006C616D656E742061757377657266656E4B
:10143000005779737577616D2066696C616D656EB3
:101440007400536F6C74616E646F2066696C616DBB
:10145000656E746F0052696C6173632E2066696CEF
:10146000616D656E746F005679736F7576616D206E
:1014700066696C616D656E7400556E6C6F61646950
:101480006E672066696C616D656E7400556E6B6E7B
:101490006F776E20636F6D6D616E643A2022004637
:1014A000696A6E696E7374656C6C696E67656E00EF
:1014B0004665696E65696E7374656C6C756E670000
:1014C0004E617374726F696300416A7573746172FF
:1014D000005265676F6C61004C61646974005475FB
:1014E0006E65005344204B61727465205B466C73DB
:1014F000684169725D006B617274612053445B46A0
:101500006C73684169725D005344206361726420AA
:101510005B466C73684169725D005344204B617295
:101520007465205B6E6F726D616C5D006B617274CF
:1015300061205344205B6E6F726D616C5D0053449B
:101540002063617264205B6E6F726D616C5D005030
:10155000494E444120542E6B616C2E205B4F4E5DF2
:101560000050494E444120542E4B616C2E205B4F5D
:101570004E5D00436965706C2E206B616C2E205BA4
:101580004F4E5D0043616C2E2074656D702E205BA4
:101590004F4E5D0043616C2E2074656D702E205B94
:1015A0004F4E5D005465706C2E206B616C2E205B7D
:1015B0004F4E5D0050494E444120542E63616C2EC5
:1015C000205B4F4E5D0050494E444120542E6B61CC
:1015D0006C2E5B4F46465D0050494E444120542ED0
:1015E0004B616C2E5B4F46465D00436965706C2E07
:1015F000206B616C2E205B4F46465D0043616C2E74
:101600002074656D702E205B4F46465D0043616C13
:101610002E2074656D702E205B4F46465D0054652C
:10162000706C2E206B616C2E205B4F46465D005027
:10163000494E444120542E63616C2E5B4F46465DFB
:101640000050494E44412074656D70657261747537
:1016500075722063616C6962726174696520697377
:10166000206B6C6161722E204B6C696B206F6D205A
:10167000646F6F72207465206761616E2E0044692B
:10168000652050494E44412054656D706572617407
:1016900075726B616C696272696572756E672069DB
:1016A0007374206265656E6465742E204B6C69638B
:1016B0006B6520756D20666F72747A7566616872ED
:1016C000656E2E00436965706C6E61206B616C699C
:1016D000627261636A61207A616B6F6E637A6F6EAA
:1016E000612E204B6F6E74796E75756A2070727AF8
:1016F000796369736B69656D0043616C69627261DE
:10170000636F6E2074656D706572617475726120AF
:101710007465726D696E6164612E205072657369C3
:101720006F6E6172207061726120636F6E74696E9A
:101730007561722E005461726174757261207465F6
:101740006D7065726174757261207465726D696E19
:101750006174612E204661726520636C69636B2041
:1017600070657220636F6E74696E756172652E00AC
:101770005465706C6F746E69206B616C6962726124
:10178000636520646F6B6F6E63656E612E20506FB2
:101790006B726163756A746520737469736B656DD0
:1017A00020746C616369746B612E0050494E444132
:1017B0002074656D70657261747572652063616C0B
:1017C0006962726174696F6E2069732066696E69FF
:1017D000736865642E20436C69636B20746F2063AB
:1017E0006F6E74696E75652E0050494E44412054E9
:1017F000656D702E6B616C2E0050494E4441205433
:10180000656D702E4B616C2E2020202020004369D6
:1018100065706C2E206B616C2E20202020202020F3
:1018200020200043616C2E2074656D702E202020D6
:10183000202020202020200043616C2E2074656D24
:10184000702E202020202020202020200054657091
:101850006C2E206B616C2E20202020202020202048
:10186000200050494E44412054656D702E63616CD8
:101870002E20202020200054656D706572617475E3
:1018800075720054656D706572617475720054658F
:101890006D70657261747572610054656D7065720A
:1018A00061747572610054656D70657261747572F2
:1018B00061005465706C6F74610054656D70657281
:1018C000617475726500506F6D6F6300536F706F58
:1018D00072746500506F64706F7261005375707040
:1018E0006F7274005072696E742073746F707065DB
:1018F0006E00447275636B20616262726563686535
:101900006E005A6174727A796D6163206472756BCE
:1019100000446574656E657220696D7072657369E7
:101920006F6E0041727265737461207374616D70C3
:1019300061005A61737461766974207469736B0015
:1019400053746F70207072696E7400474553544F22
:1019500050542E2000474553544F5050542E2000D1
:101960005041524144410041525245535441544F19
:101970002E0053544F505045442E20005374657030
:101980007261746520746F6F20686967683A20001F
:10199000546F74616C207072696E7474696A643A11
:1019A00000546F74616C6520447275636B7A65696D
:1019B000743A00437A61732063616C6B6F7769746A
:1019C00079203A005469656D706F20746F74616C92
:1019D000203A0054656D706F207374616D706120E2
:1019E000746F743A0043656C6B6F76792063617332
:1019F000203A00546F74616C207072696E742074A8
:101A0000696D65203A0046696C616D656E7420747D
:101A10006F74616C3A200046696C616D656E74206C
:101A2000476573616D743A0046696C616D656E74EB
:101A3000206C61637A6E6965203A0046696C616D5D
:101A4000656E746F20746F74616C3A0046696C61E6
:101A50006D656E746F20746F743A0046696C616DC9
:101A6000656E742063656C6B656D203A00546F740D
:101A7000616C2066696C616D656E74203A0050720D
:101A8000696E7474696A643A202020004472756338
:101A90006B7A6569743A202000437A61732064721E
:101AA000756B75203A2020005469656D706F206455
:101AB0006520696D702E3A0054656D706F20646901
:101AC000207374616D70613A0043617320746973AF
:101AD0006B75203A2020005072696E742074696D15
:101AE000653A20200046696C616D656E747665729A
:101AF000627275696B3A0046696C616D656E7476E9
:101B000065726272617563683A0046696C616D6501
:101B10006E74203A20200046696C616D656E746FAA
:101B2000203A20200046696C616D656E746F2075E7
:101B30007361746F3A0046696C616D656E74203A2A
:101B400020200046696C616D656E74207573656454
:101B50003A2020005374617469737469656B656E13
:101B60000053746174697374696B656E20005374FB
:101B70006174797374796B612020004573746164BA
:101B800069737469636120200053746174697374AC
:101B9000696368650053746174697374696B61206B
:101BA0002000537461746973746963732020004565
:101BB00072726F72202D20737461746963206D6579
:101BC0006D6F727920686173206265656E206F7633
:101BD00065727772697474656E00536E656C6865C2
:101BE000696400476573636877696E6469676B65EC
:101BF000697400507265646B6F73630056656C6F37
:101C000063696461640056656C6F63697461005256
:101C10007963686C6F73740053706565640020535A
:101C20006F667477617265205265736574004D6FDD
:101C300064652020202020205B6C656973655D0051
:101C40004D6F64202020202020205B636963687929
:101C50005D004D6F646F2020205B73696C656E635F
:101C6000696F5D004D6F646F205B73696C656E7AA0
:101C7000696F736F5D004D6F64202020202020204D
:101C80005B74696368795D004D6F64652020202076
:101C9000205B73696C656E745D004D6F6465205BDD
:101CA000486F6865204C656973745D004D6F6420F2
:101CB0005B7720777964616A6E6F73635D004D6F47
:101CC000646F205B72656E642E706C656E6F5D0074
:101CD0004D6F64652020202020205B666F72746544
:101CE0005D004D6F6420205B7679732E2076796BD2
:101CF0006F6E5D004D6F6465205B6869676820707A
:101D00006F7765725D00546F6F6E20656E647374DB
:101D10006F707300416E7A656967656E20456E73FA
:101D20006368616C74657200506F6B617A206B72CE
:101D3000616E636F776B6900456E73656E612074C9
:101D40006F70652066696E616C00537461746F20FA
:101D500066696E65636F7273610053746176206BA0
:101D60006F6E632E207370696E2E0053686F77203C
:101D7000656E642073746F70730054656D702E20EF
:101D8000696E7374656C6C656E0054656D702E655C
:101D9000696E7374656C6C656E00557374617769F8
:101DA000632074656D70657261747572650045734A
:101DB0007461626C656365722074656D702E3A00A3
:101DC000496D706F7374612074656D7065726174B4
:101DD000757261004E61737461767465207465700C
:101DE0006C6F74753A005365742074656D7065721C
:101DF00061747572653A00496E7374656C6C696ED6
:101E000067656E0045696E7374656C6C756E6765A9
:101E10006E00557374617769656E696100436F6E1A
:101E200066696775726163696F6E00496D706F7383
:101E300074617A696F6E69004E6173746176656E64
:101E4000690053657474696E6773004265647261FA
:101E500064696E6720666F7574005665726472619E
:101E60006874756E67736665686C657200426C6154
:101E70006420706F6C61637A656E6961004572728F
:101E80006F7220646520636F6E6578696F6E0045C0
:101E900072726F7265206361626C616767696F005F
:101EA0004368796261207A61706F6A656E69005774
:101EB0006972696E67206572726F72005A656C662E
:101EC00074657374202073746172742020005365EC
:101ED0006C6273747465737420737461727420001F
:101EE0004175746F746573742073616C696461000B
:101EF0004176766961206175746F746573740053FF
:101F0000656C66207465737420737461727420202C
:101F100000436F6E74726F6C656572206175623A12
:101F2000004269747465207072756566653A005385
:101F30006B6F6E74726F6C756A203A00436F6E74CB
:101F4000726F6C61203A00566572696669636172EE
:101F5000653A005A6B6F6E74726F6C756A746520A7
:101F60003A00506C6561736520636865636B203A65
:101F7000005A656C6674657374204F4B0053656C32
:101F800062737474657374204F4B004175746F7481
:101F9000657374204F4B0053656C662074657374D1
:101FA000204F4B004E6965742061616E6765736CEC
:101FB0006F74656E004E6963687420616E67657347
:101FC00063686C6F7373656E004E696520706F6433
:101FD0006C61637A6F6E6F202020004E6F20686105
:101FE0007920636F6E6578696F6E2020004E6F6E8A
:101FF00020636F6E6E6573736F004E657A61706FEC
:102000006A656E6F20202020004E6F7420636F6E13
:102010006E65637465640053696C6E696B004D6F27
:10202000746F7265004D6F746F720043616C656E02
:10203000742E2F5465726D6973746F7200526973D8
:1020400063616C642E2F5465726D6973742E004841
:1020500065617465722F546865726D6973746F720F
:1020600000526F7465657274004472656874004B49
:1020700072656369207369650056656E74696C6189
:10208000646F722067697261004769726100546F02
:102090006369207365005370696E6E696E670052E4
:1020A0006F7465657274206E69657400447265684A
:1020B00074206E69636874004E656B726563692095
:1020C0007369650056656E74696C61646F72206E29
:1020D0006F2067697261004E6F6E207369206769B7
:1020E0007261004E65746F6369207365004E6F7492
:1020F000207370696E6E696E67004C7565667465F5
:10210000727465737400546573742077656E7479A6
:102110006C61746F726100546573742064656C2027
:1021200076656E74696C61646F720050726F76616F
:102130002064656C2076656E74696C61746F7200E2
:10214000546573742076656E74696C61746F727512
:102150000046616E2074657374005A656C66746520
:102160007374206D69736C756B74200053656C62B9
:10217000737474657374206D69736C75656B74002A
:1021800053656C6674657374206E69657564616E01
:1021900079004175746F746573742066616C6C614D
:1021A000646F004175746F746573742066616C6C44
:1021B00069746F0053656C66746573742073656C25
:1021C00068616C20200053656C66746573742066CA
:1021D00061696C65642020004C696E6B65206661E6
:1021E0006E3F004C696E6B6572204C756566746558
:1021F000723F004C6577792077656E74206E6120A0
:102200006479737A653F0056656E742E20656E2082
:102210006C6120697A673F0056656E7420535820C0
:1022200073756C6C277567656C6C6F3F004C6576D9
:10223000792076656E74206E61207472797363659F
:102240003F004C65667420686F74656E642066613B
:102250006E3F005A656C667465737420466F7574C2
:1022600020210053656C6273747465737420466535
:10227000686C65722021004175746F7465737420F9
:102280006572726F7221004175746F74657374208A
:102290006E6567617469766F0053656C667465730B
:1022A00074206572726F72202100456E6473746FC2
:1022B00070206E6965742067657261616B7400459A
:1022C0006E647363682E206E2E206572726569637A
:1022D000687400546F70652066696E2E206E6F20E2
:1022E000746F632E0046696E65632E2066756F728B
:1022F0006920706F722E00456E6473746F70206E6B
:102300006F742068697400456E64736368616C74EF
:10231000657200546F7065732066696E616C00466B
:10232000696E65636F7273612028322900456E649F
:1023300073746F707300546F70652066696E616CA2
:102340000046696E65636F72736100456E647374F5
:102350006F7000566F6F72646572652066616E3FC4
:1023600000566F726465726572204C75656674659F
:10237000723F0050727A6F646E692077656E742EBA
:10238000206472756B753F0056656E742E20616C0B
:10239000206672656E74653F0056656E74206469D0
:1023A000207374616D706120616E742E3F005072F5
:1023B00065646E69207469736B6F76792076656EDB
:1023C000743F0046726F6E74207072696E7420667E
:1023D000616E3F00436F6E74726F6C656572205A58
:1023E0002061732020202000507275656665205A98
:1023F00020416368736520202020004B6F6E74724B
:102400006F6C61205A2061786973202000436F6EE1
:1024100074726F6C2064656C20656A65205A005682
:10242000657269666963612061737365205A004B48
:102430006F6E74726F6C61205A206178697320200E
:1024400000436865636B696E67205A206178697321
:10245000202000436F6E74726F6C65657220592086
:102460006173202020200050727565666520592018
:10247000416368736520202020004B6F6E74726F7B
:102480006C6120592061786973202000436F6E745D
:10249000726F6C2064656C20656A65205900566512
:1024A00072696669636120617373652059004B6FBF
:1024B0006E74726F6C6120592061786973202000FE
:1024C000436865636B696E67205920617869732082
:1024D0002000436F6E74726F6C65657220582061C6
:1024E00073202020200050727565666520582041B9
:1024F0006368736520202020004B6F6E74726F6CD0
:102500006120582061786973202000436F6E7472D7
:102510006F6C2064656C20656A6520580056657292
:10252000696669636120617373652058004B6F6E43
:1025300074726F6C612058206178697320200043A9
:102540006865636B696E6720582061786973202025
:1025500000436F6E74726F6C65657220686F74658E
:102560006E6420200050727565666520486F746542
:102570006E642020202020004B6F6E74726F6C619F
:1025800020686F74656E64202000436F6E74726FF4
:102590006C20686F74656E642000566572696669A8
:1025A0006361207567656C6C6F004B6F6E74726F42
:1025B0006C6120686F74656E6420200043686563F9
:1025C0006B696E6720686F74656E64202000436FCE
:1025D0006E74726F6C65657220656E6473746F7073
:1025E000730050727565666520456E64736368613B
:1025F0006C7465722020004B6F6E74726F6C61207A
:10260000656E6473746F707300436F6E742E207404
:102610006F7065732066696E616C005665726966DD
:102620006963612066696E65636F727361004B6FE9
:102630006E74726F6C6120656E6473746F7073007A
:10264000436865636B696E6720656E6473746F7051
:102650007300436F6E74726F6C656572206265649F
:1026600020200050727565666520426574742020D4
:10267000202020202020004B6F6E74726F6C612030
:10268000626564202020202000436F6E74726F6C9E
:102690002064652063616D610056657269666963D7
:1026A00061206C6574746F004B6F6E74726F6C6137
:1026B00020626564202020202000436865636B69E8
:1026C0006E6720626564202020202000416C6C65CC
:1026D0006D61616C20676F65642020202000416C73
:1026E0006C6573207269636874696720202020001C
:1026F00057737A7973746B6F204F4B202020202002
:102700002000546F646F2062696520004E6573730A
:10271000756E206572726F726500567365204F4B3F
:10272000202020202020202020202000416C6C2010
:10273000636F727265637420202020202000426540
:102740007474202F204865617465720043616D6167
:102750002F43616C656E7461646F72004C657474B4
:102760006F2F52697363616C642E00426564202F81
:1027700020486561746572005A656C66746573748F
:102780002020202020202020200053656C627374BC
:102790007465737420202020202020004175746F00
:1027A00074657374004175746F7465737400536558
:1027B0006C66746573742020202020202020200067
:1027C00057726974696E6720746F2066696C653A28
:1027D0002000766F6C756D652E696E697420666178
:1027E000696C6564002053697A653A20005344207F
:1027F00076657277696A64657264005344204B6140
:1028000072746520656E746665726E74004B6172D9
:1028100074612077796A657461005461726A6574C5
:102820006120726574697261646100534420726949
:102830006D6F737361004B617274612076796A6D9C
:1028400075746100436172642072656D6F766564B2
:10285000005344207072696E74696E6720627974E7
:102860006520006F70656E206661696C65642C2060
:1028700046696C653A20006F70656E526F6F742008
:102880006661696C656400534420696E67657374A2
:102890006F6B656E005344204B61727465206569EF
:1028A0006E67657365747A74004B6172746120772A
:1028B0006C6F7A6F6E61005461726A657461206931
:1028C0006E7365727461646100534420696E736550
:1028D00072697461004B6172746120766C6F7A6505
:1028E0006E61004361726420696E73657274656421
:1028F00000534420696E6974206661696C00466902
:102900006C652073656C65637465640046696C650D
:10291000206F70656E65643A20006572726F722078
:1029200077726974696E6720746F2066696C6500E0
:1029300053442063617264206F6B0043616E6E6F5D
:102940007420656E746572207375626469723A20D2
:10295000005072696E742068657276617474656E79
:1029600000447275636B20666F72747365747A6568
:102970006E00577A6E617769616E69652064727561
:102980006B75005265616E7564617220696D70725D
:102990006573696F6E005374616D706120696E209C
:1029A00072697072657361004F626E6F766F7661E7
:1029B0006E69207469736B7500526573756D696E0D
:1029C00067207072696E74005072696E7420686559
:1029D0007276617474656E00447275636B20666F05
:1029E000727467657365747A7400577A6E6F77696D
:1029F000656E6965206472756B7500526573756DDF
:102A000069656E646F20696D70726573696F6E00C1
:102A100052697072656E6469207374616D706100D3
:102A20004F626E6F76656E69207469736B750052C4
:102A30006573756D696E67207072696E740050728F
:102A4000696E742068657276617474656E00466F95
:102A500072747365747A656E004B6F6E74796E75FF
:102A60006F776163005265616E7564617220696D94
:102A7000707265732E0052697072656E646920739E
:102A800074616D706100506F6B7261636F76617419
:102A900000526573756D65207072696E74005265C1
:102AA00073656E643A2000686F77746F2E7072756C
:102AB000736133642E637A00686F77746F2E70725F
:102AC00075736133642E637A00686F77746F2E704C
:102AD0007275736133642E636F6D00666F72756D0E
:102AE0002E707275736133642E637A00666F72752F
:102AF0006D2E707275736133642E637A00666F7227
:102B0000756D2E707275736133642E636F6D007016
:102B10007275736133642E637A00707275736133FA
:102B2000642E637A00707275736133642E636F6D07
:102B300000447275636B207061757A6572656E0012
:102B4000447275636B2070617573696572740044BB
:102B500072756B207A6174727A796D616E79004951
:102B60006D70726573696F6E20656E20706175732C
:102B700061005374616D706120696E2070617573BE
:102B800061005469736B20706F7A6173746176654C
:102B90006E005072696E74207061757365640050C8
:102BA00072696E74206166676562726F6B656E0034
:102BB000447275636B206162676562726F636865FA
:102BC0006E004472756B2070727A657277616E79EF
:102BD00000496D70726573696F6E2063616E636525
:102BE0006C616461005374616D70612061626F7229
:102BF00074697461005469736B20707265727573C7
:102C0000656E005072696E742061626F72746564E3
:102C1000005072696E746572206F6E74626F6E64BC
:102C2000656E00447275636B6572206765747265CA
:102C30006E74005072696E74657220646973636F9C
:102C40006E6E656374656400656E206472756B20DA
:102C50006F70206B6E6F7000756E64204B6E6F70BE
:102C6000662064727565636B656E004E616369739F
:102C70006E696A2070727A796369736B0050756C43
:102C800073617220656C206D616E646F00652063F6
:102C90006C696363617265206D616E6F706F6C61EA
:102CA000006120737469736B6E65746520746C6168
:102CB0006369746B6F00616E64207072657373205A
:102CC000746865206B6E6F62005475697420766F4E
:102CD0006F727665727761726D656E2100447565FD
:102CE000736520766F726865697A656E21004E6142
:102CF00067727A656A206479737A6521005072651B
:102D000063616C656E746172206578747275736F3F
:102D100072005072657269732E207567656C6C6FF6
:102D2000210050726564656872656A74652074720A
:102D300079736B75210050726568656174207468E1
:102D400065206E6F7A7A6C652100566F6F727665BA
:102D5000727761726D656E00566F726865697A652B
:102D60006E0047727A616E69650050726563616CCE
:102D7000656E7461720050726572697363616C6430
:102D800061005072656465687265760050726568AE
:102D900065617400506F77657255700057616368A4
:102DA0007420617562004269747465207761727481
:102DB000656E0050726F737A6520637A656B61632C
:102DC00000506F72204661766F7220457370657295
:102DD000617200417370657474610050726F736941
:102DE0006D2063656B656A746500506C6561736521
:102DF0002077616974002020506C616E6E657242AC
:102E0000756666657242797465733A200050494E62
:102E10004441207761726D74206F700050494E44B8
:102E20004120617566776172656D656E0047727AE3
:102E3000616E69652050494E44410043616C656E86
:102E400074616E646F2050494E444100526973634F
:102E5000616C642E2050494E4441004E6168726995
:102E600076616E692050494E44410050494E4441BC
:102E70002048656174696E670050494E4441207472
:102E8000656D70657261747575722063616C6962DD
:102E9000726174696520776173206E6F67206E6957
:102EA0006574207569746765766F65726400504952
:102EB0004E44412054656D70657261747572204B8B
:102EC000616C696272696572756E6720777572648C
:102ED00065206E6F6368206E696368742061757326
:102EE000676566756568727400436965706C6E61CC
:102EF000206B616C69627261636A61206E69652032
:102F000062796C612070727A6570726F7761647A31
:102F10006F6E61004C612074656D706572617475CF
:102F200072612064652063616C6962726163696FBC
:102F30006E206E6F206861207369646F20616A750E
:102F400073746164610054617261747572612064AC
:102F5000656C6C612074656D706572617475726109
:102F6000206E6F6E20616E636F726120657365679E
:102F700075697461005469736B61726E61206E656E
:102F800062796C61207465706C6F746E65207A6B09
:102F9000616C6962726F76616E610050494E4441A6
:102FA0002074656D70657261747572652063616C03
:102FB0006962726174696F6E20686173206E6F74EC
:102FC000206265656E2072756E20796574005049C7
:102FD00044206B616C2E202020202000504944208A
:102FE0004B616C2E2020202020004B616C2E205045
:102FF00049440043616C2E20504944202020202069
:103000002020202020200043616C2E2050494400C5
:10301000504944206B616C2E20202020202020204D
:10302000202020005049442063616C2E2020202065
:10303000202020202020202000504944206B616C5B
:103040002E206B6C616172202020202020005049CE
:1030500044204B616C2E20666572746967202020C5
:103060002020004B616C2E20504944207A616B6F08
:103070006E637A6F6E610043616C2E20504944206C
:103080007465726D696E6164610043616C2E2050DD
:10309000494420636F6D706C657461005049442031
:1030A0006B616C2E20756B6F6E63656E61005049AD
:1030B000442063616C2E2066696E697368656420C4
:1030C000202000504944206B616C69627261746910
:1030D0006500504944204B616C6962726965727584
:1030E0006E67004B616C69627261636A612050496E
:1030F000440043616C6962726163696F6E2050497C
:10310000440043616C696272617A696F6E65205038
:10311000494400504944206B616C69627261636587
:10312000005049442063616C6962726174696F6E1A
:103130000050494420626564206B616C2E20005071
:1031400049442042657474204B616C2E0050494400
:10315000206265642063616C2E2000504944206227
:103160006564206B616C2E206B6C616172202000A5
:103170005049442042657474204B616C2E20666572
:103180007274696700504944206265642063616C11
:103190002E20646F6E65202020005072696E7420AE
:1031A0007061757A6572656E005061757365005067
:1031B000727A6572776163206472756B0050617515
:1031C00073617220696D70726573696F6E004D6511
:1031D00074746920696E20706175736100506F7A34
:1031E00061737461766974207469736B00506175E2
:1031F0007365207072696E74004C65672065656E3A
:103200002076656C20706170696572206F6E6465F0
:10321000722068657420747569742074696A6465C5
:103220006E73206465206B616C696272617469659C
:103230002076616E20646520656572737465203444
:103240002070756E74656E2E20416C7320686574F5
:103250002074756974206865742070617069657286
:103260002076616E67742C205072696E74657220CE
:103270006F6E6D696464656C6C696A6B20756974E6
:10328000736368616B656C656E2E004C65676520C5
:103290007761656872656E6420646572204B616C4D
:1032A000696272696572756E672064657220657205
:1032B0007374656E20342050756E6B74652065697B
:1032C0006E20426C61747420506170696572207563
:1032D0006E746572206469652044756573652E207F
:1032E00057656E6E2064696520447565736520645A
:1032F00061732050617069657220626577656774DB
:103300002C20447275636B657220736F666F7274E4
:1033100020617573736368616C74656E2100556D0F
:1033200069657363206B6172746B6520706170698D
:10333000657275206E6120706F646B6C616463658B
:1033400020692074727A796D616A20706F642064DC
:1033500079737A6120706F64637A617320706F6D26
:1033600069617275207069657277737A7963682014
:10337000342070756E6B746F772E204A65736C699C
:10338000206479737A61207A616861637A79206F49
:10339000207061706965722C2077796C61637A2086
:1033A0006472756B61726B652E00436F6C6F636145
:1033B0007220756E6120686F6A612064652070619B
:1033C00070656C20736F627265206C61207375701C
:1033D0006572666963696520646520696D707265F0
:1033E00073696F6E20647572616E7465206C612004
:1033F00063616C6962726163696F6E206465206CE1
:103400006F73207072696D65726F732034207075F0
:103410006E746F732E205369206C6120626F71751A
:10342000696C6C61206D7565766520656C207061D6
:1034300070656C2C2061706167617220696D7072BB
:1034400065736F726120696E6D6564696174616D29
:10345000656E74652E00506F72726520756E206601
:103460006F676C696F20736F74746F206C2775675A
:10347000656C6C6F20647572616E7465206C612080
:1034800063616C696272617A696F6E6520646569F7
:10349000207072696D6920342070756E74692E20F9
:1034A000496E206361736F206C277567656C6C6F64
:1034B000206D756F766120696C20666F676C696F2F
:1034C00020737065676E6572652070726F6E7461CF
:1034D0006D656E7465206C61207374616D70616ED2
:1034E00074652E00556D697374657465206C69731D
:1034F0007420706170697275206E6120706F646CE9
:103500006F7A6B752061207564727A756A746520B4
:103510006A656A20706F6420747279736B6F7520AE
:10352000626568656D206D6572656E692070727682
:103530006E696368203420626F64752E20506F6B53
:10354000756420747279736B61207A616368797431
:10355000692070617069722C207679706E6574656F
:10356000207469736B61726E752E00506C616365B7
:103570002061207368656574206F662070617065D6
:103580007220756E64657220746865206E6F7A7A39
:103590006C6520647572696E67207468652063616C
:1035A0006C6962726174696F6E206F662066697201
:1035B0007374203420706F696E74732E20496620F6
:1035C000746865206E6F7A7A6C65206361746368D5
:1035D0006573207468652070617065722C20706F4F
:1035E000776572206F666620746865207072696EF8
:1035F00074657220696D6D6564696174656C792E9E
:10360000006F6B004F6666004765656E20626577E8
:103610006567696E672E004B65696E652042657748
:103620006567756E672E0053696E206D6F76696DE4
:1036300069656E746F004E657373756E206D6F767D
:10364000696D656E746F2E004E6F206D6F76652EFE
:10365000004765656E205344206B61617274004BB6
:1036600065696E65205344204B6172746500427237
:10367000616B206B61727479205344004E6F206837
:103680006179207461726A657461205344004E65EB
:103690007373756E61205344005A61646E612053E8
:1036A00044206B61727461004E6F2053442063614B
:1036B00072640054756974004475657365004479DB
:1036C000737A6100426F7175696C6C610055676552
:1036D0006C6C6F00547279736B61004E6F7A7A6C08
:1036E000650046696C2E206E6965742067656C61A3
:1036F00064656E0046696C2E206E6963687420678D
:10370000656C6164656E004272616B2066696C6114
:103710006D656E74750046696C2E206E6F20696E43
:1037200074726F64756369646F0046696C2E206EF5
:103730006F6E20636172696361746F0046696C61CA
:103740006D656E74206E657A61766564656E00469F
:10375000696C616D656E74206E6F74206C6F61644E
:103760006564004B6C657572206E696574206475C4
:103770006964656C696A6B004661726265206E6996
:10378000636874206B6C61722E004B6F6C6F7220DB
:103790007A616E6965637A79737A2E00436F6C6F14
:1037A00072206E6F20686F6D6F67656E656F004386
:1037B0006F6C6F7265206E6F6E207075726F004255
:1037C00061727661206E656E692063697374610051
:1037D000436F6C6F72206E6F7420636C6561720052
:1037E0004E6565004E65696E004E6965004E650068
:1037F0004E6F00557067726164656E206175622E50
:1038000000426974746520616B7475616C697369D9
:103810006572656E2E0050726F737A65207A616BE7
:103820007475616C697A6F77616300416374756167
:103830006C697A617220706F72206661766F7200B7
:10384000507265676120616767696F726E612E00F3
:1038500050726F73696D20616B7475616C697A75F4
:103860006A74652E00506C656173652075706772AF
:103870006164652E004E6965757765206669726DB5
:10388000776172652076657273696520626573631E
:1038900068696B626161723A004E657565204669C0
:1038A000726D776172652056657273696F6E2076EE
:1038B0006572667565676261723A005779737A6CF2
:1038C00061206E6F776120776572736A6120666927
:1038D000726D776172653A004E7565766F20666924
:1038E000726D7761726520646973706F6E69626C66
:1038F000653A004E756F76612076657273696F6EFA
:10390000652064656C206669726D776172652064FC
:103910006973706F6E6962696C65005679736C616A
:10392000206E6F7661207665727A65206669726DA9
:10393000776172653A004E6577206669726D7761CE
:1039400072652076657273696F6E20617661696C4D
:1039500061626C653A00566572706C6161747320C7
:103960005A00426577656765205A0050727A657320
:10397000756E6163205A004D6F766572205A004D56
:10398000756F7669205A00506F73756E6F7574206D
:103990005A004D6F7665205A00566572706C6161F1
:1039A000747320590042657765676520590050722D
:1039B0007A6573756E61632059004D6F766572206C
:1039C00059004D756F7669205900506F73756E6F91
:1039D00075742059004D6F766520590056657270D8
:1039E0006C61617473205800426577656765205883
:1039F0000050727A6573756E61632058004D6F7662
:103A000065722058004D756F7669205800506F73AD
:103A1000756E6F75742058004D6F7665205800459F
:103A2000787472756972004D756F7669204573748C
:103A30007275736F72650045787472756465720093
:103A40004B616C6962726572656E2076616E20589A
:103A5000595A2E204472616169206465206B6E6F33
:103A600070206F6D206465205A2D776167656E2028
:103A70006F6D686F6F67207465206761616E207479
:103A80006F74206865742065696E64652073746F57
:103A900070706572732E204B6C696B20616C7320A3
:103AA0006B6C6161722E004B616C69627269657248
:103AB000656E20766F6E205A2E2044726568656EA2
:103AC000205369652064656E204B6E6F70662C20F4
:103AD000626973206265696465205A2D5363686C5E
:103AE000697474656E206F6265726520416E7363E0
:103AF00068616567652065727265696368656E2EC9
:103B0000204B6C69636B656E2077656E6E20626515
:103B10006964652067616E7A206F62656E207369E3
:103B20006E642E004B616C69627261636A61205A37
:103B30002E2050727A656B7265632067616C6B65CD
:103B40002C206162792070727A6573756E616320D2
:103B50006F73205A20646F20676F726E79636820DC
:103B60006B72616E636F77656B2E204E6163697354
:103B70006E696A2C20627920706F7477696572644F
:103B80007A69632E0043616C696272616E646F20B2
:103B90005A2E204769726120656C20626F746F6EC7
:103BA000207061726120737562697220656C206398
:103BB0006172726F205A20686173746120676F6C44
:103BC0007065207069657A617320737570657269BC
:103BD0006F7261732E204465737075657320686120
:103BE0007A20636C69632E0043616C696272617A4A
:103BF000696F6E65205A2E2052756F746172652050
:103C00006C61206D616E6F706F6C612070657220E9
:103C1000616C7A61726520696C2063617272656C97
:103C20006C6F205A2066696E6F20616C6C27616C26
:103C300074657A7A61206D617373696D612E2043BA
:103C40006C69636B20706572207465726D696E615A
:103C500072652E004B616C696272616365205A2E39
:103C6000204F746163656E696D20746C6163697463
:103C70006B6120706F73756E7465205A206F737559
:103C800020617A206B7E686F726E696D7520646F3B
:103C900072617A752E20506F747672647465207428
:103CA0006C616369746B656D2E0043616C6962724F
:103CB0006174696E67205A2E20526F74617465209A
:103CC000746865206B6E6F6220746F206D6F76650F
:103CD00020746865205A206361727269616765208B
:103CE000757020746F2074686520656E642073742D
:103CF0006F70706572732E20436C69636B207768F8
:103D0000656E20646F6E652E004B616C6962726532
:103D100072656E2076616E2058595A2E2044726169
:103D20006169206465206B6E6F70206F6D20646523
:103D3000205A2D776167656E206F6D686F6F672001
:103D40007465206761616E20746F742068657420EB
:103D500065696E64652073746F70706572732E2070
:103D60004B6C696B20616C73206B6C6161722E000F
:103D70004B616C696272696572656E20766F6E2048
:103D800058595A2E2044726568656E205369652023
:103D900064656E204B6E6F70662C206269732062C2
:103DA00065696465205A2D5363686C697474656E27
:103DB000206F6265726520416E7363686165676537
:103DC0002065727265696368656E2E204B6C69634D
:103DD0006B656E2077656E6E20626569646520672D
:103DE000616E7A206F62656E2073696E642E004B7F
:103DF000616C69627261636A612058595A2E205061
:103E0000727A656B7265632067616C6B652C2061EB
:103E100062792070727A6573756E6163206F7320AA
:103E20005A20646F20676F726E796368206B7261CD
:103E30006E636F77656B2E204E616369736E696A7E
:103E40002C20627920706F7477696572647A696377
:103E50002E0043616C696272616E646F2058595A1A
:103E60002E204769726120656C20626F746F6E202E
:103E70007061726120737562697220656C20636184
:103E800072726F205A20686173746120676F6C7062
:103E900065207069657A6173207375706572696FEA
:103EA0007261732E20446573707565732068617A42
:103EB00020636C69632E0043616C696272617A6988
:103EC0006F6E652058595A2E2052756F7461726555
:103ED000206C61206D616E6F706F6C612070657217
:103EE00020616C7A61726520696C20636172726511
:103EF0006C6C6F205A2066696E6F20616C6C276154
:103F00006C74657A7A61206D617373696D612E20BE
:103F1000436C69636B20706572207465726D696EA5
:103F20006172652E004B616C696272616365205835
:103F3000595A2E204F746163656E696D20746C61EF
:103F40006369746B6120706F73756E7465205A209D
:103F50006F737520617A206B7E686F726E696D7504
:103F600020646F72617A752E20506F74767264745B
:103F70006520746C616369746B656D2E0043616CC0
:103F80006962726174696E672058595A2E20526FA7
:103F90007461746520746865206B6E6F6220746F45
:103FA000206D6F766520746865205A206361727297
:103FB0006961676520757020746F2074686520657D
:103FC0006E642073746F70706572732E20436C6919
:103FD000636B207768656E20646F6E652E00417399
:103FE00020766572706C61617473656E00426577EE
:103FF0006567652041636873650052756368206F6B
:104000007369004D6F76657220656A6573004D7542
:104010006F7669206173736500506F73756E6F758D
:1040200074206F7375004D6F766520617869730039
:104030004D657368206C6976656C2E206C657474B0
:104040006F004D65736820426564204C6576656C31
:10405000696E67004B616C69627261746965004BDF
:10406000616C696272696572756E67004B616C693B
:10407000627261636A610043616C69627261636963
:104080006F6E0043616C696272617A696F6E650080
:104090004B616C6962726163650043616C69627255
:1040A0006174696F6E002076616E20390020766F32
:1040B0006E203900207A20390020646520390020E4
:1040C0007375203900207A203900206F662039006E
:1040D0004D6574656E2076616E20726566657265E9
:1040E0006E636520686F6F6774652076616E20640B
:1040F00065206B616C6962726174696570756E745C
:10410000004D657373656E20646572205265666547
:1041100072656E7A686F65686520646573204B61AF
:104120006C69627269657270756E6B746573004F4D
:104130006B7265736C616D207779736F6B6F7363EE
:10414000206F646E69657369656E69612070756E54
:104150006B7475206B616C6962726163796A6E65FC
:10416000676F004D65646972206C6120616C7475C5
:1041700072612064656C2070756E746F20646520B8
:104180006C612063616C6962726163696F6E004D7E
:1041900069737572617265206C27616C74657A7AD7
:1041A00061206469207269666572696D656E746FFD
:1041B0002064656C2070756E746F20646920636183
:1041C0006C696272617A696F6E65004D6572696DC6
:1041D000207265666572656E636E69207679736BB1
:1041E00075206B616C69627261636E69686F2062D1
:1041F0006F6475004D6561737572696E67207265D5
:10420000666572656E636520686569676874206FAE
:10421000662063616C6962726174696F6E20706F91
:10422000696E7400486F6F66646D656E75004861F5
:104230007570746D656E7565004D656E7520676C83
:104240006F776E65004D656E75207072696E63697B
:1042500070616C004D656E75207072696E63697077
:10426000616C6500486C61766E69206E616269649C
:104270006B61004D61696E004D32323120496E76BE
:10428000616C696420657874727564657220004D94
:1042900032313820496E76616C69642065787472B9
:1042A0007564657220004D32303020496E76616C45
:1042B0006964206578747275646572200052657057
:1042C0006F7274696E6720656E6473746F702073AB
:1042D0007461747573004649524D574152455F4EA3
:1042E000414D453A4D61726C696E2056312E302E2B
:1042F000323B20537072696E7465722F6772626C04
:10430000206D617368757020666F722067656E3608
:10431000204649524D574152455F55524C3A6874B8
:104320007470733A2F2F6769746875622E636F6DAE
:104330002F707275736133642F50727573612D69BC
:10434000332D506C75732F2050524F544F434F4CA8
:104350005F56455253494F4E3A312E30204D41431E
:1043600048494E455F545950453A50727573612023
:104370006933204D4B322045585452554445525FC5
:10438000434F554E543A3120555549443A30303018
:1043900030303030302D303030302D303030302D26
:1043A000303030302D303030303030303030303010
:1043B000300A004D31303920496E76616C696420D5
:1043C000657874727564657220004D31303520490E
:1043D0006E76616C696420657874727564657220AC
:1043E000004D31303420496E76616C696420657807
:1043F00074727564657220004C6F736572207075FD
:104400006C6C6579004B6F6C6F207061736F7765B2
:1044100000506F6C6561207375656C746100507538
:104420006C6567676961206C656E74610055766FB5
:104430006C6E656E612072656D656E69636B61009F
:104440004C6F6F73652070756C6C65790046696C94
:10445000616D656E74206C6164656E0046696C61A7
:104460006D656E74206C6164656E005770726F7755
:1044700061647A2066696C616D656E7400496E7462
:10448000726F64756369722066696C616D2E00439A
:1044900061726963612066696C616D656E746F003D
:1044A0005A61766573742066696C616D656E74001F
:1044B0004C6F61642066696C616D656E74004C615F
:1044C0006164652046696C616D656E740046696C57
:1044D000616D656E74206C61656474005770726FF5
:1044E000772E2066696C616D656E747500496E7417
:1044F000726F64756369656E646F2066696C616D67
:104500002E004361726963616E646F2066696C613D
:104510006D2E005A61766164656E692066696C6112
:104520006D656E7475004C6F6164696E67206669B5
:104530006C616D656E74004C61616465206B6C65C7
:104540007572004C61646520466172626500437A51
:1045500079737A637A2E206B6F6C6F72750043618A
:104560006D6269616E646F20636F6C6F720043618E
:10457000726963616E646F20636F6C6F7265004374
:10458000697374656E69206261727679004C6F613F
:1045900064696E6720636F6C6F72004B696573208E
:1045A0007461616C00576165686C6520537072615D
:1045B000636865005779626F72206A657A796B610A
:1045C0000043616D6269616520656C206964696F93
:1045D0006D610053656C657A696F6E61206C696E00
:1045E000677561005679626572206A617A796B61DC
:1045F0000053656C656374206C616E6775616765F7
:10460000004E656465726C616E6473004465757418
:1046100073636800506F6C736B6900457370616EF3
:104620006F6C004974616C69616E6F0043657374EF
:10463000696E6100456E676C697368004E4F4F4448
:1046400053544F502F4B494C4C45442E200041426F
:10465000474542524F4348454E2E2000504152415B
:10466000444120444520454D455247454E4349412C
:1046700000494E2054494C542E004B494C4C454463
:104680002E2000496E76616C6964206578747275BD
:104690006465720046696C616D656E7420696E7345
:1046A00074656B656E0046696C616D656E7420653E
:1046B000696E6C6567656E005770726F7761647ABA
:1046C0002066696C616D656E7400496E74726F640A
:1046D000756369722066696C616D656E746F0049FF
:1046E0006E7365726972652066696C616D656E7462
:1046F0006F00566C6F7A74652066696C616D656ECB
:104700007400496E736572742066696C616D656EC4
:1047100074002076616E20390020766F6E2039009B
:10472000207A2039002064652039002073752039F3
:1047300000207A203900206F662039004E6175779D
:104740006B65757269676865696420766572626514
:10475000746572656E2062696A206B616C69627251
:104760006174696570756E740047656E617569671F
:104770006B656974207665726265737365726E200D
:10478000626569204B616C69627269657270756EF1
:104790006B7400506F7072617769616D2070726523
:1047A00063797A796A6E6F73632070756E6B747556
:1047B000206B616C6962726163796A6E65676F0014
:1047C0004D656A6F72616E646F2063616D61207008
:1047D000756E746F2064652063616C6962726163D9
:1047E000696F6E0050657266657A696F6E2E20691A
:1047F0006C206C6574746F2070756E746F206469C2
:104800002063616C696272617A2E005A6C65707304
:10481000756A6920707265736E6F7374206B616C5A
:1048200069627261636E69686F20626F64750049C6
:104830006D70726F76696E67206265642063616C6B
:104840006962726174696F6E20706F696E74004B7B
:10485000616C6962726572656E205A004B616C69A9
:10486000627269657265205A004B616C696272758B
:104870006A65205A0043616C696272616E646F20E0
:104880005A0043616C696272616E646F205A004B1A
:10489000616C696272756A69205A0043616C696271
:1048A000726174696E67205A004B616C6269627252
:1048B00061746965204F4B004B616C696272696578
:1048C00072756E67204F4B004B616C696272616359
:1048D0006A61204F4B0043616C6962726163696F6A
:1048E0006E204F4B0043616C696272617A696F6E32
:1048F00065204F4B004B616C696272616365204FAC
:104900004B0043616C6962726174696F6E20646F01
:104910006E65004B616C6962726572656E205A004B
:104920004B616C696272696572656E205A004B61F9
:104930006C696272756A205A0043616C69627261C7
:1049400072205A0043616C69627261205A004B61A7
:104950006C6962726F766174205A0043616C69629F
:1049600072617465205A004F707761726D656E20B8
:104970006B6C6161722E0041756667656865697A66
:10498000656E206B6C61722E0047727A616E69658C
:10499000204F4B2E0043616C656E74616D69656ECE
:1049A000746F2066696E616C2E0052697363616C6E
:1049B000642E20636F6D706C65746F005A6168724D
:1049C0006976616E69204F4B2E0048656174696E8F
:1049D0006720646F6E652E004F707761726D656E33
:1049E000004175666865697A656E0047727A616E26
:1049F00069652E2E2E0043616C656E74616E646F66
:104A00002E2E2E0052697363616C64616D656E7445
:104A10006F2E2E2E005A6168726976616E690048A9
:104A2000656174696E67002046726565204D656D2D
:104A30006F72793A20005072696E746572206973E2
:104A4000206E6F67206E6965742067656B616C69A5
:104A50006272656572642E20566F6C6720646520F3
:104A600068616E646C656964696E672C20686F6F3D
:104A700066647374756B2046697273742073746511
:104A800070732C207365637469652043616C69627F
:104A9000726174696F6E20666C6F772E0044657268
:104AA00020447275636B6572207775726465206E41
:104AB0006F6368206E69636874206B616C696272F1
:104AC000696572742E20426974746520666F6C6724
:104AD000656E205369652064656D2048616E64626F
:104AE0007563682C204B61706974656C204669722F
:104AF00073742073746570732C2041627363686EE5
:104B00006974742043616C6962726174696F6E20AC
:104B1000666C6F772E004472756B61726B61206EEC
:104B20006965207A6F7374616C61206A65737A635A
:104B30007A6520736B616C6962726F77616E612E4A
:104B40002050726F737A65206B6965726F7761634D
:104B50002073696520696E737472756B636A612C6A
:104B600020726F7A647A69616C205A61637A796E17
:104B7000616D792C20706F64726F7A647A69616CF0
:104B80002053656C66746573742E00496D70726590
:104B9000736F7261206E6F20657374612063616C46
:104BA00069627261646120746F64617669612E204C
:104BB000506F72206661766F722075736172206526
:104BC0006C206D616E75616C2C20656C206361706A
:104BD0006974756C6F2046697273742073746570A4
:104BE000732C2073656C656363696F6E2043616C21
:104BF0006962726174696F6E20666C6F772E005304
:104C000074616D70616E746520616E636F72612096
:104C10006E6F6E2063616C6962726174612E2053E5
:104C200069207072656761206469207365677569C2
:104C3000726520696C206D616E75616C652C2063F6
:104C4000617069746F6C6F205052494D492050411A
:104C50005353492C2073657A696F6E652064656CC7
:104C60006C612063616C696272617A696F6E652E36
:104C7000005469736B61726E61206E6562796C615C
:104C8000206A65737465207A6B616C6962726F76F5
:104C9000616E612E20506F73747570756A74652033
:104CA00070726F73696D20706F646C65206D616EDA
:104CB00075616C752C206B617069746F6C61205A22
:104CC0006163696E616D652C206F647374617665D4
:104CD0006320506F73747570206B616C69627261D0
:104CE00063652E005072696E74657220686173206E
:104CF0006E6F74206265656E2063616C69627261BB
:104D0000746564207965742E20506C65617365202C
:104D1000666F6C6C6F7720746865206D616E75616D
:104D20006C2C2063686170746572204669727374BC
:104D30002073746570732C2073656374696F6E20C3
:104D400043616C6962726174696F6E20666C6F7723
:104D50002E004475726368666C7573730050727AC6
:104D600065706C797700466C756A6F00466C757378
:104D7000736F00507275746F6B00466C6F770042F2
:104D800065776567696E67656E2061667765726BCA
:104D9000656E004265776567756E67656E20626552
:104DA000656E64656E004B6F6E637A656E69652033
:104DB0006472756B75005465726D2E206D6F766927
:104DC0006D69656E746F73004172726573746F20E4
:104DD000696E20636F72736F00446F6B6F6E636FE9
:104DE00076616E6920706F687962750046696E69D8
:104DF0007368696E67206D6F76656D656E7473009C
:104E00002076616E20340020766F6E203400207A88
:104E10002034002064652034002073752034002085
:104E20007A203400206F662034005A6F656B65204D
:104E3000626564206B616C6962726174696570752A
:104E40006E740053756368652042657474204B610D
:104E50006C69627269657270756E6B7400537A75F5
:104E60006B616D2070756E6B7475206B616C69621F
:104E7000726163796A6E65676F20706F646B6C61D5
:104E8000646B690042757363616E646F2063616D6A
:104E9000612070756E746F2064652063616C696257
:104EA000726163696F6E0052696365726361206449
:104EB000656C206C6574746F2070756E746F2064FF
:104EC000692063616C696272617A2E00486C656466
:104ED000616D206B616C69627261636E6920626FE3
:104EE0006420706F646C6F7A6B79005365617263D4
:104EF00068696E67206265642063616C69627261D3
:104F000074696F6E20706F696E74004865726861B5
:104F10006C696E672000576965646572686F6C75AF
:104F20006E6720004974657261636A612000526592
:104F3000697465726163696F6E200052656974659A
:104F400072617A696F6E652000497465726163658C
:104F50002000497465726174696F6E2000446F6E41
:104F60006520736176696E672066696C652E004402
:104F70006F6E65207072696E74696E672066696C09
:104F800065004973206B6C657572207A756976656A
:104F9000723F0049737420466172626520726569D0
:104FA0006E3F00437A79206B6F6C6F72206A657375
:104FB0007420637A797374793F00457320656C209F
:104FC0006E7565766F20636F6C6F72206E697469A1
:104FD000646F3F00496C20636F6C6F7265206527BA
:104FE000206E697469646F3F004A65206261727661
:104FF000612063697374613F00497320636F6C6F54
:105000007220636C6561723F0057697373656C2031
:1050100066696C616D656E740046696C616D656E84
:10502000742D5765636873656C0057796D69656E9B
:1050300069632066696C616D656E740043616D62C1
:105040006961722066696C616D656E746F004361A1
:105050006D622E2066696C616D656E746F005679A5
:105060006D656E69742066696C616D656E74004370
:1050700068616E67652066696C616D656E74004677
:10508000616E20736E656C68656964004C75656659
:105090007465722D54656D706F00507265646B6F2E
:1050A00073632077656E742E0056656C6F63696458
:1050B00061642056656E742E0056656C6F6369746A
:1050C000612076656E742E00527963686C6F73741C
:1050D0002076656E742E0046616E2073706565647F
:1050E00000656E717565696E67202200456B73748B
:1050F0007275646572004578747275736F720045DD
:1051000073747275736F7265004578747275646537
:1051100072002045787465726E616C20526573650B
:1051200074005072696E7465722073746F7070656C
:10513000642064756520746F206572726F72732EBF
:105140002046697820746865206572726F722061EC
:105150006E6420757365204D39393920746F207263
:105160006573746172742E202854656D7065726168
:10517000747572652069732072657365742E20538F
:105180006574206974206166746572207265737439
:10519000617274696E6729004E6F204C696E6520DC
:1051A0004E756D6265722077697468206368656307
:1051B0006B73756D2C204C617374204C696E653A6D
:1051C00020004E6F20436865636B73756D207769AF
:1051D0007468206C696E65206E756D6265722C2036
:1051E0004C617374204C696E653A200020746F6FB7
:1051F000206C6F6E6720657874727573696F6E20AE
:1052000070726576656E746564004C696E65204EDB
:10521000756D626572206973206E6F74204C6173C6
:1052200074204C696E65204E756D6265722B312C51
:10523000204C617374204C696E653A20005072698D
:105240006E7465722068616C7465642E206B696C85
:105250006C28292063616C6C6564210020636F6C8D
:105260006420657874727573696F6E2070726576EC
:10527000656E74656400636865636B73756D206D3E
:1052800069736D617463682C204C617374204C6980
:105290006E653A2000464F55543A004645484C4505
:1052A000523A00424C41443A004552524F52453A1C
:1052B0000043485942413A004552524F523A004544
:1052C0006E642066696C65206C697374006F70652C
:1052D0006E0054524947474552454400656E647319
:1052E000746F7073206869743A2000536C61706544
:1052F0006E2E2E2E0057617274656E2E2E2E004576
:105300006E2065737065726100536F7370656E73A4
:10531000696F6E652E2E2E00536C6565702E2E2ED5
:10532000004D6F746F72656E20756974004D6F74F7
:105330006F72656E206175730057796C61637A795D
:10534000632073696C6E696B69004170616761729B
:10535000206D6F746F726573004469736162696C6C
:105360006974206D6F746F7269005679706E6F7515
:1053700074206D6F746F72790044697361626C653B
:105380002073746570706572730041637475656530
:105390006C00416B7475656C6C65730054796C6B53
:1053A0006F20616B7475616C6E650041637475612B
:1053B0006C0041747475616C6500506F757A65207E
:1053C000616B7475616C6E690043757272656E74A1
:1053D0000020436F756E7420583A2000576973732C
:1053E000656C206F6B3F005765636873656C206F59
:1053F0006B3F0057796D69616E61206F6B3F0043B1
:10540000616D626961646F20636F72726563742E8F
:105410003F0043616D626961746F20636F72722E29
:105420003F0056796D656E61206F6B3F0043686188
:105430006E67656420636F72726563746C793F0098
:1054400041666B6F656C656E0041626B7565686C7B
:10545000656E00577963686C6F647A696300456EA6
:1054600066726961720052616666726564646100A9
:105470005A63686C6164697400436F6F6C646F7722
:105480006E005265696E696720686574207475697D
:105490007420766F6F72206465206B616C69627234
:1054A00061746965206175622E204B6C696B2061A7
:1054B0006C73206B6C6161722E004269747465209C
:1054C0007265696E6967656E2053696520646965F8
:1054D000204475657365207A7572204B616C696232
:1054E00072696572756E672E204B6C69636B656EB1
:1054F0002077656E6E207361756265722E00446C54
:1055000061207072617769646C2E206B616C6962D6
:105510007261636A692070726F737A65206F637A53
:105520007973636963206479737A652E20506F7490
:10553000772E2067757A696B69656D2E004C696DF1
:105540007069617220626F7175696C6C6120706145
:1055500072612063616C6962726163696F6E2E2093
:10556000436C69636B206375616E646F2061636176
:105570006265732E0050756C697265206C277567C3
:10558000656C6C6F20706572206C612063616C6962
:105590006272617A696F6E652C20706F6920666136
:1055A000726520636C69636B2E0050726F20757397
:1055B0007065736E6F75206B616C6962726163698F
:1055C000206F636973746574652070726F73696DA1
:1055D000207469736B6F766F7520747279736B7555
:1055E0002E20506F74767264746520746C616369E8
:1055F000746B656D2E00506C6561736520636C651E
:10560000616E20746865206E6F7A7A6C6520666FB3
:10561000722063616C6962726174696F6E2E2043DF
:105620006C69636B207768656E20646F6E652E0011
:105630005A696A6E206265696465205A20776167DD
:10564000656E206865656C656D61616C20626F7662
:10565000656E3F0053696E64206265696465205A17
:10566000205363686C697474656E2067616E7A207C
:105670006F62656E3F004F626120776F7A6B6920C1
:10568000646F6A656368616C7920646F20676F720C
:105690006E656A2072616D793F00436172726F734B
:1056A000205A20697A712E2F6465722E20657374DA
:1056B000616E20617272696261206D6178696D6FDF
:1056C0003F00492063617272656C6C69205A2073D7
:1056D000696E2F64657320736F6E6F20616C7465E3
:1056E0007A7A61206D61783F00446F6A656C792039
:1056F0006F6261205A20766F7A696B79206B7E68C1
:105700006F726E696D7520646F72617A753F0041CA
:105710007265206C65667420616E642072696768CA
:1057200074205A7E63617272696167657320616C6F
:105730006C2075703F00204C61737420557064615B
:105740007465643A20004B696573204578747275FE
:1057500064657200576165686C656E2053696520E9
:105760004578747275646572005779626965727AFA
:1057700020656B7374727564657200456C6567694A
:1057800072206578747275736F723A0053656C6538
:105790007A696F6E61206573747275736F72653AA2
:1057A00000567962657274652065787472756465F7
:1057B000723A0043686F6F73652065787472756420
:1057C00065723A0057697373656C2073756363651E
:1057D00073766F6C21005765636873656C20657222
:1057E000666F6C677265696368210057796D6961DE
:1057F0006E61206F6B210043616D62696F20636F82
:1058000072726563746F0043616D62696F207269C3
:1058100075736369746F21005A6D656E61207573CD
:105820007065736E6121004368616E6765207375F2
:10583000636365737321005072696E742076616EC4
:1058400020534400447275636B656E20766F6E2042
:105850005344004472756B207A205344004D656EAA
:1058600075207461726A65746120534400537461D9
:105870006D7061206461205344005469736B207A19
:10588000205344005072696E742066726F6D20530D
:10589000440050494E44412054656D702E206B6188
:1058A0006C2E0050494E44412054656D702E204BA3
:1058B000616C2E00436965706C6E61206B616C6970
:1058C00062722E0043616C6962726163696F6E205F
:1058D00074656D702E00546172617475726120740C
:1058E000656D702E005465706C6F742E206B616C4A
:1058F0006962726163650050494E44412054656D90
:10590000702E2063616C2E0050494E444120546536
:105910006D702E206B616C2E0050494E4441205416
:10592000656D702E204B616C2E00536B616C69624B
:10593000726F7761630043616C69627261720043E8
:10594000616C696272617265005A6B616C69627246
:105950006F7661740050494E44412054656D702E3D
:105960002063616C2E0052657365742058595A206B
:105970006B616C6962722E005265736574205859B0
:105980005A204B616C6962722E00526573657420F7
:105990006B616C6962722E2058595A0052657365AA
:1059A000742058595A206B616C6962722E005265DE
:1059B0007365742058595A2063616C6962722E00B5
:1059C0004B616C696272617469652058595A004B69
:1059D000616C696272696572756E672058595A0008
:1059E0004B616C69627261636A612058595A004365
:1059F000616C696272612058595A0043616C696236
:105A000072612058595A004B616C6962726163651A
:105A10002058595A0043616C69627261746520585C
:105A2000595A002042726F776E206F75742052654C
:105A300073657400426567696E2066696C65206CE9
:105A40006973740058595A206B616C696272617491
:105A50006965206765636F6D70726F6D69747465D9
:105A60006572642E204C696E6B73766F6F72206B5B
:105A7000616C6962726174696570756E74206E69BB
:105A800065742062657265696B626161722E00588F
:105A9000595A2D4B616C696272696572756E672027
:105AA000756E67656E61752E204C696E6B65722030
:105AB000766F726465726572204B616C696272699F
:105AC000657270756E6B74206E69636874206572A0
:105AD00072656963686261722E004B616C69627203
:105AE00061636A612058595A206E6965646F6B6CF6
:105AF00061646E612E204C6577792070727A6564DE
:105B00006E692070756E6B74207A62797420777973
:105B100073756E6965747920646F2070727A6F6432
:105B2000752E0043616C696272617A696F6E2058EC
:105B3000595A20636F6D70726F6D65746964612E60
:105B40002050756E746F2064656C616E7465726F41
:105B500020697A7175696572646F206E6F20616C5F
:105B600063616E7A61626C652E0043616C6962727A
:105B7000617A696F6E652058595A20636F6D707233
:105B80006F6D657373612E2050756E746F20616E3A
:105B9000746572696F72652073696E697374726F70
:105BA000206E6F6E207261676769756E67696269E2
:105BB0006C652E004B616C69627261636520585997
:105BC0005A206E65707265736E612E204C65767911
:105BD00020707265646E6920626F64206D6F63204F
:105BE0007670726564752E0058595A2063616C692D
:105BF00062726174696F6E20636F6D70726F6D6930
:105C00007365642E204C6566742066726F6E742016
:105C100063616C6962726174696F6E20706F696E26
:105C200074206E6F7420726561636861626C652EAA
:105C30000058595A206B616C696272617469652001
:105C40006765636F6D70726F6D697474656572649A
:105C50002E20566F6F727A696A6465206B616C6979
:105C600062726174696570756E74656E206E6965C7
:105C7000742062657265696B626161722E005859A9
:105C80005A2D4B616C696272696572756E67207519
:105C90006E67656E61752E20566F72646572652041
:105CA0004B616C69627269657270756E6B746520A8
:105CB0006E69636874206572726569636862617297
:105CC0002E004B616C6962722E2058595A206E6901
:105CD00065646F6B6C61646E612E2050727A6564CE
:105CE0006E69652070756E6B7479206B616C69628A
:105CF000722E205A627974207779732E20646F2077
:105D000070727A6F64752E0043616C696272617A99
:105D1000696F6E2058595A20636F6D70726F6D6590
:105D2000746964612E2050756E746F2064656C61B7
:105D30006E7465726F73206E6F20616C63616E7A32
:105D400061626C65732E0043616C696272617A698D
:105D50006F6E652058595A20636F6D70726F6D6554
:105D60007373612E2050756E746920616E74657254
:105D7000696F7269206E6F6E207261676769756EF8
:105D8000676962696C692E004B616C69627261635C
:105D9000652058595A206E65707265736E612E20A9
:105DA000507265646E69206B616C69627261636ECA
:105DB0006920626F6479206D6F632076707265640C
:105DC000752E0058595A2063616C6962726174695A
:105DD0006F6E20636F6D70726F6D697365642E20D6
:105DE00046726F6E742063616C6962726174696F70
:105DF0006E20706F696E7473206E6F7420726561AF
:105E0000636861626C652E0058595A206B616C6939
:105E1000627261746965206F6B2E20582F592D6155
:105E20007373656E207A696A6E2069657473207376
:105E300063686565662E2053636865656668656995
:105E40006420776F726474206175746F6D6174691A
:105E5000736368206765636F7272696765657264F2
:105E60002E20476F65642067656461616E2100586C
:105E7000595A2D4B616C696272696572756E672043
:105E80006F6B2E20582F592D41636873656E2073F8
:105E9000696E6420657477617320736368696566F1
:105EA0002E20536368696566686569742077697236
:105EB00064206175746F6D617469736368206B6FC2
:105EC00072726967696572742E2047757420676500
:105ED0006D6163687421004B616C69627261636A11
:105EE000612058595A207072617769646C6F7761CC
:105EF0002E204F73696520582F59206C656B6B6F8E
:105F000020736B6F736E652E20446F627261207216
:105F10006F626F7461210043616C696272616369D1
:105F20006F6E2058595A20636F7272656374612EC8
:105F3000204C6F7320656A65732058202F205920EC
:105F4000657374616E206C69676572616D656E74EE
:105F50006520696E636C696E61646F732E20427593
:105F6000656E2074726162616A6F210043616C69C1
:105F70006272617A696F6E2058595A20636F72722B
:105F8000657474612E204173736920582F59206CF9
:105F900065676765726D656E74652073746F727482
:105FA000692E2042656E20666174746F21004B611A
:105FB0006C6962726163652058595A207620706F4F
:105FC0007261646B752E20582F59206F7379206D84
:105FD00069726E65207A6B6F73656E652E20446FF3
:105FE000627261207072616365210058595A2063A2
:105FF000616C6962726174696F6E20616C6C207291
:10600000696768742E20582F592061786573206164
:10601000726520736C696768746C7920736B65773F
:1060200065642E20476F6F64206A6F6221005859A3
:106030005A206B616C69627261746965206F6B2EA6
:1060400020582F592D617373656E207A696A6E200E
:106050006865656C207363686565662E20536368A8
:106060006565666865696420776F72647420617520
:10607000746F6D617469736368206765636F7272B2
:106080006967656572642E0058595A2D4B616C69B9
:106090006272696572756E67206F6B2E20582F597A
:1060A0002D41636873656E2073696E642073656843
:1060B00072207363686965662E205363686965663C
:1060C000686569742077697264206175746F6D61A9
:1060D0007469736368206B6F727269676965727443
:1060E0002E004B616C69627261636A612058595A73
:1060F000207072617769646C6F77612E20536B6FCB
:1061000073792062656461206175746F6D61747963
:10611000637A6E6965207779726F776E616E65203C
:1061200070727A79206472756B752E0043616C69A8
:1061300062726163696F6E2058595A20636F727280
:10614000656374612E204C6120696E636C696E61B9
:1061500063696F6E20736520636F72726567697221
:1061600061206175746F6D61746963616D656E74D2
:10617000652E0043616C696272617A696F6E2058A6
:10618000595A20636F7272657474612E204C6120BD
:10619000646973746F7273696F6E6520766572726D
:1061A0006127206175746F6D61746963616D656EDF
:1061B000746520636F6D70656E736174612E004B42
:1061C000616C6962726163652058595A207620704B
:1061D0006F7261646B752E205A6B6F73656E6920E8
:1061E00062756465206175746F6D617469636B7944
:1061F000207679726F766E616E6F2070726920748E
:1062000069736B752E0058595A2063616C6962720C
:106210006174696F6E20616C6C2072696768742E9E
:1062200020536B65772077696C6C20626520636F03
:1062300072726563746564206175746F6D617469F1
:1062400063616C6C792E0058595A206B616C6962DD
:106250007261746965206D69736C756B742E204270
:106260006564206B616C6962726174696570756EDA
:1062700074206E696574206765766F6E64656E2E36
:106280000058595A2D4B616C696272696572756E5E
:1062900067206665686C67657363686C6167656EC7
:1062A0002E20426574742D4B616C6962726965724F
:1062B00070756E6B74206E696368742067656675AF
:1062C0006E64656E2E004B616C6962722E205859A7
:1062D0005A206E69657564616E612E204B616C6930
:1062E00062726163796A6E792070756E6B7420706A
:1062F0006F646B6C61646B69206E69657A6E616C4A
:10630000657A696F6E792E0043616C6962726163B0
:10631000696F6E2058595A2066616C6C6164612EF9
:106320002050756E746F732064652063616C6962C0
:10633000726163696F6E20656E206C612063616DB0
:1063400061206E6F20656E636F6E747261646F732F
:106350002E0043616C696272617A696F6E652058C4
:10636000595A2066616C6C6974612E20496C2070EA
:10637000756E746F2064692063616C696272617A02
:10638000696F6E652073756C206C6574746F206E18
:106390006F6E20652720737461746F2074726F763E
:1063A00061746F2E004B616C696272616365205885
:1063B000595A2073656C68616C612E204B616C6961
:1063C000627261636E6920626F6420706F646C6FCB
:1063D0007A6B79206E656E616C657A656E2E0058F9
:1063E000595A2063616C6962726174696F6E2066CC
:1063F00061696C65642E204265642063616C69622A
:10640000726174696F6E20706F696E74207761734A
:10641000206E6F7420666F756E642E0058595A2076
:106420006B616C69627261746965206F6B2E2058B4
:106430002F592D617373656E20737461616E2070C6
:10644000657270656E646963756C6169722E204750
:106450006566656C69636974656572642100585985
:106460005A2D4B616C696272696572756E67206F37
:106470006B2E20582F592D41636873656E20736908
:106480006E642073656E6B7265636874207A7565DF
:10649000696E616E6465722E20476C7565636B77FB
:1064A000756E73636821004B616C69627261636A27
:1064B000612058595A206F6B2E204F736965205800
:1064C0002F592073612070726F73746F7061646CE8
:1064D000652E2047726174756C61636A65210043A3
:1064E000616C6962726163696F6E2058595A206FDE
:1064F0006B2E20456A657320582F59207065727085
:10650000656E646963756C617265732E2046656C97
:10651000696369746163696F6E6573210043616CBF
:10652000696272617A696F6E652058595A204F4BC3
:106530002E20476C69206173736920582F5920738E
:106540006F6E6F2070657270656E6469636F6C61E9
:1065500072692E20436F6D706C696D656E74692170
:10656000004B616C6962726163652058595A2076EC
:1065700020706F7261646B752E20582F59206F73D5
:1065800079206A736F75206B6F6C6D652E20477272
:106590006174756C756A69210058595A2063616C81
:1065A0006962726174696F6E206F6B2E20582F596B
:1065B0002061786573206172652070657270656E08
:1065C000646963756C61722E20436F6E67726174CB
:1065D000756C6174696F6E73210058595A206B6134
:1065E0006C69627261746965206D69736C756B7436
:1065F0002E2052616164706C656567206465206857
:10660000616E646C656964696E672E0058595A2D15
:106610004B616C696272696572756E672066656848
:106620006C67657363686C6167656E2E2042697480
:106630007465207363686175656E205369652069B0
:106640006E206461732048616E64627563682E0019
:106650004B616C69627261636A612058595A206E9D
:106660006965706F776965647A696F6E612E205312
:1066700070726177647A6963207720696E737472CF
:10668000756B636A692E0043616C6962726163694C
:106690006F6E2058595A2066616C6C6164612E20BF
:1066A000436F6E73756C74617220656C206D616EE2
:1066B00075616C20706F72206661766F722E004378
:1066C000616C696272617A696F6E652058595A20EF
:1066D00066616C6C6974612E205369207072656705
:1066E0006120646920636F6E73756C7461726520DC
:1066F000696C206D616E75616C652E004B616C6913
:1067000062726163652058595A2073656C68616CC8
:10671000612E204E61686C65646E65746520646FDF
:10672000206D616E75616C752E0058595A20636139
:106730006C6962726174696F6E206661696C656410
:106740002E20506C6561736520636F6E73756C7479
:1067500020746865206D616E75616C2E0058595A01
:10676000206B616C69627261746965206D69736C1C
:10677000756B742E204C696E6B73766F6F72206B25
:10678000616C6962726174696570756E74206E699E
:1067900065742062657265696B626161722E005872
:1067A000595A2D4B616C696272696572756E67200A
:1067B0006665686C67657363686C6167656E2E20DB
:1067C0004C696E6B657220766F6465726572204BE2
:1067D000616C69627269657270756E6B74206E6946
:1067E00063687420657272656963686261722E0005
:1067F0004B616C6962722E2058595A206E6965751A
:1068000064616E612E204C6577792070727A6564C0
:106810006E692070756E6B74207A62797420646F73
:106820002070727A6F64752E205779726F776E615F
:1068300063206472756B61726B652E0043616C69D5
:1068400062726163696F6E2058595A2066616C6C80
:1068500061642E2050756E746F2064656C616E7477
:1068600065726F20697A7175696572646F206E6FE9
:1068700020616C63616E7A61626C652E0043616CAD
:10688000696272617A696F6E652058595A20666133
:106890006C6C6974612E2050756E746F20616E741B
:1068A0006572696F72652073696E697374726F20A7
:1068B0006E6F6E207261676769756E676962696C79
:1068C000652E004B616C6962726163652058595A8C
:1068D0002073656C68616C612E204C657679207040
:1068E0007265646E6920626F64206D6F63207670DC
:1068F000726564752E2053726F766E656A746520BA
:106900007469736B61726E752E0058595A206361F9
:106910006C6962726174696F6E206661696C65642E
:106920002E204C6566742066726F6E742063616CF5
:106930006962726174696F6E20706F696E74206E27
:106940006F7420726561636861626C652E005859CE
:106950005A206B616C69627261746965206D69733C
:106960006C756B742E20566F6F727A696A6465203D
:106970006B616C6962726174696570756E74656E65
:10698000206E6965742062657265696B626161720F
:106990002E0058595A2D4B616C6962726965727587
:1069A0006E67206665686C67657363686C616765B0
:1069B0006E2E20566F7264657265204B616C696241
:1069C0007269657270756E6B7465206E6963687448
:1069D00020657272656963686261722E004B616C3A
:1069E0006962722E2058595A206E69657564616E0D
:1069F000612E2050727A65642E2070756E6B7479EA
:106A0000206B616C6962722E207A62797420646FE7
:106A10002070727A6F64752E205779726F776E616D
:106A200063206472756B61726B652E0043616C69E3
:106A300062726163696F6E2058595A2066616C6C8E
:106A400061642E2050756E746F2064656C616E7485
:106A500065726F73206E6F20616C63616E7A616224
:106A60006C65732E0043616C696272617A696F6E46
:106A7000652058595A2066616C6C6974612E2050EB
:106A8000756E746920616E746572696F7269206ECB
:106A90006F6E207261676769756E676962696C699C
:106AA0002E004B616C6962726163652058595A20EF
:106AB00073656C68616C612E20507265646E69202C
:106AC0006B616C69627261636E6920626F647920C8
:106AD0006D6F63207670726564752E2053726F76C9
:106AE0006E656A7465207469736B61726E752E00D1
:106AF00058595A2063616C6962726174696F6E20C3
:106B00006661696C65642E2046726F6E74206361E5
:106B10006C6962726174696F6E20706F696E7473F4
:106B2000206E6F7420726561636861626C652E000F
:106B3000426564206E6976656C6C6572696E67206B
:106B40006D69736C756B742E53656E736F72206E06
:106B50006965742061616E6765736C6F74656E2022
:106B60006F66206B6162656C20676562726F6B6532
:106B70006E2E5761636874206F7020726573657440
:106B800000426574742D4E6976656C6C696572752A
:106B90006E67206665686C67657363686C616765BE
:106BA0006E2E2053656E736F72206E696368742059
:106BB000616E67657363686C6F7373656E206F6475
:106BC0006572204B6162656C20646566656B742E2E
:106BD0002057617274652061756620526573657413
:106BE0002E004B616C69627261636A61206E696537
:106BF0007564616E612E2053656E736F72206F64D1
:106C00006C61637A6F6E79206C75622075737A6B34
:106C10006F647A2E206B6162656C2E20437A656BFF
:106C2000616D206E612072657365742E004E697609
:106C3000656C6163696F6E2066616C6C6164612E66
:106C40002053656E736F7220646573636F6E656346
:106C50007461646F206F206361626C65732064618E
:106C60006E61646F732E204573706572616E646F20
:106C70002072657365742E004C6976656C6C616D6D
:106C8000656E746F206C6574746F2066616C6C69DE
:106C9000746F2E2053656E736F7265206469736321
:106CA0006F6E2E206F204361766F2044616E6E2ED2
:106CB00020496E2061747465736120646920726577
:106CC0007365742E004B616C696272616365205A52
:106CD0002073656C68616C612E2053656E736F72F2
:106CE000206A65206F64706F6A656E79206E6562D8
:106CF0006F20707265727573656E79206B61626565
:106D00006C2E2043656B616D206E6120726573652A
:106D1000742E00426564206C6576656C696E672030
:106D20006661696C65642E2053656E736F722064B2
:106D30006973636F6E6E6563746564206F72206340
:106D400061626C652062726F6B656E2E205761699F
:106D500074696E6720666F722072657365742E00A9
:106D6000426564206E6976656C6C6572696E672039
:106D70006D69736C756B742E2053656E736F722022
:106D8000776173206E6965742067656163746976E5
:106D9000656572642E205675696C206F70206E6F69
:106DA0007A7A6C653F205761636874206F70207237
:106DB000657365742E00426574742D4E6976656C3A
:106DC0006C696572756E67206665686C676573636C
:106DD000686C6167656E2E2053656E736F722077E5
:106DE00075726465206E6963687420617573676588
:106DF0006C6F6573742E205363686D75747A696760
:106E0000652044756573653F205761727465206124
:106E100075662052657365742E004B616C696272F1
:106E200061636A61206E69657564616E612E2053CD
:106E3000656E736F72206E696520646F746B6E612E
:106E40006C2E205A616E6965637A79737A2E20649C
:106E500079737A613F20437A656B616D206E6120A2
:106E600072657365742E004E6976656C6163696F37
:106E70006E2066616C6C6164612E2053656E736F69
:106E800072206E6F2066756E63696F6E612E20458D
:106E900073636F6D62726F7320656E20426F7175E0
:106EA000692E3F204573706572616E646F20726554
:106EB0007365742E004C6976656C6C616D656E74DB
:106EC0006F206C6574746F2066616C6C69746F2ED2
:106ED0004E6F5269737053656E736F722052657393
:106EE00069647569207375207567656C6C6F3F20E8
:106EF000496E2061747465736120646920726573E2
:106F000065742E004B616C696272616365205A2062
:106F100073656C68616C612E2053656E736F7220AF
:106F20006E657365706E756C2E205A6E656369733D
:106F300074656E6120747279736B613F2043656B79
:106F4000616D206E612072657365742E0042656408
:106F5000206C6576656C696E67206661696C656436
:106F60002E2053656E736F72206469646E74207492
:106F70007269676765722E20446562726973206F5B
:106F80006E206E6F7A7A6C653F2057616974696E06
:106F90006720666F722072657365742E00426564A7
:106FA000206E6976656C6C6572696E67206D6973B9
:106FB0006C756B742E2045656E2073656E736F72F1
:106FC00020686565667420746520686F6F67206748
:106FD0006574726967676572642E205761636874AF
:106FE000206F702072657365742E00426574742D75
:106FF0004E6976656C6C696572756E67206665684A
:107000006C67657363686C6167656E2E2053656E8F
:10701000736F72207775726465207A7520686F636C
:10702000682061757367656C6F6573742E20576196
:10703000727465206175662052657365742E004B0D
:10704000616C69627261636A61205A206E6965755C
:1070500064616E612E2053656E736F7220646F746D
:107060006B2E207A61207779736F6B6F2E20437AB5
:10707000656B616D206E612072657365742E004EC4
:107080006976656C6163696F6E2066616C6C6164C2
:10709000612E2053656E736F722066756E63696F23
:1070A0006E612064656D61736961646F2074656DE4
:1070B0007072616E6F2E204573706572616E646FC1
:1070C0002072657365742E004C6976656C6C616D19
:1070D000656E746F206C6574746F2066616C6C698A
:1070E000746F2E526973702073656E736F726520B2
:1070F00074726F70706F2070726573746F496E2058
:107100006174746573612064692072657365742E9F
:10711000004B616C696272616365205A2073656C13
:1071200068616C612E2053656E736F722073657099
:107130006E756C207072696C6973207679736F6BF1
:107140006F2E2043656B616D206E612072657365E3
:10715000742E00426564206C6576656C696E6720EC
:107160006661696C65642E2053656E736F7220745E
:10717000726967676572656420746F6F20686967FC
:10718000682E2057616974696E6720666F7220727D
:10719000657365742E00426564206F707761726D4F
:1071A000656E0042657474206175666865697A650C
:1071B0006E0047727A616E69652073746F6C696BDB
:1071C000612E2E0043616C656E74616E646F2042A7
:1071D0006173650052697363616C642E206C657421
:1071E000746F005A6168726976616E6920626564C5
:1071F000004265642048656174696E670042656499
:10720000204F4B2E0042657474204F4B0053746F17
:107210006C696B204F4B2E00426173652070726564
:107220007061726164610050696174746F2066619D
:1072300074746F2E00426564204F4B2E00426564CB
:1072400020646F6E6500526563687473202020208F
:107250005B756D5D00526563687473202020205B50
:10726000756D5D005720707261776F205B756D5D85
:1072700000446572656368612020205B756D5D0068
:10728000446573747261202020205B756D5D00562B
:10729000707261766F205B756D5D0052696768740E
:1072A00020736964655B756D5D005A757275656301
:1072B0006B7365747A656E00526573657400416323
:1072C00068746572202020205B756D5D0048696ED2
:1072D00074656E202020205B756D5D00446F207406
:1072E000796C7520205B756D5D004174726173204F
:1072F000202020205B756D5D00526574726F202028
:107300002020205B756D5D00567A61647520205BDE
:10731000756D5D00526561722073696465205B75EF
:107320006D5D00426564206A75697374004265741E
:1073300074206C6576656C206B6F7272656B74007F
:107340004B6F72656B746120706F646B6C61646B02
:107350006900436F72722E206465206C6120636146
:107360006D6100436F7272657A2E206C69762E6CA7
:107370006574746F004B6F72656B636520706F642A
:107380006C6F7A6B7900426564206C6576656C2061
:10739000636F7272656374004C696E6B732020209A
:1073A00020205B756D5D004C696E6B732020202082
:1073B000205B756D5D0057206C65776F20205B75D5
:1073C0006D5D00497A71756965726461205B756DE8
:1073D0005D0053696E697374726120205B756D5D29
:1073E00000566C65766F20205B756D5D004C6566A0
:1073F000742073696465205B756D5D00566F6F72F4
:107400007275697420205B756D5D00566F726E65D4
:1074100020202020205B756D5D00446F2070727A03
:107420006F6475205B756D5D004164656C616E74A1
:107430006520205B756D5D0046726F6E746520205F
:1074400020205B756D5D00567072656475205B75FC
:107450006D5D0046726F6E7420736964655B756D57
:107460005D00426574740053746F6C696B00426117
:107470007365004C6574746F004265640041667307
:1074800074616E642074757373656E207469702006
:1074900076616E20686574207475697420656E204D
:1074A000686574207072696E74206F707065727692
:1074B0006C616B206E6F67206E69657420766173F6
:1074C0007467657374656C642E20566F6C672064F6
:1074D000652068616E646C656964696E672C20461E
:1074E000697273742073746570732C207365637490
:1074F0006965204669727374206C617965722063D6
:10750000616C6962726174696F6E2E0044657220ED
:1075100041627374616E64207A7769736368656E23
:107520002064657220537069747A652064657220E6
:10753000447565736520756E6420646572204472BD
:1075400075636B6F626572666C6165636865202F39
:10755000204265747420697374206E6F6368206EB6
:10756000696368742065696E67657374656C6C74B3
:107570002E20426974746520666F6C67656E2053B7
:1075800069652064656D2048616E64627563682C6E
:107590002046697273742073746570732C20416285
:1075A0007363686E697474204669727374206C61C9
:1075B0007965722063616C6962726174696F6E2EA5
:1075C000004F646C65676C6F7363206479737A79BC
:1075D000206F6420706F646B6C61646B69206E69EE
:1075E00065206A65737420736B616C6962726F7772
:1075F000616E612E20506F73746570756A207A67B2
:107600006F646E6965207A20696E737472756B633E
:107610006A6120726F7A647A69616C205A61637A58
:10762000796E616D792C20706F64726F7A647A69FB
:10763000616C204B616C69627261636A6120706980
:10764000657277737A656A20776172737477792EC1
:107650000044697374616E63696120656E7472655C
:10766000206C612070756E7461206465206C6120EF
:10767000626F7175696C6C612079206C6120737523
:107680007065726669636965206465206C6120635A
:10769000616D61206E6F2066696A61646120617549
:1076A0006E2E20506F72206661766F72207369674C
:1076B0006120656C206D616E75616C2C206361705A
:1076C0006974756C6F204669727374207374657089
:1076D000732C2073656363696F6E204669727374DF
:1076E000206C617965722063616C69627261746992
:1076F0006F6E2E0044697374616E7A6120747261DA
:10770000206C612070756E74612064656C6C2775E7
:1077100067656C6C6F2065206C6120737570657295
:1077200066696369652064656C206C6574746F209C
:107730006E6F6E20616E636F726120696D706F7322
:1077400074612E205369207072656761206469201E
:107750007365677569726520696C206D616E75610E
:107760006C652C2063617069746F6C6F2046697260
:1077700073742073746570732C2073657A696F6EEF
:1077800065204669727374206C617965722063614B
:107790006C6962726174696F6E2E004E656E69204D
:1077A0007A6B616C6962726F76616E6120767A6461
:1077B000616C656E6F737420747279736B79206F6E
:1077C00064207469736B6F766520706F646C6F7A78
:1077D0006B792E20506F73747570756A74652070A4
:1077E000726F73696D20706F646C65206D616E756A
:1077F000616C752C206B617069746F6C61205A61CB
:1078000063696E616D652C206F6473746176656366
:10781000204E6173746176656E69207072766E6950
:10782000207672737476792E0044697374616E6386
:1078300065206265747765656E20746970206F6677
:1078400020746865206E6F7A7A6C6520616E6420A2
:107850007468652062656420737572666163652073
:10786000686173206E6F74206265656E2073657445
:10787000207965742E20506C6561736520666F6C8D
:107880006C6F7720746865206D616E75616C2C205B
:1078900063686170746572204669727374207374D2
:1078A0006570732C2073656374696F6E204669720E
:1078B0007374206C617965722063616C69627261B6
:1078C00074696F6E2E004C697665205A2061616E76
:1078D00070617373656E004C697665205A20656926
:1078E0006E7374656C6C656E00446F7374726F6A4E
:1078F000656E6965206F7379205A004D6963726FF8
:107900007061736F20456A65205A00436F6D706522
:107910006E73617A696F6E65205A00446F6C6164A2
:10792000656E69206F7379205A004C697665206115
:10793000646A757374205A0041646A757374696E61
:1079400067205A005374617274706F73697469654B
:10795000005374617274706F736974696F6E004C58
:107960006C6576617220616C206F726967656E006C
:1079700054726F7661206F726967696E6500417538
:10798000746F20686F6D6500207C20417574686F8E
:10799000723A2000416C6C6500416C6C6500577355
:1079A0007A7973746B6F00546F646F7300547574DD
:1079B00074690056736500416C6C004163746976AC
:1079C000652045787472756465723A2000B410A41D
:1079D000108F107C10681053103E10C810D010D8B3
:1079E00010E110E91005110111FE10FB10F710F461
:1079F00010F1100911111119117111671158114C61
:107A0000114111351129118F1267122F12FD11CE5C
:107A100011A4117D11FF12FF12ED12DB12FF12C72C
:107A200012B21281136D135A134713361323131016
:107A300013FB13EA13D813C713B813A513931379C1
:107A40001467145514421431141E140B148C14DED4
:107A500014D814D114C914C014B0149F14081508F4
:107A60001508150815F614E31408153E153E153EC5
:107A7000153E152C151A153E15B415A4159415842C
:107A800015731561154F152F161E160D16FC15EAE8
:107A900015D815C615AB1770173517F916C4167E0D
:107AA00016411662184D18381823180E18F917E9E0
:107AB00017BA18B218A6189A188E1883187718DCF7
:107AC00018D418DC18CC18C618DC18DC1840193289
:107AD00019231911190219F218E418721972196789
:107AE000196019721955194B197C19F319E519D335
:107AF00019C419B319A11990196D1A5B1A4C1A3BC4
:107B00001A281A171A061AD71AC91AB81AA81A99C7
:107B10001A8C1A7E1A431B361B251B171B0A1BF7D0
:107B20001AE51AA21B951B891B7B1B6E1B611B543C
:107B30001BAF1B181C0F1C061CFC1BF31BE31BDAE2
:107B40001B1E1C881C761C641C521C401C2E1C888E
:107B50001CF41CE21CD01CBE1CAC1C9A1CF41C6B3C
:107B60001D5A1D4A1D381D281D141D061DE61DD455
:107B70001DC01DAE1D9A1D8A1D7A1D421E381E2B6A
:107B80001E1D1E121E041EF71DAF1EA01E8F1E7D81
:107B90001E6D1E5A1E4B1EFF1EFF1EF01EE01EFF16
:107BA0001ECE1EBC1E621F531F471F3C1F2F1F21CE
:107BB0001F111F971F971F8B1F971F971F7D1F71E7
:107BC0001F0920FA1FED1FDB1FC91FB51FA41F25AA
:107BD0002025201E2025201720252025204F204F3E
:107BE000203D202B204F204F204F2096208E208993
:107BF0002079206F2069206120ED20E320D720C468
:107C000020B820AC209F20512140212B2117210694
:107C100021FA205121C621B421A321922180216C77
:107C2000215A2142222D2218220722F321E321D8B2
:107C3000219922992287227722992263225322F7BF
:107C400022F722E522D322F722BF22AA222D232DBA
:107C5000231F2313232D2307232D234B234B2341A2
:107C60002336234B234B234B23C323AE2399238853
:107C70002373236123532341242F241F240D24FB2A
:107C800023E823D423C024AE249E248C247A2467A2
:107C90002453243F252D251D250B25F924E624D228
:107CA00024BC25AA259A258A2578256525512540B5
:107CB000262E261B260926F725E225CE25BA26A83C
:107CC00026992689267726632652262C271A270CE2
:107CD000270227F026DE26CC266B276B275C274C55
:107CE000276B273E276B27AE27AE27A5279C27AEFD
:107CF000278A277827C027D227E527442836282B2C
:107D0000281A280D28FB27ED27512863287728E318
:107D100028D528C928B728A92895288728F128FE1A
:107D2000280C291A2930293B29B929A82996298301
:107D3000297229612951292F2A202A102AFB29EA90
:107D400029D829C829912A862A762A652A592A4EAD
:107D50002A3E2A9E2AC92AB82AC92AC92AA72AC974
:107D60002AC92AFD2AEC2AFD2AFD2ADB2AFD2AFD42
:107D70002A252B1A2B252B252B0F2B252B252B9238
:107D80002B822B722B5F2B4F2B402B312B032CF58F
:107D90002BE52BD12BC22BB02B9F2B332C332C3329
:107DA0002C332C332C232C112CB62CA12C8D2C7D78
:107DB0002C6B2C582C482C362D222D122DFD2CEE00
:107DC0002CDD2CC92C8C2D822D762D6A2D622D5800
:107DD0002D4A2D942DEA2DDB2DD32DC12DB32DA6AB
:107DE0002D9C2DF62D6B2E5B2E4C2E3B2E2D2E1CFE
:107DF0002E0D2E9B2F752F462F142FE92EAE2E7988
:107E00002E243010300730F32FEA2FDC2FCE2FAE88
:107E1000309C308A30773063304E30393021311326
:107E2000310231F230E330D230C3304D314D314D7B
:107E3000314D314D313F313131853185318531859C
:107E400031853170315B31ED31DD31CE31BD31AF56
:107E500031A9319A316B35E4345634AA331E338B51
:107E600032F9310136043648364836363627364838
:107E70003617360836A83699368E367C366E365F1B
:107E8000365136DB36D436CD36C436BE36B836B388
:107E9000364F373C372A3716370737F436E236D0B5
:107EA00037BF37AF379C378A3778376337F037EDCE
:107EB00037F037F037E937E437E037653850384086
:107EC000382B3816380138F33736391B39F338D8A0
:107ED00038BB3899387538923987397F3977396B9B
:107EE0003962395639D539CA39C239BA39AE39A5A4
:107EF000399939183A0D3A053AFD39F139E839DC42
:107F000039373A373A273A1F3A373A373A373AAA9F
:107F10003C543CE83B853B243BA73A403A7D3F2517
:107F20003FB73E523EEF3D703D093D264019400EA1
:107F3000400340FA3FED3FDE3F4240424030404286
:107F4000404240424042409A409040834077406CDB
:107F5000405F405440CA40C540BF40B940B440AD06
:107F600040A640F441CB418F4163412F410141D0B4
:107F700040734264425442454239422E4224427880
:107F8000428F42A642BD42D642B343CA43E1434078
:107F9000442D441E4411440544F8434044B044A0D9
:107FA000448F447D446B445C444D44264513450254
:107FB00045ED44DC44CD44BE448D457F456E455E71
:107FC000454E4543453745F145E445D345C145B4A4
:107FD00045A5459B4534462C4623461B4614460C76
:107FE0004601467A467A4671465C467A464E463C9B
:107FF0004683460247F246DF46CA46B846A646943E
:1080000046364731472B4725472047194712472F08
:10801000480B48E447C047934769473C479B488F14
:10802000488248754869485C484F480249F548E528
:1080300048D648C848B848A9485B494E49444939D8
:10804000492E4920491349CA49BC49AA4995498939
:1080500049774967491F4A154A044AF649EB49E1FD
:1080600049D849274AE44C714CFF4B8B4B164B9D2A
:108070004A364A7A4D734D6C4D664D5D4D524D7A80
:108080004DEC4DD94DC84DB64DA64D934D7F4D2469
:108090004E1F4E194E134E0E4E074E004EEB4ECC59
:1080A0004EA74E844E5D4E434E2A4E524F494F3B93
:1080B0004F2E4F244F164F0B4F5D4F6F4FF94FE927
:1080C0004FD44FBA4FA34F934F824F6F505E504ED5
:1080D000503C502A5019500950D750C850B950A997
:1080E000509A508C507F50E15009510951FF50F681
:1080F00050EC5009510951125122519851C251EC82
:10810000510A523D525C527652B852B152A952B8FD
:1081100052A3529B529552BF52CD52D252DC5218AA
:108120005318530953FF521853F552EB5279536ABF
:108130005359534A5339532D532153C953BA53B248
:1081400053AB539C5392538A53D1532D5422541200
:1081500054FF53F353E753DC537954705466545E21
:1081600054535449544054F655AA5575553D55FE3F
:1081700054BA5482540F57E956C2569A56765654FA
:108180005630563657B357A1578C577B57695754BB
:10819000574657275818580758F757EB57D657C41C
:1081A0005784587A586D585D58535844583758F783
:1081B00058E558D658C458B458A3589258555949F8
:1081C000593F5936592A5919590859AE599C59AE2F
:1081D00059AE598A5978596659155A075AFB59EFB9
:1081E00059E059CF59C059235A345AE85BB45B6AF5
:1081F0005B235BDA5A8F5A445AC35D885D475D083A
:108200005DC25C7E5C315CEB5FAE5F6C5F175FD71D
:108210005E6F5E085E0662BF6173612C61E260881A
:10822000602E60DF63A56352630863C662816247A4
:1082300062996561651D65DF64A7645E641C642ADC
:1082400067FC66BF66876650660C66DA650A69C3B6
:10825000687D683C68F0679F675D67F06AA26A6541
:108260006A2C6ADD6992694E69136DC56C786C2D54
:108270006CE26B816B306B4D6F046FB56E676E1A7D
:108280006EB66D606D53711171C8707F703F70EB89
:108290006F9D6FF171E371D471C471B271A3719666
:1082A000713D723572277218720D720572FD719BE5
:1082B000728F7280727172647255724672B872B83F
:1082C00072B872B872B872AA72B87214730873F97D
:1082D00072EA72DC72CD72BE72867375736373520A
:1082E0007340732D732373ED73E173D273C373B64D
:1082F00073A773987353744774387429741A740B82
:1083000074FC737974797473746E746774627479BD
:108310007429789B77F4765176C1750C757D742A33
:10832000791B790B79FB78E978D778C67838797E2C
:10833000797E7970795F797E79517944798879B7D6
:1083400079B379AD79A7799E7999799479BB794593
:108350007872656D65207370616E206F6620746839
:1083600065205A2076616C7565732100626F7474A4
:108370006F6D00746F700000506F696E74206865D7
:108380006967687420746F6F20736D616C6C3A203C
:10839000007269676874006C6566740000506F69EC
:1083A0006E7420776964746820746F6F20736D61D8
:1083B0006C6C3A2000002C20003A200046696E6167
:1083C0006C2063616C63756C6174656420626564C4
:1083D00020706F696E74200000793A000044697360
:1083E00074616E63652066726F6D206D696E3A0010
:1083F0000043616C63756C6174696F6E206F6620F9
:10840000746865206D616368696E6520736B65775C
:1084100020616E64206F6666736574206661696CA6
:1084200065642E00002C20003A200046696E616CC5
:10843000206D656173757265642062656420706F7C
:10844000696E74200000206661696C65642E204CA2
:108450006F776572696E67207A20746F20002C2018
:10846000697465726174696F6E2000496D70726F16
:1084700076696E672062656420706F696E74200093
:10848000002C207A002C20697465726174696F6E0B
:108490002000496D70726F76696E67206265642096
:1084A000706F696E742000006C6F7765722074685D
:1084B000616E20596D696E2E205920636F6F726452
:1084C000696E61746520636C616D70696E67207799
:1084D000617320757365642E0043616C696272611B
:1084E00074696F6E20706F696E742000417420593A
:1084F0005F4D494E5F504F53004174205930004941
:108500006D70726F76696E6720626564206F666653
:1085100073657420616E6420736B657700002C2096
:10852000002C200020004D65617375726564200089
:10853000002C200041646A757374656420706F7349
:108540006974696F6E3A2000002C20683A002C2074
:10855000646D61783A005061727469616C20706F6B
:10856000696E7420657374696D61746564207261ED
:108570006469757320746F6F20736D616C6C3A2041
:1085800000005061727469616C20706F696E7420B4
:108590006469616D6574657220746F6F20736D61BD
:1085A0006C6C3A2000746F70007269676874006CBC
:1085B000656674007269676874006C65667400743F
:1085C0006F70006661696C6564202D206E6F742089
:1085D000666F756E640A007269676874006C656620
:1085E0007400002C2000496E697469616C20706F02
:1085F000736974696F6E3A200066696E6420626503
:108600006420696E64756374696F6E2073656E7340
:108610006F7220706F696E74207A005920736561E3
:10862000726368696E672072616469757320686936
:1086300067686572207468616E20585F4D41582EDE
:1086400020436C616D70696E672077617320646F81
:108650006E652E005920736561726368696E6720CC
:10866000726164697573206C6F77657220746861DC
:108670006E20595F4D494E2E20436C616D70696EBE
:10868000672077617320646F6E652E0058207365D4
:1086900061726368696E67207261646975732068CE
:1086A0006967686572207468616E20585F4D415833
:1086B0002E20436C616D70696E6720776173206452
:1086C0006F6E652E005820736561726368696E670E
:1086D00020726164697573206C6F776572207468AD
:1086E000616E20585F4D494E2E20436C616D70695C
:1086F0006E672077617320646F6E652E005361761C
:10870000696E67206265642063616C69627261747E
:10871000696F6E20766563746F727320746F204585
:108720004550524F4D0050657270656E64696375B7
:108730006C6172697479005A65726F20706F696E2E
:108740007420636F7272656374696F6E3A005920AA
:10875000766563746F72206C656E6774683A005852
:1087600020766563746F72206C656E6774683A007A
:10877000203C20005741524E494E473A2046726FE6
:108780006E7420706F696E74206E6F7420726561F4
:10879000636861626C652E205920636F6F72646933
:1087A0006E6174653A000070745B315D3A007074FC
:1087B0005B305D3A00004D656173757265643A0027
:1087C0000063757272656E745F706F736974696F40
:1087D0006E5B5A5F415849535D3A0000637572728F
:1087E000656E745F706F736974696F6E5B595F411A
:1087F0005849535D3A000063757272656E745F701C
:108800006F736974696F6E5B585F415849535D3A85
:1088100000417420592D3400417420593000006308
:108820006E74725B315D3A0000636E74725B305D32
:108830003A00007665635F795B315D3A00007665EA
:10884000635F795B305D3A00007665635F785B312A
:108850005D3A00007665635F785B305D3A0056658F
:1088600063746F72733A2000497465726174696F42
:108870006E3A2000496E76616C69642062656420FE
:10888000636F7272656374696F6E206D6174726973
:10889000782E20526573657474696E6720746F203A
:1088A0006964656E746974792E00496E76616C69CD
:1088B000642062656420636F7272656374696F6EB1
:1088C000206D61747269782E20582F592061786567
:1088D0007320617265206661722066726F6D20621E
:1088E00065696E672070657270656E646963756C2A
:1088F00061722E00496E76616C6964206265642045
:10890000636F7272656374696F6E206D61747269F2
:10891000782E205368696674206F7574206F662006
:1089200072616E67652E005A65726F20706F696E96
:108930007420636F7272656374696F6E3A00496E7A
:1089400076616C69642062656420636F727265632E
:1089500074696F6E206D61747269782E204C656E3B
:10896000677468206F662074686520592076656397
:10897000746F72206F7574206F662072616E676508
:108980002E005920766563746F72206C656E677473
:10899000683A00496E76616C6964206265642063A0
:1089A0006F7272656374696F6E206D61747269783D
:1089B0002E204C656E677468206F66207468652091
:1089C0005820766563746F72206F7574206F66200F
:1089D00072616E67652E005820766563746F722031
:1089E0006C656E6774683A00556E646566696E659D
:1089F000642062656420636F7272656374696F6E70
:108A0000206D61747269782E00000043616C63759B
:108A10006C617465206F666673657420616E642096
:108A2000736B65772072657475726E696E672072FC
:108A30006573756C743A000000292C206572726FA2
:108A4000723A20002C2000293B2074617267657403
:108A50003A2028002C2000293B206D656173757237
:108A600065642D636F727265637465643A202800D3
:108A70002C20006D656173757265643A2028007062
:108A80006F696E74202300446966666572656E6363
:108A90006520616674657220636F727265637469C4
:108AA0006F6E3A2000002C200063656E7465722C96
:108AB0002061646A75737465643A2000002C20009C
:108AC0005920766563746F722C2061646A757374C3
:108AD00065643A2000002C20005820766563746F8E
:108AE000722C2061646A75737465643A20000063B7
:108AF0006E74725B315D3A0000636E74725B305D60
:108B00003A0046696E616C20636E74722076616C07
:108B10007565733A0000000077793A0000636E745F
:108B2000725B315D3A00005765696768745F793A36
:108B3000000077783A0000636E74725B305D3A0033
:108B4000005765696768745F783A00005665727906
:108B5000206C6974746C6520736B65772064657430
:108B600065637465642E204F7274686F676F6E6101
:108B70006C697A696E672074686520617865732E08
:108B800000004D61782E206572726F7220657563EA
:108B90006C696469616E3A004D61782E206572726D
:108BA0006F7220593A004D61782E206572726F7293
:108BB00020583A004D61782E206572726F72733AB8
:108BC0000000002C206572726F7220593A20002C30
:108BD000206572726F7220583A20006572726F724F
:108BE0003A200029002C2000293B2074617267651F
:108BF000743A2028002C2000293B20636F72726594
:108C0000637465643A2028002C20006D65617375DB
:108C10007265643A202800002C206572726F722001
:108C20003E206D61782E206572726F7220657563CB
:108C30006C696469616E00506F696E74206E6F7448
:108C4000206F6E20666972737420726F77002C201B
:108C50006572726F722059203E206D61782E2065FA
:108C600072726F722059002C206572726F722058D8
:108C7000203E206D61782E206572726F7220580040
:108C80002C2077656967746820593A2000506F6915
:108C90006E74206F6E20666972737420726F770035
:108CA0003A00706F696E742023004572726F7220F3
:108CB000616674657220636F7272656374696F6E4A
:108CC0003A2000002C200063656E746572206E658A
:108CD000772C20696E7665727465643A2000002CEA
:108CE00020005920766563746F72206E65772C20A2
:108CF000696E7665727465643A2000002C20005815
:108D000020766563746F72206E65772C20696E76AD
:108D100065727465643A2000002C2000636F7272E3
:108D2000656374696F6E20616E676C65733A2000CD
:108D3000002C2000636F7272656374656420616E3D
:108D4000676C65733A2000002C2000636F727265B7
:108D50006374656420782F793A2000002C20002C61
:108D600020002C20003B20636F7272656374696F72
:108D70006E20766563746F723A2000697465726163
:108D800074696F6E3A200000292C206572726F7230
:108D90003A20002C2000293B207461726765743AE8
:108DA0002028002C2000206D656173757265643A7F
:108DB000202800706F696E74202300002C2000634F
:108DC000656E7465722C20696E697469616C3A20F5
:108DD00000002C20005920766563746F722C206986
:108DE0006E697469616C3A2000002C20005820766E
:108DF0006563746F722C20696E697469616C3A20C6
:108E00000063616C63756C617465206D6163686992
:108E10006E6520736B657720616E64206F66667384
:108E20006574204C53000000E442FCFFFFBF0000CB
:108E300057430000C0420000E442000042430000EB
:108E400040410000C04200004041FCFFFFBF000065
:108E5000E442FCFFFFBF00005743FCFFFFBF0000E0
:108E600057430000C0420000E4420000C04200003E
:108E700040410000C0420000404100004243000069
:108E8000E4420000424300005743000042434530A3
:108E90003A20005A3A2000593A2000583A20004D12
:108EA00053312C4D53322050696E730A005A002002
:108EB0005A3A00590020593A00580020583A0024E4
:108EC000F4D43050C38E20C2A24017828B7011128E
:108ED0007A910D816CD90AA861E108C758660761CB
:108EE0005143061E4B5D05C145A7041A41110409F3
:108EF0003D9803713931034036DB0265339102D46A
:108F0000305402802E1D02632CEE01752AC501B07B
:108F100028A001102781018F2564012B244B01E03B
:108F2000223401AC211F018D200D01801FFC008423
:108F30001EED00971DDF00B81CD200E61BC6002006
:108F40001BBC00641AB200B219A8000A19A0006A7A
:108F5000189900D117910040178B00B51684003185
:108F6000167E00B31579003A157300C7146F0058C8
:108F7000146A00EE1366008813630025135E00C7B1
:108F8000125B006C12570015125400C11151007091
:108F9000114F0021114B00D61049008D104700469B
:108FA00010440002104200C00F4000800F3E0042FB
:108FB0000F3C00060F3B00CB0E3800930E37005CD1
:108FC0000E3500270E3400F30D3200C10D31009034
:108FD0000D3000600D2E00320D2D00050D2C00D936
:108FE0000C2B00AE0C2900850C29005C0C270035E9
:108FF0000C27000E0C2600E80B2400C40B2400A054
:109000000B23007D0B23005A0B2100390B21001884
:109010000B2000F80A1F00D90A1E00BB0A1E009D83
:109020000A1D00800A1D00630A1C00470A1B002C51
:109030000A1B00110A1A00F7091A00DD091900C4F9
:10904000091900AB091900920917007B0918006380
:109050000917004C09160036091600200916000AE7
:10906000091500F5081500E0081400CC081400B834
:10907000081400A4081400900813007D0812006B67
:109080000813005808120046081200340811002383
:109090000811001208110001081100F0071000E08B
:1090A000071000D0071000C0071000B0070F00A184
:1090B00007100091070E0083070F0074070F00656B
:1090C000070E0057070E0049070E003B070D002E44
:1090D000070E0020070D0013070D0006070D00F90D
:1090E000060C00ED060D00E0060C00D4060C00C8CE
:1090F000060C00BC060C00B0060C00A4060B009980
:10910000060C008D060B0082060B0077060B006C28
:10911000060B0061060A0057060B004C060A0042C7
:10912000060A0038060A002E060A0024060A001A5B
:10913000060A001006090007060A00FD050900F4EA
:10914000050900EB050900E2050900D9050900D071
:10915000050900C7050900BE050900B5050800ADF1
:10916000050800A50509009C050800940508008C69
:10917000050800840508007C050800740508006CDB
:10918000050700650508005D050700560508004E47
:1091900005070047050700400508003805070031AE
:1091A0000507002A050700230507001C0506001611
:1091B0000507000F0507000805060002050700FB6C
:1091C000040600F5040700EE040600E8040600E2C9
:1091D000040700DB040600D5040600CF040600C91E
:1091E000040600C3040600BD040600B7040600B16F
:1091F000040500AC040600A6040600A00405009BBC
:1092000004060095040500900406008A0405008504
:10921000040500800406007A04050075040500704A
:109220000405006B04050066040500610405005C8C
:1092300004050057040500520405004D04050048CC
:10924000040500430405003E0404003A040500350B
:10925000040500300404002C040500270404002346
:109260000405001E0404001A04040016040500117D
:109270000404000D040400090405000404040000B3
:10928000040400FC030400F8030400F4030400F0E9
:10929000030400EC030400E8030400E4030400E01A
:1092A000030400DC030400D8030400D4030400D04A
:1092B000030400CC030400C8030300C50303002417
:1092C000F404D9201BC40C5C0E9804C4095F026529
:1092D000077101F405F900FB04B30048048700C1DD
:1092E0000369005803550003034500BE023A008499
:1092F00002310053022A002902250004022000E462
:10930000011C00C8011900AF011700980114008466
:10931000011300710110006101100051010E0043A2
:10932000010D0036010B002B010B0020010B001575
:109330000109000C01090003010800FB000800F30B
:10934000000800EB000700E4000600DE000600D87D
:10935000000600D2000600CC000500C7000500C2D0
:10936000000500BD000400B9000400B5000400B110
:10937000000400AD000400A9000400A5000300A241
:109380000003009F0004009B000300980003009569
:1093900000020093000300900003008D0002008B88
:1093A00000030088000200860002008400030081A0
:1093B0000002007F0002007D0002007B00020079B5
:1093C00000020077000100760002007400020072C3
:1093D000000100710002006F0002006D0001006CCE
:1093E0000002006A000100690002006700010066D7
:1093F00000010065000100640002006200010061DC
:10940000000100600001005F0002005D0001005CDF
:109410000001005B0001005A0001005900010058E2
:1094200000010057000100560001005500010054E2
:1094300000010053000000530001005200010051E0
:10944000000100500001004F0001004E0000004EDE
:109450000001004D0001004C0001004B0000004BDA
:109460000001004A000100490001004800000048D6
:1094700000010047000100460000004600010045D1
:1094800000000045000100440001004300000043CB
:1094900000010042000000420001004100000041C4
:1094A000000100400001003F0000003F0001003EBD
:1094B0000000003E0001003D0000003D0001003CB6
:1094C0000000003C0000003C0001003B0000003BAD
:1094D0000001003A0000003A0001003900000039A4
:1094E000000100380000003800000038000100379B
:1094F0000000003700010036000000360000003692
:109500000001003500000035000000350001003486
:10951000000000340000003400010033000000337C
:109520000000003300010032000000320000003271
:109530000001003100000031000000310001003066
:1095400000000030000000300001002F0000002F5C
:109550000000002F0000002F0001002E0000002E50
:109560000000002E0001002D0000002D0000002D45
:109570000000002D0001002C0000002C0000002C39
:109580000000002C0001002B0000002B0000002B2D
:109590000000002B0001002A0000002A0000002A21
:1095A0000000002A00010029000000290000002915
:1095B0000000002900000029000100280000002808
:1095C00000000028000000280000002800010027FB
:1095D00000000027000000270000002700000027EF
:1095E00000010026000000260000002600000026E2
:1095F00000000026000100250000002500000025D5
:1096000000000025000000250000002500010024C6
:1096100000000024000000240000002400000024BA
:1096200000010023000000230000002300000023AD
:10963000000000230000002300000023000100229E
:109640000000002200000022000000220000002292
:109650000000002200010021000000210000002184
:109660000000002100000021000000210000002176
:109670000001002000000020000000200000002069
:10968000000000200000002000000020000000205A
:109690000001001F0000001F0000001F0000001F4D
:1096A0000000001F0000001F0000001F0001001E3E
:1096B0000000001E0000001E0000001E000000450B
:1096C00072723A204D494E54454D50204245440057
:1096D00054656D706572617475726520686561743A
:1096E00065642062656420737769746368656420CB
:1096F0006F66662E204D494E54454D502074726958
:109700006767657265642021004572723A204D4199
:109710005854454D50204245440054656D70657263
:109720006174757265206865617465642062656442
:10973000207377697463686564206F66662E204DB8
:10974000415854454D50207472696767657265646D
:109750002021004572723A204D494E54454D50002B
:109760003A20457874727564657220737769746302
:10977000686564206F66662E204D494E54454D50F5
:109780002074726967676572656420210045727292
:109790003A204D415854454D50003A204578747256
:1097A00075646572207377697463686564206F6699
:1097B000662E204D415854454D502074726967679C
:1097C0006572656420210020484F54454E44205462
:1097D0004845524D414C2052554E41574159002069
:1097E0004845415442454420544845524D414C203F
:1097F00052554E4157415900544845524D414C2015
:1098000052554E4157415900424544205448455213
:109810004D414C2052554E41574159002054484526
:10982000524D414C2052554E41574159202820500D
:1098300052454845415420484F54454E4429002044
:10984000544845524D414C2052554E4157415920A4
:1098500028205052454845415420484541544245EE
:1098600044290050524548454154204552524F52D8
:1098700000424544205052454845415420455252EB
:109880004F5200202D20496E76616C696420657806
:10989000747275646572206E756D62657220210048
:1098A000504944204175746F74756E652066696E09
:1098B0006973686564212050757420746865206C34
:1098C000617374204B702C204B6920616E64204BB7
:1098D0006420636F6E7374616E74732066726F6D53
:1098E0002061626F766520696E746F20436F6E66CB
:1098F000696775726174696F6E2E68005049442003
:109900004175746F74756E65206661696C6564215C
:109910002074696D656F75740020403A006F6B208C
:10992000543A006F6B20423A00504944204175740C
:109930006F74756E65206661696C6564212054657D
:109940006D706572617475726520746F6F206869DF
:10995000676800204B643A2000204B693A200020C1
:109960004B703A200020436C617373696320504947
:109970004420002054753A2000204B753A200020E6
:109980006D61783A2000206D696E3A200020643ABB
:10999000200020626961733A20001000C9021001A2
:1099A0002C014001220170011801B0010E01F001EB
:1099B00004015002FA00B002F0003003E600D003C8
:1099C000DC009004D2007005C800A006BE000008AC
:1099D000B400B009AA00D00BA000600E9600601180
:1099E0008C000015820020197800C01D6E00A02296
:1099F0006400B0275A00902C500000314600E0343B
:109A00003C0010383200903A2800603C1E00A03D17
:109A10001400803E0A00203F000070012C019001DC
:109A20002701B0012201C0011D01F001180110023F
:109A3000130130020E016002090190020401C0020C
:109A4000FF000003FA004003F5008003F000D0039C
:109A5000EB002004E6007004E100E004DC004005B7
:109A6000D700C005D2004006CD00D006C800800750
:109A7000C3003008BE00F008B900C009B400B00A45
:109A8000AF00B00BAA00D00CA500000EA000500F34
:109A90009B00C01096005012910000148C00C0155D
:109AA0008700B0178200B0197D00D01B7800001E1F
:109AB000730040206E0090226900F024640040276B
:109AC0005F0090295A00E02B5500102E50002030E6
:109AD0004B0010324600E033410090353C00103717
:109AE000370070383200A0392D00B03A2800A03B72
:109AF0002300603C1E00103D1900903D1400103EF4
:109B00000F00703E0A00C03E0500003F0000436F9A
:109B10006E74696E7565207769746820616E6F7404
:109B200068657220626F7764656E3F004737360064
:109B30004D3435205A004D34350047383000200070
:109B40003E003E0020003E003E00005365766572F8
:109B50006520736B65773A0000536C696768742001
:109B6000736B65773A002D2D2D2D2D2D2D2D2D2D3F
:109B70002D2D2D2D2D2D2D2D2D2D004E2F41004D18
:109B80006561737572656420736B65773A20004E6A
:109B90002F41006D6D000052696768743A0043659B
:109BA0006E7465723A004C6566743A0059206469B7
:109BB0007374616E63652066726F6D206D696E3AB5
:109BC000004D373031004D373032004D35303000E8
:109BD0004D353030004731205A313520463135304F
:109BE000300047393100473120583530205931395C
:109BF0003020453020463730303000473930004D76
:109C0000373032004D3730322043004D373032206C
:109C100055004D373032004731205A31352046311A
:109C20003530300047393100473120583530205920
:109C3000313930204530204637303030004D383310
:109C400000473930004D3834004D31303420533026
:109C500000473930004731204531004D3832004D42
:109C60003833004D31303620532564004D323230C8
:109C700020532564003A200020202020202020208E
:109C8000202020202020202020202000203A2000FA
:109C900020202020202020202020202020202020C4
:109CA00020202020002020202020202020202020D4
:109CB0002020002573002020002D2D3A2D2D00207E
:109CC00000200020004C002020002046002D2D2DDB
:109CD000003E555342005344002D2D0025202020E6
:109CE0002020002020002020000120002020202D06
:109CF0002D2D200020205A002020000120004D366C
:109D0000303000464C4558202D20203233302F353E
:109D1000300050502020202D20203235342F31307B
:109D2000300048495053202D20203232302F31301E
:109D3000300050455420202D20203234302F39302F
:109D40000041425320202D20203235352F31303034
:109D500000504C4120202D20203231352F35350048
:109D60004D3234004D323320257300052E2E00581D
:109D70000059005A0045787472756465720047395D
:109D8000390044697361626C65206661726D206D93
:109D90006F64653F0044697361626C65206661723F
:109DA0006D206D6F6465004661726D206E756D6229
:109DB0006572004D3834004D3834004731205A3137
:109DC00035004732382057005A30005A3100593098
:109DD00000593100583000583100456E64207374CA
:109DE0006F70732064696167004D34340047323806
:109DF00020570058595A2063616C2E2064657461A5
:109E0000696C73002D2D2D2D2D2D2D2D2D2D2D2DEE
:109E100000466C6173684169722049502041646456
:109E2000723A002D2D2D2D2D2D2D2D2D2D2D2D006A
:109E300033442D677573736E65722C20546573748B
:109E4000004A756C2020362032303137004461746E
:109E5000653A20002D2D2D2D2D2D2D2D2D2D2D2D27
:109E600000453344763666756C6C0052414D426F46
:109E700031336100315F37356D6D5F4D4B32002DF1
:109E80002D2D2D2D2D2D2D2D2D2D2D004657202DF9
:109E900020332E302E31322D524332004669726DFE
:109EA00077617265202D20332E302E31322D5243B2
:109EB000320025642E25642E25642E25640046611B
:109EC000726D206E756D62657200706F7369746972
:109ED0006F6E00726573746F72650000726300626A
:109EE00065746100616C7068610064657600505251
:109EF0005553413344465700332E302E31322D52C4
:109F000043320000000A0B02090C0D0E080703047F
:109F10000100000000000000000000000000000040
:109F2000000000000000000000000000000000121F
:109F30001110000000000000000000000000000000
:109F40000000000000000000000000000000000011
:109F5000000000000000000000010210202008089E
:109F6000102040102040800201020108040201017B
:109F70000204081020408080402010080402018064
:109F800004020180402010080402010804020101BB
:109F900002040810204080010204081020408010B4
:109FA00008040880102040044080102040048005F0
:109FB000050505070508080808020202020A0A0842
:109FC0000804040404010101010101010103030368
:109FD0000303030303040707070C0C0C0C0C0C0C05
:109FE0000C0202020206060606060606060B0B0B0C
:109FF0000B0B0B0B0B07070A0A0A0A0A0A050505D1
:10A000000404040808000020002300260029002C76
:10A01000002F0032000001000003010601090100C9
:10A02000002200250028002B002E00310034000201
:10A03000010000050108010B010000210024002798
:10A04000002A002D00300033000101000004010748
:10A05000010A01024E414E494E495459494E46CDDE
:10A06000CCCC3D0AD7233C17B7D13877CC2B3295CF
:10A0700095E6241FB14F0A000020410000C84200AD
:10A08000401C4620BCBE4CCA1B0E5AAEC59D740077
:10A0900072B5A40172014A01ADB511241FBECFEF04
:10A0A000D1E2DEBFCDBF00E00CBF16E0A0E0B2E021
:10A0B000EAECF8E903E00BBF02C007900D92A03F65
:10A0C000B107D9F728E1A0EFB6E001C01D92AD3786
:10A0D000B207E1F710EAC8E9D0EA00E006C022972B
:10A0E0000109FE010BBF0F9456C5C039D10780E0AE
:10A0F0000807A9F70F940BBF0D9454CC0C940000E3
:10A10000EF92FF920F931F93CF93DF931F92CDB7E0
:10A11000DEB78C017B01460FF70161917F01F801E9
:10A120008081918149830F948DCBF8018081918149
:10A1300001969183808349814E11EECF0F90DF917C
:10A14000CF911F910F91FF90EF900895EF92FF92A2
:10A150000F931F93CF93DF931F92CDB7DEB78C0180
:10A160007B01460FF8018081918149830F945DCB7B
:10A17000F70181937F01F80180819181019691839C
:10A18000808349814E11EECF0F90DF91CF911F91C7
:10A190000F91FF90EF9008950F931F93CF93DF934C
:10A1A000CDB7DEB72C970FB6F894DEBF0FBECDBF8C
:10A1B00080E390E3A0E3B0E08D839E83AF83B88714
:10A1C00004E110E01C870B8744E0BE016B5F7F4F0A
:10A1D000CE010B9695DF40E16EE276E1CE010B9663
:10A1E0008FDF40E16EE376E1CE010B9689DF40E13F
:10A1F0006EE176E1CE010B9683DF44E066E176E125
:10A20000CE010B967DDF44E062E176E1CE010B9654
:10A2100077DF44E06AE176E1CE010B9671DF44E03E
:10A220006EEF75E1CE010B966BDF44E06EE476E1F4
:10A23000CE010B9665DF44E062E076E1CE010B963D
:10A240005FDF44E066E076E1CE010B9659DF44E043
:10A250006AE076E1CE010B9653DF44E06EE076E1F2
:10A26000CE010B964DDF4CE064E17AE0CE010B9617
:10A2700047DF44E06DE07AE0CE010B9641DF44E039
:10A2800066E972E0CE010B963BDF44E062E972E0E2
:10A29000CE010B9635DF44E06EE872E0CE010B96FE
:10A2A0002FDF44E066E872E0CE010B9629DF44E040
:10A2B00062E872E0CE010B9623DF44E06EE772E0C5
:10A2C000CE010B961DDF80E290E09A87898742E0FD
:10A2D000BE01675F7F4FCE010B9612DF41E069E060
:10A2E0007AE0CE010B960CDF44E06DE172E0CE0126
:10A2F0000B9606DF44E065E172E0CE010B9600DFCD
:10A3000044E064E07AE0CE010B96FADE44E060E0DF
:10A310007AE0CE010B96F4DE44E061E172E0CE011A
:10A320000B96EEDE41E060E37AE0CE010B96E8DECC
:10A3300044E06DE372E0CE010B96E2DE86E591E348
:10A34000A0E0B0E089839A83AB83BC831C870B8732
:10A3500044E0BE016F5F7F4FCE010B96D1DEECE390
:10A36000FDE08491882341F09091C00095FFFCCFDF
:10A370008093C6003196F5CFE7EFF6E0849188230D
:10A3800041F09091C00095FFFCCF8093C6003196BC
:10A39000F5CF8091C00085FFFCCF8AE08093C60096
:10A3A0002C960FB6F894DEBF0FBECDBFDF91CF91D4
:10A3B0001F910F910895CF93DF93CCE3DDE0FE0171
:10A3C0008491882341F09091C00095FFFCCF809349
:10A3D000C6003196F5CFE7EEF6E08491882341F090
:10A3E0009091C00095FFFCCF8093C6003196F5CFC9
:10A3F0008091C00085FFFCCF8AE08093C600FE01FB
:10A400008491ECE3FDE0882349F09091C00095FF32
:10A41000FCCF8093C60031968491F5CF40912E16E3
:10A4200050912F1660913016709131168FED96E095
:10A430000E94C862409132165091331660913416D2
:10A44000709135168CED96E00E94C86240913616E8
:10A4500050913716609138167091391689ED96E053
:10A460000E94C86240913A1650913B1660913C168A
:10A4700070913D1686ED96E00E94C8628091C00002
:10A4800085FFFCCF8AE08093C600FE018491ECE357
:10A49000FDE0882349F09091C00095FFFCCF8093A8
:10A4A000C60031968491F5CFECEBF6E084918823D9
:10A4B00041F09091C00095FFFCCF8093C60031968B
:10A4C000F5CF8091C00085FFFCCF8AE08093C60065
:10A4D000FE018491ECE3FDE0882349F09091C000F7
:10A4E00095FFFCCF8093C60031968491F5CF4091C3
:10A4F0003E1650913F16609140167091411683EBC5
:10A5000096E00E94C86240914216509143166091B5
:10A5100044167091451680EB96E00E94C862409107
:10A5200046165091471660914816709149168DEA6B
:10A5300096E00E94C86240914A1650914B16609175
:10A540004C1670914D168AEA96E00E94C86280917E
:10A55000C00085FFFCCF8AE08093C600FE01849195
:10A56000ECE3FDE0882349F09091C00095FFFCCF1B
:10A570008093C60031968491F5CFECE8F6E08491A3
:10A58000882341F09091C00095FFFCCF8093C600D6
:10A590003196F5CF8091C00085FFFCCF8AE0809393
:10A5A000C600FE018491ECE3FDE0882349F0909120
:10A5B000C00095FFFCCF8093C60031968491F5CF03
:10A5C00040911E1650911F16609120167091211611
:10A5D00083E896E00E94D96240912216509123169A
:10A5E000609124167091251680E896E00E94D96249
:10A5F00040912616509127166091281670912916C1
:10A600008DE796E00E94D96240912A1650912B1650
:10A6100060912C1670912D168AE796E00E94D962FF
:10A620008091C00085FFFCCF8AE08093C600FE01C8
:10A630008491ECE3FDE0882349F09091C00095FF00
:10A64000FCCF8093C60031968491F5CFE5E4F6E027
:10A650008491882341F09091C00095FFFCCF8093B6
:10A66000C6003196F5CF8091C00085FFFCCF8AE00F
:10A670008093C600FE018491ECE3FDE0882349F05D
:10A680009091C00095FFFCCF8093C60031968491D5
:10A69000F5CF4091161650911716609118167091CB
:10A6A00019168CE396E00E94C862409112165091F0
:10A6B0001316609114167091151689E396E00E94A6
:10A6C000C8628091C00085FFFCCF8AE08093C600FD
:10A6D000FE018491ECE3FDE0882349F09091C000F5
:10A6E00095FFFCCF8093C60031968491F5CFE6E8C4
:10A6F000F5E08491882341F09091C00095FFFCCF54
:10A700008093C6003196F5CF8091C00085FFFCCFC5
:10A710008AE08093C600FE018491ECE3FDE088238B
:10A7200049F09091C00095FFFCCF8093C600319610
:10A730008491F5CF40911A1650911B1660911C160A
:10A7400070911D168DE795E00E94C8624091FE153C
:10A750005091FF1560910016709101168AE795E0FF
:10A760000E94C86240914E1650914F16609150164B
:10A770007091511687E795E00E94D96240910216C8
:10A7800050910316609104167091051684E795E0C8
:10A790000E94C862409106165091071660910816F3
:10A7A0007091091681E795E00E94C86240910A16EF
:10A7B00050910B1660910C1670910D168EE695E077
:10A7C0000E94C86240910E1650910F1660911016AB
:10A7D000709111168BE695E00E94C8628091C000CE
:10A7E00085FFFCCF8AE08093C600FE018491ECE3F4
:10A7F000FDE0882349F09091C00095FFFCCF809345
:10A80000C60031968491F5CFE9E5F5E0849188237F
:10A8100041F09091C00095FFFCCF8093C600319627
:10A82000F5CF8091C00085FFFCCF8AE08093C60001
:10A83000FE018491ECE3FDE0882349F09091C00093
:10A8400095FFFCCF8093C60031968491F5CF40915F
:10A85000140A5091150A6091160A7091170A80E542
:10A8600095E00E94C8624091180A5091190A6091BF
:10A870001A0A70911B0A8DE495E00E94C86240910B
:10A880001C0A50911D0A60911E0A70911F0A8AE4E9
:10A8900095E00E94C8628091C00085FFFCCF8AE0ED
:10A8A0008093C600FE018491ECE3FDE0882349F02B
:10A8B0009091C00095FFFCCF8093C60031968491A3
:10A8C000F5CFECE3F5E08491882341F09091C0004E
:10A8D00095FFFCCF8093C6003196F5CF8091C000E4
:10A8E00085FFFCCF8AE08093C600FE018491ECE3F3
:10A8F000FDE0882349F09091C00095FFFCCF809344
:10A90000C60031968491F5CF4091960250919702FE
:10A91000609198027091990282E395E00E94C8626A
:10A9200060919202709193028091940290919502AD
:10A930000F943053AB01BC018FE295E00E94C862D6
:10A9400060918E0270918F0280919002909191029D
:10A950000F943C53AB01BC018CE295E00E94C862AD
:10A960008091C00085FFFCCF8AE08093C600FE0185
:10A970008491ECE3FDE0882349F09091C00095FFBD
:10A98000FCCF8093C60031968491F5CFE6E1F5E0E7
:10A990008491882341F09091C00095FFFCCF809373
:10A9A000C6003196F5CF8091C00085FFFCCF8AE0CC
:10A9B0008093C600FE018491ECE3FDE0882349F01A
:10A9C0009091C00095FFFCCF8093C6003196849192
:10A9D000F5CF409186025091870260918802709174
:10A9E00089028CE095E00E94C862609182027091B9
:10A9F000830280918402909185020F943053AB01C1
:10AA0000BC0189E095E00E94C86260917E0270916D
:10AA10007F0280918002909181020F943C53AB01A0
:10AA2000BC0186E095E00E94C8628091C00085FF6D
:10AA3000FCCF8AE08093C600FE018491ECE3FDE048
:10AA4000882349F09091C00095FFFCCF8093C60009
:10AA500031968491F5CFE2EDF4E08491882341F0C2
:10AA60009091C00095FFFCCF8093C6003196F5CF42
:10AA70008091C00085FFFCCF8AE08093C600FE0174
:10AA80008491ECE3FDE0882349F09091C00095FFAC
:10AA9000FCCF8093C60031968491F5CF40911D0282
:10AAA00050911E0260911F027091200288EC94E088
:10AAB0000E94C86220E030E040E752E46091150255
:10AAC0007091160280911702909118020F940BC397
:10AAD000AB01BC0185EC94E00E94C8624091040A7D
:10AAE0005091050A6091060A7091070A82EC94E081
:10AAF0000E94C8628091C00085FFFCCF8AE08093ED
:10AB0000C600FE018491ECE3FDE0882349F09091BA
:10AB1000C00095FFFCCF8093C60031968491F5CF9D
:10AB2000E6E9F4E08491882341F09091C00095FF1C
:10AB3000FCCF8093C6003196F5CF8091C00085FF91
:10AB4000FCCF8AE08093C600FE018491ECE3FDE037
:10AB5000882349F09091C00095FFFCCF8093C600F8
:10AB600031968491F5CF4091000A5091010A60918D
:10AB7000020A7091030A8CE894E00E94C86220E007
:10AB800030E040E752E4609111027091120280912E
:10AB90001302909114020F940BC3AB01BC0189E81E
:10ABA00094E00E94C8628091C00085FFFCCF8AE0DB
:10ABB0008093C600FE018491ECE3FDE0882349F018
:10ABC0009091C00095FFFCCF8093C6003196849190
:10ABD000F5CFEFE2F4E08491882341F09091C0003A
:10ABE00095FFFCCF8093C6003196F5CF8091C000D1
:10ABF00085FFFCCF8AE08093C600FE018491ECE3E0
:10AC0000FDE0882349F09091C00095FFFCCF809330
:10AC1000C60031968491F5CF4091090A50E060E07A
:10AC200070E085E294E00E94D9628091C00085FFC7
:10AC3000FCCF8AE08093C600FE018491ECE3FDE046
:10AC4000882349F09091C00095FFFCCF8093C60007
:10AC500031968491F5CF8091300A8823A1F1E2E109
:10AC6000F4E08491882341F09091C00095FFFCCFDF
:10AC70008093C6003196F5CF8091C00085FFFCCF50
:10AC80008AE08093C600FE01C491ECE3FDE0CC2392
:10AC900049F08091C00085FFFCCFC093C60031967B
:10ACA000C491F5CF40913D0250913E0260913F0228
:10ACB0007091400288E094E00E94C8628091C000D8
:10ACC00085FFFCCF11C0ECEEF3E08491882341F0C6
:10ACD0009091C00095FFFCCF8093C6003196F5CFD0
:10ACE0008091C00085FFFCCF8AE08093C600DF9191
:10ACF000CF910895AF92BF92CF92DF92EF92FF92E1
:10AD00000F931F93CF93DF93CDB7DEB7E0970FB6C6
:10AD1000F894DEBF0FBECDBF80E1EBEAF2E0DE01CA
:10AD2000919601900D928A95E1F780E1EBEBF2E0CC
:10AD3000DE01519601900D928A95E1F780E1EBECEE
:10AD4000F2E0DE01119601900D928A95E1F76E0115
:10AD500081E2C80ED11C8EE2E82E86E1F82E8E012B
:10AD60000F5E1F4F6EE376E1AE014F5F5F4F9EE1D6
:10AD7000A92E96E1B92E20E030E0F6018191919163
:10AD8000A191B1916F01F70181939193A193B19337
:10AD90007F01F80181919191A191B1918F01FB0106
:10ADA00081939193A193B193BF01FA018191919104
:10ADB000A191B191AF01F50181939193A193B193C9
:10ADC0005F012F5F3F4F24303105B9F60F946A348D
:10ADD00080E090E8ABEBB4E48093161690931716DE
:10ADE000A0931816B0931916809312169093131609
:10ADF000A0931416B093151610921A1610921B16E3
:10AE000010921C1610921D1680E29EE4A0E0B0E0A5
:10AE100080934E1690934F16A0935016B0935116F0
:10AE20001092FE151092FF15109200161092011646
:10AE300080E090E0A0E2B1E48093021690930316C4
:10AE4000A0930416B09305168093061690930716E8
:10AE5000A0930816B09309168DEC9CECACE4BEE30D
:10AE600080930A1690930B16A0930C16B0930D16B0
:10AE700080E090E0A0E2B0E480930E1690930F166D
:10AE8000A0931016B093111610921C0A10921D0A6E
:10AE900010921E0A10921F0A1092180A1092190A94
:10AEA00010921A0A10921B0A1092140A1092150A94
:10AEB0001092160A1092170A88EB9EE1A3EBB1E4F8
:10AEC0008093960290939702A0939802B093990270
:10AED00064EA70E78DEF9FE30F942A536093920228
:10AEE0007093930280939402909395026BE774E1C0
:10AEF0008DE792E40F94365360938E0270938F0225
:10AF000080939002909391020F947F4480E090E0B0
:10AF1000A0E8BFE380938A0290938B02A0938C02F7
:10AF2000B0938D021092090A80E090E0A0E4B0E4B2
:10AF300080931D0290931E02A0931F02B0932002E3
:10AF400040E050E064E372E440931502509316022F
:10AF500060931702709318021092040A1092050A67
:10AF60001092060A1092070A1092000A1092010A23
:10AF70001092020A1092030A40E050E060E071E48F
:10AF800040931102509312026093130270931402C3
:10AF90001092300A80933D0290933E02A0933F02AC
:10AFA000B09340020E94EE76ECE3FDE084918823AA
:10AFB00041F09091C00095FFFCCF8093C600319680
:10AFC000F5CFE0EBF3E08491882341F09091C0004D
:10AFD00095FFFCCF8093C6003196F5CF8091C000DD
:10AFE00085FFFCCF8AE08093C600E0960FB6F89408
:10AFF000DEBF0FBECDBFDF91CF911F910F91FF90AC
:10B00000EF90DF90CF90BF90AF900895CF93DF93F4
:10B01000CDB7DEB72C970FB6F894DEBF0FBECDBF0D
:10B0200084E190E09C878B8786E591E3A0E0B0E027
:10B0300089839A83AB83BC8344E0BE016B5F7F4FFF
:10B04000CE010B9683D843E050E0BE016B5F7F4F8B
:10B05000CE0101960F94DCC8892B09F0E1C040E1D4
:10B060006EE276E1CE010B9671D840E16EE376E1B7
:10B07000CE010B966BD840E16EE176E1CE010B96E6
:10B0800065D80F946A3444E066E176E1CE010B9610
:10B090005DD844E062E176E1CE010B9657D844E0FA
:10B0A0006AE176E1CE010B9651D844E06EEF75E18E
:10B0B000CE010B964BD844E06EE476E1CE010B96C0
:10B0C00045D844E062E076E1CE010B963FD844E0FB
:10B0D00066E076E1CE010B9639D844E06AE076E18D
:10B0E000CE010B9633D844E06EE076E1CE010B96AC
:10B0F0002DD84CE064E17AE0CE010B9627D844E0ED
:10B100006DE07AE0CE010B9621D844E066E972E06A
:10B11000CE010B961BD844E062E972E0CE010B969B
:10B1200015D844E06EE872E0CE010B960FD844E0EB
:10B1300066E872E0CE010B9609D844E062E872E05E
:10B14000CE010B9603D844E06EE772E0CE010B9679
:10B150000E94A65042E0BE01675F7F4FCE010B9672
:10B160000E94A65041E069E07AE0CE010B960E9471
:10B17000A65044E06DE172E0CE010B960E94A6500D
:10B1800044E065E172E0CE010B960E94A65044E0D7
:10B1900064E07AE0CE010B960E94A65044E060E0A5
:10B1A0007AE0CE010B960E94A65044E061E172E085
:10B1B000CE010B960E94A65041E060E37AE0CE01FA
:10B1C0000B960E94A65044E06DE372E0CE010B9610
:10B1D0000E94A6500E94EE760F947F44ECE3FDE0BF
:10B1E0008491882341F09091C00095FFFCCF80931B
:10B1F000C6003196F5CFE2EDF3E08491882341F06B
:10B200009091C00095FFFCCF8093C6003196F5CF9A
:10B210008091C00085FFFCCF8AE08093C60001C00A
:10B2200069DD2C960FB6F894DEBF0FBECDBFDF915F
:10B23000CF910895CF93DF93EC0160E08E810F945E
:10B2400048B981E090E00F948AB761E08E810F9455
:10B2500048B981E090E00F948AB760E08E810F9446
:10B2600048B984E690E0DF91CF910D948AB7CF92F0
:10B27000DF92EF92FF920F931F93CF93DF937C01A6
:10B28000C0E0D0E0C62ED12C87010C0F1D1F61E05D
:10B29000F80187810F940FB9B6010C2E02C0759585
:10B2A00067950A94E2F76170F80187810F9448B9B5
:10B2B0002196C430D10541F7C701DF91CF911F918D
:10B2C0000F91FF90EF90DF90CF90B4CFCF92DF92AD
:10B2D000EF92FF920F931F93CF93DF937C01C0E017
:10B2E000D0E0C62ED12C87010C0F1D1F61E0F801A4
:10B2F00087810F940FB9B6010C2E02C07595679522
:10B300000A94E2F76170F80187810F9448B9219699
:10B31000C830D10541F7C701DF91CF911F910F913F
:10B32000FF90EF90DF90CF9085CF1F93CF93DF9367
:10B33000EC01162F642F8C810F9448B98D818F3FBB
:10B3400019F060E00F9448B98F85612F84FF05C024
:10B35000CE01DF91CF911F91B9CF70E084E0759558
:10B3600067958A95E1F7CE0182DF612FCE01DF91EB
:10B37000CF911F917CCF40E0D8CF61E0FCDF80E42B
:10B3800096E00D948AB762E0F6DF80E496E00D94D3
:10B390008AB7CF93DF93CDB7DEB728970FB6F8946F
:10B3A000DEBF0FBECDBF28E0EBEDF2E0DE0111966F
:10B3B00001900D922A95E1F7FC012389421710F0C4
:10B3C0004FEF420FFE013196E40FF11DE40FF11D26
:10B3D0002081260F2068622F28960FB6F894DEBFD2
:10B3E0000FBECDBFDF91CF91C6CFFC016089262F64
:10B3F0002460208B6C60BFCFCF93DF93EC01423091
:10B4000018F08F8588608F874B8B1C8A222329F048
:10B41000413019F48F8584608F8780E593EC0F9419
:10B420008AB760E08C810F9448B960E08E810F94F8
:10B4300048B98D818F3F19F060E00F9448B96F854E
:10B4400064FD19C063E0CE0112DF84E991E10F943D
:10B450008AB763E0CE010BDF84E991E10F948AB7EC
:10B4600063E0CE0104DF86E990E00F948AB762E0E2
:10B47000CE01FDDE13C06062CE017DDF84E991E183
:10B480000F948AB76F856062CE0175DF86E990E020
:10B490000F948AB76F856062CE016DDF6F85606241
:10B4A000CE0169DF8CE390E00F948AB784E0888B4B
:10B4B000CE019BDF8CE390E00F948AB7CE015DDF75
:10B4C00088EB9BE00F948AB782E0898B66E0CE011F
:10B4D00052DF8CE390E0DF91CF910D948AB76F92A9
:10B4E0007F928F92AF92CF92EF920F931F93CF9351
:10B4F000DF93CDB7DEB73C01162F842F5E854F85D5
:10B5000038899989F301848325830683E782C0867D
:10B51000A1868286538744873587968761E00F949A
:10B520000FB9F30185818F3F19F061E00F940FB9D6
:10B5300061E0F30186810F940FB9112319F0F30133
:10B54000178603C080E1F301878720E041E060E1D6
:10B55000C301DF91CF911F910F91EF90CF90AF90EA
:10B560008F907F906F9048CF8F92AF92CF92EF9253
:10B570000F93DC0113961C921E921297ECE3F3E0FA
:10B58000ED93FC931F921F921F921F928C2CAE2C56
:10B59000C02EE22E042F2FEF462F61E0A0DF0F9088
:10B5A0000F900F900F900F91EF90CF90AF908F90E2
:10B5B0000895CF93DF93EC01423018F08F858860B7
:10B5C0008F874B8B1C8A222329F0413019F48F85F9
:10B5D00084608F8780E593EC0F948AB760E08C815C
:10B5E0000F9448B960E08E810F9448B98D818F3FE8
:10B5F00019F060E00F9448B96F8564FD19C063E0ED
:10B60000CE0135DE84E991E10F948AB763E0CE0183
:10B610002EDE84E991E10F948AB763E0CE0127DE44
:10B6200086E990E00F948AB762E0CE0120DE13C075
:10B630006062CE01A0DE84E991E10F948AB76F8544
:10B640006062CE0198DE86E990E00F948AB76F853C
:10B650006062CE0190DE6F856062CE018CDE8CE38D
:10B6600090E00F948AB784E0888BCE01BEDE8CE335
:10B6700090E00F948AB7CE0186DE80E496E00F94C6
:10B680008AB782E0898B66E0CE0175DE8CE390E0BC
:10B690000F948AB740E068E0CE017BDE68E776E091
:10B6A000CE010F94E3B941E068E0CE0172DE68E7B5
:10B6B00076E0CE010F94E3B942E066E0CE0169DEA8
:10B6C00066E776E0CE01DF91CF910D94E3B9CF929A
:10B6D000DF92EF92FF920F931F93CF93DF931F920E
:10B6E0001F92CDB7DEB78C01677088E0689FB0010C
:10B6F00011246064C80149835A833DDE4981C42E08
:10B700005A81D52EE12CF12CD6016D916D01D80115
:10B71000ED91FC910190F081E02DC8011995BFEFEA
:10B72000EB1AFB0AE8E0EE16F10471F70F900F90A8
:10B73000DF91CF911F910F91FF90EF90DF90CF900D
:10B74000089541E0F2DD81E090E008951F920F92AC
:10B750000FB60F9211240BB60F922F933F934F9376
:10B760005F936F938F939F93EF93FF93CF93DF93A9
:10B770001F92CDB7DEB78091C00084FF04C08091D6
:10B78000C600898319C06091C6002091710730916D
:10B790007207C90101968F779927409173075091DD
:10B7A00074078417950741F0F901EF50F94F608352
:10B7B00090937207809371070F90DF91CF91FF9163
:10B7C000EF919F918F916F915F914F913F912F9149
:10B7D0000F900BBE0F900FBE0F901F9018959A01FF
:10B7E000AB01211581EE38074105510549F182E091
:10B7F0008093C00060E079E08DE390E00F941EC577
:10B800002150310941095109CA01B90122E030E052
:10B8100040E050E00F941EC53093C5002093C40053
:10B820008091C10080618093C1008091C1008860D7
:10B830008093C1008091C10080688093C100089509
:10B840001092C00020E130E0E7CF209173073091E3
:10B85000740780917107909172078217930771F0B6
:10B86000F901EF50F94F80812F5F3F4F2F7733273A
:10B87000309374072093730790E008958FEF9FEF44
:10B880000895809173079091740790937207809345
:10B89000710708954F925F926F927F928F929F925D
:10B8A000AF92BF92CF92DF92EF92FF920F931F93CE
:10B8B000CF93DF93CDB7DEB7A0970FB6F894DEBF76
:10B8C0000FBECDBF5C014115510561057105E9F45D
:10B8D00020E030E040E350E060E070E0A0960FB67A
:10B8E000F894DEBF0FBECDBFDF91CF911F910F91B6
:10B8F000FF90EF90DF90CF90BF90AF909F908F9090
:10B900007F906F905F904F905BC08E010F5F1F4FD5
:10B91000C12CD12C76014801422E512C612C712C66
:10B920008FEFC81AD80AE80AF80ACB01BA01A301B6
:10B9300092010F94FCC4CA01F80161938F01A9011F
:10B94000BC01411551056105710551F7F1E0CF1AB0
:10B95000D108E108F108F401EC0DFD1D80818A3069
:10B9600010F440E301C047E3480F552747FD5095C9
:10B97000652F752F20E030E0C50122D081E0C81A84
:10B98000D108E108F108EFEFCE16DE06EE06FE065E
:10B9900011F7A0960FB6F894DEBF0FBECDBFDF91B2
:10B9A000CF911F910F91FF90EF90DF90CF90BF90BC
:10B9B000AF909F908F907F906F905F904F90089581
:10B9C0002115310539F48091C00085FFFCCF4093EB
:10B9D000C60008952A30310509F43FC05BCF9A01B3
:10B9E000462F552747FD5095652F752FE9CFCF93EB
:10B9F000DF93EC0120E030E04DE050E060E070E0EB
:10BA0000DFDF20E030E04AE050E060E070E0CE01AF
:10BA1000DF91CF91D5CFFB012191BF01222339F0D6
:10BA20003091C00035FFFCCF2093C600F4CFDFCFAC
:10BA30009A01AB01662757FD6095762FC1CFCF9352
:10BA4000DF93EC019A01AB01662757FD6095762FD5
:10BA5000B7DFCE01DF91CF91CACFCF92DF92EF92C5
:10BA6000FF92CF93DF93EC016A017B0177FF0FC058
:10BA700020E030E04DE250E060E070E0A1DFF094C3
:10BA8000E094D094C094C11CD11CE11CF11C2AE0AC
:10BA9000B701A601CE01DF91CF91FF90EF90DF902B
:10BAA000CF90F8CE2115310539F48091C00085FF83
:10BAB000FCCF4093C6000895EDCECF93DF93EC0109
:10BAC0009A01462F50E060E070E0ECDFCE01DF919C
:10BAD000CF918DCFCF93DF93EC019A01AB0160E062
:10BAE00070E0E0DFCE01DF91CF9181CFCF93DF9384
:10BAF000EC01D8DFCE01DF91CF9179CF8F929F9269
:10BB0000AF92BF92CF92DF92EF92FF921F93CF93AB
:10BB1000DF93EC016A017B01122F20E030E0A901E4
:10BB2000C701B6010F940AC087FF0CC020E030E0C7
:10BB30004DE250E060E070E0CE0142DFF7FAF094B1
:10BB4000F7F8F094B12C60E070E080E09FE3B1166C
:10BB500041F020E030E040E251E40F9411C0B39492
:10BB6000F6CF9B01AC01C701B6010F941ABF6B0160
:10BB70007C010F947EC04B015C010F94AAC09B0115
:10BB8000AC01C701B6010F9419BF6B017C012AE01B
:10BB9000B501A401CE017EDE112361F0EBE7F4E0F4
:10BBA0008191882339F09091C00095FFFCCF80935C
:10BBB000C600F6CF112319F120E030E040E251E455
:10BBC000C701B6010F940BC36B017C010F9479C0C0
:10BBD0004B01AA2497FCA094BA2CB501A401CE0174
:10BBE0003CDFC501B4010F94ACC09B01AC01C7019F
:10BBF000B6010F9419BF6B017C011150DBCFDF91AF
:10BC0000CF911F91FF90EF90DF90CF90BF90AF90BA
:10BC10009F908F90089572CFCF93DF93EC016EDFEA
:10BC2000CE01DF91CF91E3CEFC01659175918591B5
:10BC3000949108952091DB073091DC07BC01C90184
:10BC40008252984F0F94F9C89093D2078093D107EE
:10BC500021E0892B09F420E0822F0895682F7727AF
:10BC600067FD70958091DB079091DC078252984FB9
:10BC70000F94C1C89093D2078093D10721E0892BFC
:10BC800009F420E0822F08958091D1079091D20786
:10BC90004AE050E060E070E001960D94DDC6CF937D
:10BCA000C82F40910B0250910C0260910D027091CF
:10BCB0000E024093D7095093D8096093D909709325
:10BCC000DA09209147023091480230938C0A209380
:10BCD0008B0A24E630E030934802209347020F9409
:10BCE00024B76093CD077093CE078093CF079093CE
:10BCF000D0078C2FCF910D947C3580E00F947C354C
:10BD00008091D7099091D809A091D909B091DA0909
:10BD100080930B0290930C02A0930D02B0930E023D
:10BD200080918B0A90918C0A9093480280934702ED
:10BD30000F9424B76093CD077093CE078093CF07FD
:10BD40009093D00708950F931F93CF93DF930091A3
:10BD5000D1071091D20765E470E0C8010F94C1C803
:10BD6000EC01C8010196209741F460E070E0DF919A
:10BD7000CF911F910F910D9475C5188260E070E00E
:10BD80000F9475C525E42883DF91CF911F910F9102
:10BD900008958091D1079091D20760E070E00196FC
:10BDA0000D9475C52091DB073091DC07E091D90730
:10BDB000F091DA072E173F0739F44091D7075091D9
:10BDC000D807141615068CF1AF01480F591FE2175A
:10BDD000F3073CF446595F4F81E04217530734F1B3
:10BDE00024C0BA0165597F4F6E3E7140E0F04E5F4E
:10BDF0005F4F4E3E514018F429363105A4F4865960
:10BE00009F4F821793078CF44DEE51E04E1B5F0B52
:10BE100060E070E0CF018352984F0F949CC810925D
:10BE2000DA071092D90781E0089580E008952F92F3
:10BE30003F924F925F926F927F928F929F92AF92BA
:10BE4000BF92CF92DF92EF92FF920F931F93CF9307
:10BE5000DF93CDB7DEB72A970FB6F894DEBF0FBEDB
:10BE6000CDBF9E838D83FC01E350F34FB490880FC8
:10BE7000991F880F991F9A878987805E954F9A83AB
:10BE80008983DC011D921D921D921C92139738E24A
:10BE9000232E3AE0332EF101E080F18002811381FC
:10BEA000A4E2BAE02D913D914D915C91E0E2FAE07F
:10BEB0006081718182819381ECE2CE2EEAE0DE2EF8
:10BEC0000F94C03289859A85845F924FADDE6B01F5
:10BED0007C016B2D772767FD7095872F972F0F9427
:10BEE000ACC02B013C0129853A852551364F3C8356
:10BEF0002B8320E030E040EC5FE3C701B6010F94F4
:10BF00000BC3A30192010F940BC3AB81BC816D9352
:10BF10007D938D939C931397E985FA85E75BFD4F9D
:10BF2000F887EF83608171818281938160930B0236
:10BF300070930C0280930D0290930E0220E030E08B
:10BF400040E752E40F9411C04B015C01A3EFB9E04C
:10BF5000ED90FD900D911C91EFEEF9E02081318183
:10BF600042815381ABEEB9E06D917D918D919C91B1
:10BF7000ACE0BAE0BF93AF93F7EFCF2EF9E0DF2E3E
:10BF80000F9415260F94B93EA981BA811D921D9276
:10BF90001D921C921397F101E080F18002811381C0
:10BFA000A4E2BAE02D913D914D915C91E0E2FAE07E
:10BFB0006081718182819381ACE2CA2EAAE0DA2E7F
:10BFC0000F94C03229853A852050334F1901C90199
:10BFD0002BDE9058A30192010F940BC3AB81BC815F
:10BFE0006D937D938D939C93139720E030E040E711
:10BFF00052E460910B0270910C0280910D029091BD
:10C000000E020F9411C04B015C01E3EFF9E0E080F8
:10C01000F18002811381AFEEB9E02D913D914D91F8
:10C020005C91EBEEF9E06081718182819381ACE0FB
:10C03000BAE0BF93AF93B7EFCB2EB9E0DB2E0F94EE
:10C0400015260F94B93EC101EFDD9B01AC010F94A1
:10C050001ABFA30192010F940BC3AB81BC816D93F6
:10C060007D938D939C93139720E030E040E05FE355
:10C07000EF81F88560817181828193810F940BC378
:10C0800060930B0270930C0280930D0290930E024A
:10C0900020E030E040E752E40F9411C04B015C0116
:10C0A000A3EFB9E0ED90FD900D911C91EFEEF9E05A
:10C0B0002081318142815381ABEEB9E06D917D9158
:10C0C0008D919C91ACE0BAE0BF93AF930F9415268D
:10C0D0000F94B93E89859A85885E924FA5DD0985C2
:10C0E0001A850C5E154FD8012D913D914D915C91B3
:10C0F0000F941ABFE981FA816083718382839383ED
:10C1000089859A85805D924F8FDD29853A85235DEB
:10C110003D4F7901D8012D913D914D915C910F9446
:10C120001ABFF701608371838283938389859A851F
:10C130008C5D924F79DD29853A852F5D3D4F7901E0
:10C14000D8012D913D914D915C910F941ABFF7014B
:10C150006083718382839383E981FA8180819181F5
:10C16000A281B381EB81FC8180839183A283B3831D
:10C1700010920B0210920C0210920D0210920E02FD
:10C180000F946435ED81FE81EF5EF54F81E0808391
:10C190000F900F900F900F900F900F902A960FB660
:10C1A000F894DEBF0FBECDBFDF91CF911F910F91ED
:10C1B000FF90EF90DF90CF90BF90AF909F908F90C7
:10C1C0007F906F905F904F903F902F9008954F9287
:10C1D0005F926F927F929F92AF92BF92CF92DF92C7
:10C1E000EF92FF920F931F93CF93DF937C015B013C
:10C1F0008A01E9019090920F911014C0FC01808196
:10C200009181A281B381FA0180839183A283B38358
:10C21000FB0180819181A281B38188839983AA8364
:10C22000BB837FC091FE55C0FC01208131814281DA
:10C2300053816091820F7091830F8091840F909150
:10C24000850F0F940BC32B013C01F5012081318137
:10C25000428153816091860F7091870F8091880F82
:10C260009091890F0F940BC39B01AC01C301B201E4
:10C270000F941ABFF8016083718382839383F7015F
:10C28000208131814281538160918A0F70918B0F9F
:10C2900080918C0F90918D0F0F940BC36B017C01DB
:10C2A000F501208131814281538160918E0F70911F
:10C2B0008F0F8091900F9091910F0F940BC39B0162
:10C2C000AC01C701B6010F941ABF688379838A83D2
:10C2D0009B8390FE26C020916A0F30916B0F409196
:10C2E0006C0F50916D0FF801608171818281938193
:10C2F0000F941ABFF8016083718382839383209126
:10C300006E0F30916F0F4091700F5091710F6881D7
:10C3100079818A819B810F941ABF688379838A838C
:10C320009B83DF91CF911F910F91FF90EF90DF9052
:10C33000CF90BF90AF909F907F906F905F904F9005
:10C3400008952F923F924F925F926F927F928F92B9
:10C350009F92AF92BF92CF92DF92EF92FF920F9394
:10C360001F93CF93DF93CDB7DEB728970FB6F8941E
:10C37000DEBF0FBECDBF8C011B019E012F5F3F4F63
:10C38000AE014B5F5F4F23DF20E030E0A9016D81FC
:10C390007E818F8198850F940AC087FF07C01D8218
:10C3A0001E821F821886FF24F39401C0F12C2DEC0D
:10C3B0003CEC4CE050EC69817A818B819C810F943C
:10C3C0000AC087FF0AC08DEC9CECACE0B0EC89831E
:10C3D0009A83AB83BC83FF24F39420E030E04AE7E8
:10C3E00053E46D817E818F8198850F9439C2181630
:10C3F00054F480E090E0AAE7B3E48D839E83AF839A
:10C40000B887FF24F39420E030E042E553E46981EB
:10C410007A818B819C810F9439C218164CF480E08C
:10C4200090E0A2E5B3E489839A83AB83BC8303C025
:10C43000FF2009F483C0C980DA80EB80FC808D8006
:10C440009E80AF80B8847090920F71100BC0F8017D
:10C4500080829182A282B382F101C082D182E28283
:10C46000F3826AC070FE1CC020916A0F30916B0F7E
:10C4700040916C0F50916D0FC501B4010F9419BF1D
:10C480004B015C0120916E0F30916F0F4091700F46
:10C490005091710FC701B6010F9419BF6B017C0158
:10C4A00071FE4AC02091720F3091730F4091740F4A
:10C4B0005091750FC501B4010F940BC32B013C01C2
:10C4C0002091760F3091770F4091780F5091790F2E
:10C4D000C701B6010F940BC39B01AC01C301B201AC
:10C4E0000F941ABFF8016083718382839383209134
:10C4F0007A0F30917B0F40917C0F50917D0FC501D9
:10C50000B4010F940BC34B015C0120917E0F30915D
:10C510007F0F4091800F5091810FC701B6010F949A
:10C520000BC39B01AC01C501B4010F941ABFF1010B
:10C530006083718382839383FF24F3948F2D2896E5
:10C540000FB6F894DEBF0FBECDBFDF91CF911F9124
:10C550000F91FF90EF90DF90CF90BF90AF909F90A2
:10C560008F907F906F905F904F903F902F900895A5
:10C57000682F87EF9FE00D946FCB089586EA9FE0C8
:10C580000F945DCB91E0811101C090E0892F089557
:10C59000FC012491222341F03091C00035FFFCCFF3
:10C5A0002093C6000196F4CF22E030E080EF96E0C1
:10C5B00032CBFC012491222341F03091C00035FFA1
:10C5C000FCCF2093C6000196F4CF2AE030E080EF44
:10C5D00096E068CA8091D7079091D8071816190677
:10C5E0000CF056C001979093D8078093D707892BFA
:10C5F00099F48091D4079091D507892B21F410925A
:10C60000DA071092D9078091D9079091DA079093B1
:10C61000DC078093DB073AC02091DB073091DC0711
:10C620002F5F3F4F2F5F3F4FF901E452F84F40819A
:10C630004111F8CFC901382F292F8D3E41E09407D1
:10C6400040F09093DC078093DB078D3E9140F1F43E
:10C650000EC00196FC01E452F84F4081442359F387
:10C660003093DB072093DC07832F922FEECF80E0FF
:10C6700090E0382F292F0196FC01E452F84F4081B9
:10C680004423B9F33093DB072093DC0781E008955E
:10C6900080E008959FDF8111FDCF08950F931F93D0
:10C6A000CF93DF93EC018036910514F080E052C007
:10C6B0008091D607811104C08DDF81E08093D60779
:10C6C0004091DB075091DC078091D9079091DA0700
:10C6D0004817590739F42091D7073091D807121617
:10C6E000130624F32091D4073091D50712161306B0
:10C6F00024F49C012F593F4F01C09C0184179507DA
:10C7000044F44C1B5D0B425051094217530774F21D
:10C7100009C0CE010196841795074CF44C1B5D0BA4
:10C72000425051095093DC074093DB0712C00BEED7
:10C7300011E00C1B1D0B021713070CF4B7CF60E0C0
:10C7400070E08DED97E00F949CC81093DC07009388
:10C75000DB0781E0DF91CF911F910F910895803623
:10C7600091050CF41FCB80E00895FF920F931F9367
:10C77000CF93DF93EC01F62E662321F00F942EC8A1
:10C780008C0109C0FC0101900020E9F78F010150E4
:10C790001109081B190BC801E2DF882309F474C0D2
:10C7A0008091D9079091DA07FC01E352F84F23E01A
:10C7B00020830196BE018352984FFF2019F00F94F9
:10C7C00027C802C00F94D5C8ECE3FDE0849188230C
:10C7D00041F09091C00095FFFCCF8093C600319648
:10C7E000F5CFE7EEF0E885919491FC0124912223A6
:10C7F00041F03091C00035FFFCCF2093C600019678
:10C80000F4CFE091D907F091DA07E252F84F819125
:10C81000882339F09091C00095FFFCCF8093C6002B
:10C82000F6CFEBEFFCE08491882341F09091C000BB
:10C8300095FFFCCF8093C6003196F5CF8091C00064
:10C8400085FFFCCF8AE08093C6000E5F1F4F80916A
:10C85000D9079091DA07080F191F0D3EF1E01F0765
:10C8600029F01093DA070093D90704C01092DA0771
:10C870001092D9078091D7079091D807019690938D
:10C88000D8078093D70748C0E2E4FDE0849188236D
:10C8900041F09091C00095FFFCCF8093C600319687
:10C8A000F5CFE7EEF0E885919491FC0124912223E5
:10C8B00041F03091C00035FFFCCF2093C6000196B7
:10C8C000F4CFFF2091F0FE018491882389F09091AC
:10C8D000C00095FFFCCF8093C6002196F4CF9091C5
:10C8E000C00095FFFCCF8093C60089918111F7CFDE
:10C8F000E4EEFCE007C09091C00095FFFCCF809370
:10C90000C600319684918111F6CF8091C00085FFD9
:10C91000FCCF8AE08093C600DF91CF911F910F91E9
:10C92000FF9008951F93CF93DF93EC01162F66239A
:10C9300019F00F942EC808C0FC0101900020E9F7FF
:10C94000CF0101978C1B9D0BA9DE882309F459C0E8
:10C950008091DB079091DC07FC01E352F84F23E064
:10C9600020830196BE018352984F112319F00F9432
:10C9700027C802C00F94D5C88091D7079091D807D7
:10C9800001969093D8078093D707ECE3FDE084915C
:10C99000882341F09091C00095FFFCCF8093C600A2
:10C9A0003196F5CFEBECFCE08491882341F0909137
:10C9B000C00095FFFCCF8093C6003196F5CFE09183
:10C9C000DB07F091DC07E252F84F8191882339F0C0
:10C9D0009091C00095FFFCCF8093C600F6CFE9ECA4
:10C9E000FCE08491882341F09091C00095FFFCCF3A
:10C9F0008093C6003196F5CF8091C00085FFFCCFB3
:10CA000042C0E2E4FDE08491882341F09091C000AF
:10CA100095FFFCCF8093C6003196F5CFE0EBFCE0AC
:10CA20008491882341F09091C00095FFFCCF8093C2
:10CA3000C6003196F5CF112391F0FE018491882331
:10CA400089F09091C00095FFFCCF8093C60021969D
:10CA5000F4CF9091C00095FFFCCF8093C6008991E0
:10CA60008111F7CFE9E9FCE007C09091C00095FF84
:10CA7000FCCF8093C600319684918111F6CF8091CE
:10CA8000C00085FFFCCF8AE08093C600DF91CF9184
:10CA90001F91089581E02091D7073091D807232B6B
:10CAA00009F080E008959B9AA3980895EF92FF9271
:10CAB0000F931F93CF93DF931F92CDB7DEB7898378
:10CAC0000F9432618981823009F468C0B4F58823FB
:10CAD00009F442C0813009F0F4C09FB7F894809106
:10CAE00002018460809302019FBFEFEFF1EE24E02A
:10CAF000E150F0402040E1F700C000009FB7F894FB
:10CB0000809102018B7F809302019FBF40E050E043
:10CB1000BA018DEE9FE00F9481CB40E050E0BA0166
:10CB200081EF9FE00F9481CB0F90DF91CF911F9108
:10CB30000F91FF90EF900D940892833009F45CC040
:10CB4000843009F0BEC00F90DF91CF911F910F91FB
:10CB5000FF90EF900D94B9999FB7F89480910201DE
:10CB60008460809302019FBF2FEF81EE94E02150FB
:10CB700080409040E1F700C000009FB7F89480919A
:10CB800002018B7F809302019FBF0F90DF91CF91B5
:10CB90001F910F91FF90EF900D94DB610F94DB617B
:10CBA00080EFE6DC10921C1810921B1860911D1883
:10CBB00084EC9FE00F946FCB6BE178E181EC9FE018
:10CBC0000F9460619FB7F894809102018460809314
:10CBD00002019FBF8FEF91EEE4E081509040E04072
:10CBE000E1F700C000009FB7F894809102018B7FAD
:10CBF000809302019FBF65C08BE89CE00F94BE78D4
:10CC00004AE75CE062E081E00F94B1A09FB7F8943E
:10CC1000809102018460809302019FBFFFEF21EEAB
:10CC200084E0F15020408040E1F700C000009FB751
:10CC3000F894809102018B7F809302019FBF109234
:10CC4000B9071092B80743E75CE063E083E00F9414
:10CC5000B1A04091B8075091B90763E083E00F9409
:10CC60003D61E12CF12C09E210E06FEFC7010F9458
:10CC70008DCBC701B8010F94E9C4892BD9F48091F9
:10CC8000B8079091B90701969093B9078093B807B8
:10CC90004CE65CE063E083E00F94B1A04091B807FC
:10CCA0005091B90763E083E00F943D618AE69CE010
:10CCB0000F94BE789FEFE91AF90AE114E0E1FE064D
:10CCC000A1F60F90DF91CF911F910F91FF90EF9000
:10CCD000089580E1E0E2FAE0ABEEB9E001900D9258
:10CCE0008A95E1F708954F925F926F927F928F92AB
:10CCF0009F92AF92BF92CF92DF92EF92FF92CF932B
:10CD0000DF9300D01F92CDB7DEB70F94B93E8BE40E
:10CD10000E942E5E882391F016D86B017C0120E0E2
:10CD200030E0A9010F9439C287FD08C0C0926D1090
:10CD3000D0926E10E0926F10F092701082E50E9417
:10CD40002E5E882361F00E94A35E6B017C0120E0CF
:10CD500030E0A9010F940AC087FF89C006C0C12C2A
:10CD6000D12CF0E8EF2EFFEBFF2E84E40E942E5E24
:10CD7000882329F00E94A35E4B015C0106C0812C30
:10CD8000912CE0E8AE2EEFEBBE2E87E50E942E5EE2
:10CD9000882329F00E94A35E2B013C0106C0412C90
:10CDA000512C70E8672E7FEB772E88E40E942E5E70
:10CDB000882339F00E94A35E69837A838B839C83E6
:10CDC00008C080E090E0A0E8BFEB89839A83AB8342
:10CDD000BC8320E030E0A901C501B4010F9439C241
:10CDE00087FD45C020E030E0A901C301B2010F94E6
:10CDF00039C287FD3CC020E030E0A90169817A8119
:10CE00008B819C810F9439C287FD31C020E030E0D6
:10CE1000A901C501B4010F940AC0882391F120E053
:10CE200030E040E05FE3C501B4010F940BC36B0138
:10CE30007C0129813A814B815C81C301B2010F944D
:10CE40000BC34B015C01A7019601C701B6010F940A
:10CE50000BC32BED3FE049E450E40F940BC39B015F
:10CE6000AC01C501B4010F9411C06B017C0120E03D
:10CE700030E0A901C701B6010F9439C287FF04C091
:10CE80000BC0C12CD12C7601C0926910D0926A10CF
:10CE9000E0926B10F0926C10ECE3FDE0849188233B
:10CEA00041F09091C00095FFFCCF8093C600319671
:10CEB000F5CFE4EEF7E08491882341F09091C00033
:10CEC00095FFFCCF8093C6003196F5CF40916D1051
:10CED00050916E1060916F107091701022E030E0F0
:10CEE00080EF96E00E940B5E8091C00085FFFCCF32
:10CEF0008AE08093C600EEEDF7E08491882341F04C
:10CF00009091C00095FFFCCF8093C6003196F5CF7D
:10CF1000C0906910D0906A10E0906B10F0906C1087
:10CF200020E030E0A901C701B6010F940AC08823B0
:10CF300069F022E030E0B701A60180EF96E00E94A0
:10CF40000B5E8091C00085FFFCCF11C0E9EDF7E0DA
:10CF50008491882341F09091C00095FFFCCF80938D
:10CF6000C6003196F5CF8091C00085FFFCCF8AE0E6
:10CF70008093C6000F900F900F900F90DF91CF918C
:10CF8000FF90EF90DF90CF90BF90AF909F908F90E9
:10CF90007F906F905F904F9008958330910510F4CB
:10CFA0000C94175F0895CF92DF92EF92FF920F9348
:10CFB0001F938FDE80E090E00E94175F81E090E099
:10CFC0000E94175FE090280AF090290A00912A0A2F
:10CFD00010912B0A2091240A3091250A4091260AAB
:10CFE0005091270A6091200A7091210A8091220AAB
:10CFF0009091230AACE2CA2EAAE0DA2E0F94C03236
:10D000001F910F91FF90EF90DF90CF900D946435BA
:10D010000F9424B76093CD077093CE078093CF070A
:10D020009093D007089520E030E0A90168EB71E00B
:10D0300084E50F9472BB69E170E080E090E00F94AA
:10D0400053B784E50F9498BE64E170E080E090E00F
:10D050000D9453B77F928F929F92AF92BF92CF92CF
:10D06000DF92EF92FF920F931F93CF93DF9300D045
:10D070001F92CDB7DEB7109243171092421710924D
:10D080004117109240170F94326185E09CE00F9495
:10D09000BE788E010F5F1F4F7E0125E0E20EF11C6E
:10D0A00080EF96E00E94255C8F3FEFEF9E07C1F373
:10D0B000F80181938F01EE15FF0591F789809A8021
:10D0C000AB80BC808091C00085FFFCCF8BE2809359
:10D0D000C600C12CD12C7601BBE27B2E8091520A76
:10D0E000882309F450C007E717E0C814D904EA04FC
:10D0F000FB04A1F080EF96E00E94255C8F3FFFEFDC
:10D100009F07C1F32FEFC21AD20AE20AF20AF8010E
:10D1100081938F01F7E0073B1F0739F767E777E057
:10D120008DE99AE00E940DCD8091C00085FFFCCF73
:10D130007092C6000F94224DC814D904EA04FB046F
:10D1400069F671DF60E08DE99AE00E9442CE1092AC
:10D15000520AE9EBF0E885919491FC012491222395
:10D1600041F03091C00035FFFCCF2093C6000196FE
:10D17000F4CF8091C00085FFFCCF8AE08093C60089
:10D1800080E090E000C00F900F900F900F90DF9123
:10D19000CF911F910F91FF90EF90DF90CF90BF90B4
:10D1A000AF909F908F907F9008950F9424B76093D5
:10D1B000CD077093CE078093CF079093D007E0916F
:10D1C000DB07F091DC07E352F84F80818130B9F43E
:10D1D000E3E6FEE785919491FC012491222341F03E
:10D1E0003091C00035FFFCCF2093C6000196F4CFEC
:10D1F0008091C00085FFFCCF8AE08093C60008952F
:10D2000080EF96E00E94415CE3E5FDE78591949113
:10D21000FC012491222341F03091C00035FFFCCF66
:10D220002093C6000196F4CF4091CF095091D009C8
:10D230006091D1097091D2094F5F5F4F6F4F7F4F5F
:10D240002AE030E080EF96E00E94E05C8091C00030
:10D2500085FFFCCF8AE08093C600A7CF8F929F9274
:10D26000AF92BF92CF92DF92EF92FF920F931F93F4
:10D27000CF93DF93C7E2EC2EC4E0FC2E00E21AE06D
:10D28000CBEED9E08DE8C82E8AE0D82EF701819147
:10D290007F010E942E5E882319F10E94C95E4B0116
:10D2A0005C01F6018081811103C06091CA0901C04F
:10D2B00061E070E080E090E00F94ACC0F801208164
:10D2C0003181428153810F940BC39B01AC01C50195
:10D2D000B4010F941ABF688379838A839B8309C042
:10D2E000F80180819181A281B38188839983AA8387
:10D2F000BB830C5F1F4F2496FFEFCF1ADF0A8BE230
:10D30000E81684E0F80611F686E40E942E5E882373
:10D31000D9F00E94C95E6B017C016093DB097093B8
:10D32000DC098093DD099093DE0920E030E0A9015B
:10D330000F9439C2181644F4C0920B02D0920C021A
:10D34000E0920D02F0920E02DF91CF911F910F91AA
:10D35000FF90EF90DF90CF90BF90AF909F908F9015
:10D3600008957CDF89E40E942E5E882359F00E9494
:10D37000C95E6093DF097093E0098093E10990939F
:10D38000E20908C01092DF091092E0091092E10949
:10D390001092E2098AE40E942E5E882359F00E94CE
:10D3A000C95E6093E3097093E4098093E509909363
:10D3B000E60908951092E3091092E4091092E50934
:10D3C0001092E6090895CF92DF92EF92FF92CF93E9
:10D3D000DF93EC01BC016C5F7F4F0E94A16120E0F4
:10D3E00030E0A901609135027091360280913702D8
:10D3F000909138020F941ABF6B017C019B01AC0124
:10D40000688579858A859B850F940AC087FF04C04B
:10D41000C886D986EA86FB86C0902902D0902A0267
:10D42000E0902B02F0902C02A70196016885798587
:10D430008A859B850F9439C2181624F4C886D9862C
:10D44000EA86FB86DF91CF91FF90EF90DF90CF903F
:10D4500008952F923F924F925F926F927F928F9298
:10D460009F92AF92BF92CF92DF92EF92FF920F9373
:10D470001F93CF93DF93CDB7DEB7AB970FB6F8947A
:10D48000DEBF0FBECDBF9F878E87798B688B5B8B8E
:10D490004A8B3D8B2C8B1F8B0E8BED82DC018D908C
:10D4A0009D90AD90BC904090200A5090210A6090D1
:10D4B000220A7090230ADB018D919D910D90BC9101
:10D4C000A02D88879987AA87BB87C090240AD0900F
:10D4D000250AE090260AF090270A2091280A309128
:10D4E000290A40912A0A50912B0AEA89FB89608116
:10D4F0007181828193810F9419BF688F798F8A8F90
:10D500009B8F8091930F811173C0AE89BF898D90DD
:10D510009D90AD90BC90EA89FB89E080F18002810A
:10D520001381A889B9892D913D914D915C91EE852A
:10D53000FF856081718182819381FE013596FF9321
:10D54000EF93CC88DD880F941526EE85FF858081CA
:10D550009181A281B3818093200A9093210AA093A4
:10D56000220AB093230AE889F98980819181A281F6
:10D57000B3818093240A9093250AA093260AB0933E
:10D58000270AEA89FB8980819181A281B3818093F6
:10D59000280A9093290AA0932A0AB0932B0AEC89AF
:10D5A000FD8980819181A281B38180932C0A90931F
:10D5B0002D0AA0932E0AB0932F0A0F900F90AB96CE
:10D5C0000FB6F894DEBF0FBECDBFDF91CF911F9194
:10D5D0000F91FF90EF90DF90CF90BF90AF909F9012
:10D5E0008F907F906F905F904F903F902F90089515
:10D5F000A3019201C501B4010F9419BF2B013C0195
:10D6000020E030E0A9010F9439C2530142011816FD
:10D6100024F0B7FAB094B7F8B094A70196016885E2
:10D6200079858A859B850F9419BF688779878A8752
:10D630009B8720E030E0A9010F9439C22885398505
:10D640004A855B8518160CF05058C501B4010F943B
:10D650001ABF6B017C0120E030E0A9010F9439C2B0
:10D6600018160CF052CF20E030E040EF51E4C70133
:10D67000B6010F9411C00F94F7BF0F9479C07D8746
:10D680006C87623071050CF440CF20912C0A3091E8
:10D690002D0A40912E0A50912F0AAC89BD896D91B7
:10D6A0007D918D919C910F9419BF6C8F7D8F8E8F82
:10D6B0009F8F22242394312C8C859D85AA2797FD4A
:10D6C000A095BA2F88A799A7AAA7BBA7DE01159690
:10D6D000BF83AE83B101882777FD8095982F0F9483
:10D6E000ACC06B017C0168A579A58AA59BA50F94A8
:10D6F000ACC09B01AC01C701B6010F9411C06B0116
:10D700007C01EE89FF8980809180A280B3802C8D7E
:10D710003D8D4E8D5F8D0F940BC39B01AC016091CD
:10D720002C0A70912D0A80912E0A90912F0A0F9445
:10D730001ABF69837A838B839C83288D398D4A8DA8
:10D740005B8DC701B6010F940BC32091280A30915D
:10D75000290A40912A0A50912B0A0F941ABF68A3F4
:10D7600079A38AA39BA3288539854A855B85C70150
:10D77000B6010F940BC32091240A3091250A4091E1
:10D78000260A5091270A0F941ABF6CA37DA38EA37B
:10D790009FA3A3019201C701B6010F940BC320916F
:10D7A000200A3091210A4091220A5091230A0F94B5
:10D7B0001ABFFF81FF932E812F93DE0111966D0119
:10D7C000E8A0F9A00AA11BA12CA13DA14EA15FA137
:10D7D0000F941526BFEF2B1A3B0A0F900F90EC8584
:10D7E000FD852E163F0609F075CF8FCE4F925F92C2
:10D7F0006F927F928F929F92AF92BF92CF92DF9261
:10D80000EF92FF920F931F93CF93DF93CDB7DEB7C5
:10D8100028970FB6F894DEBF0FBECDBF8BEE99E010
:10D82000D2DD0F9424B76093CD077093CE07809319
:10D83000CF079093D0078091EB099091EC09A091CC
:10D84000ED09B091EE098D839E83AF83B8879C016B
:10D85000AD016091200A7091210A8091220A909175
:10D86000230A0F940AC0811197C04090EF0950908D
:10D87000F0096090F1097090F209A30192016091A2
:10D88000240A7091250A8091260A9091270A0F9404
:10D890000AC0811181C020E030E040E752E460918D
:10D8A0000B0270910C0280910D0290910E020F9468
:10D8B00011C04B015C01E090F309F090F409009174
:10D8C000F5091091F6098CE09AE09F938F9327EF6A
:10D8D000C22E29E0D22EA30192016D817E818F811B
:10D8E00098850F9415260F900F908091EB099091D9
:10D8F000EC09A091ED09B091EE098093200A909374
:10D90000210AA093220AB093230A8091EF099091F3
:10D91000F009A091F109B091F2098093240A909343
:10D92000250AA093260AB093270A8091F3099091C3
:10D93000F409A091F509B091F6098093280A909313
:10D94000290AA0932A0AB0932B0A8091F709909193
:10D95000F809A091F909B091FA0980932C0A9093E3
:10D960002D0AA0932E0AB0932F0A28960FB6F8948A
:10D97000DEBF0FBECDBFDF91CF911F910F91FF9002
:10D98000EF90DF90CF90BF90AF909F908F907F905F
:10D990006F905F904F900895E0900C0A609147025D
:10D9A00070914802882777FD8095982F0F94ACC01E
:10D9B00020910B0230910C0240910D0250910E0209
:10D9C0000F940BC32EE333EC4EE259E30F940BC3D9
:10D9D00069837A838B839C838E010F5F1F4F27EFB0
:10D9E00039E043EF59E06FEE79E08BEE99E031DDFD
:10D9F0007CCF4F925F926F927F928F929F92AF9265
:10DA0000BF92CF92DF92EF92FF920F931F93CF932B
:10DA1000C62FE0910C0AF0E0882309F4D9C0DF0199
:10DA2000A85FB54F8C918111AFC18091200A909170
:10DA3000210AA091220AB091230A8093EB099093C6
:10DA4000EC09A093ED09B093EE098091240A90911E
:10DA5000250AA091260AB091270A8093EF09909396
:10DA6000F009A093F109B093F2098091280A9091EE
:10DA7000290AA0912A0AB0912B0A8093F309909366
:10DA8000F409A093F509B093F609C0902C0AD09040
:10DA90002D0AE0902E0AF0902F0AC092F709D0923A
:10DAA000F809E092F909F092FA09EE0FFF1FEE0F64
:10DAB000FF1FE75CFD4F2081318142815381662346
:10DAC00049F06091190270911A0280911B029091A5
:10DAD0001C0208C060911D0270911E0280911F02FD
:10DAE000909120020F9411C09B01AC01C701B601B7
:10DAF0000F941ABF60932C0A70932D0A80932E0AFC
:10DB000090932F0A8CE29AE00F94443480900B0299
:10DB100090900C02A0900D02B0900E0220E030E038
:10DB200040E752E46091150270911602809117024D
:10DB3000909118020F940BC360930B0270930C0228
:10DB400080930D0290930E02E0910C0AF0E0E85FE2
:10DB5000F54F81E080834ADE2091040A3091050A66
:10DB60004091060A5091070A6091280A7091290A8B
:10DB700080912A0A90912B0A0F9419BF7B018C0186
:10DB80006093280A7093290A80932A0A90932B0A9B
:10DB90002091240A3091250A4091260A5091270AA3
:10DBA0006091200A7091210A8091220A9091230AA3
:10DBB000ECE2CE2EEAE0DE2E0F94C03217DE809229
:10DBC0000B0290920C02A0920D02B0920E02DCC0E9
:10DBD000E85FF54F8081882309F4D6C08090200A41
:10DBE0009090210AA090220AB090230A8092EB091B
:10DBF0009092EC09A092ED09B092EE094090240AAF
:10DC00005090250A6090260A7090270A4092EF09EA
:10DC10005092F0096092F1097092F2096091280A1D
:10DC20007091290A80912A0A90912B0A6093F30936
:10DC30007093F4098093F5099093F60900912C0AEA
:10DC400010912D0A20912E0A30912F0A0093F70986
:10DC50001093F8092093F9093093FA092091040AE6
:10DC60003091050A4091060A5091070A0F941ABF95
:10DC70007B018C016093280A7093290A80932A0AF9
:10DC800090932B0A3CE2C32E3AE0D32EA3019201DB
:10DC9000C501B4010F94C03210910C0ACC2389F055
:10DCA0002091FC093091FD094091FE095091FF0936
:10DCB0006091190270911A0280911B0290911C02CE
:10DCC00010C02091000A3091010A4091020A50913F
:10DCD000030A60911D0270911E0280911F029091B3
:10DCE00020020F941ABF24E0129FF0011124E75C78
:10DCF000FD4F20813181428153810F9411C09B01DE
:10DD0000AC0160912C0A70912D0A80912E0A90919D
:10DD10002F0A0F9419BF60932C0A70932D0A8093D9
:10DD20002E0A90932F0A8CE29AE00F944434C0900C
:10DD30000B02D0900C02E0900D02F0900E0220E059
:10DD400030E040E752E4609111027091120280913C
:10DD50001302909114020F940BC360930B02709303
:10DD60000C0280930D0290930E02E0910C0AF0E0F9
:10DD7000E85FF54F10823ADDC0920B02D0920C02A0
:10DD8000E0920D02F0920E02CF911F910F91FF9041
:10DD9000EF90DF90CF90BF90AF909F908F907F904B
:10DDA0006F905F904F900895AF92BF92CF92DF92A5
:10DDB000EF92FF920F931F93CF93DF93D82F209171
:10DDC000E3093091E4094091E5095091E609609139
:10DDD000DF097091E0098091E1099091E2090F94C7
:10DDE00046C2C62F172F082FF92E60914702709157
:10DDF0004802882777FD8095982F0F94ACC020911A
:10DE00000B0230910C0240910D0250910E020F94C2
:10DE10000BC320E030E040E752E40F9411C020E053
:10DE200030E048EC52E40F9411C020910C0A2F937B
:10DE3000DF93FF920F931F93CF935B016C01B2E0CE
:10DE4000EB2E01E020E04FED59E06BEE79E080E24F
:10DE50009AE00F94A11B8091EB099091EC09A0919D
:10DE6000ED09B091EE098093200A9093210AA093C6
:10DE7000220AB093230A8091EF099091F009A091B2
:10DE8000F109B091F2098093240A9093250AA09396
:10DE9000260AB093270A8091F3099091F409A09182
:10DEA000F509B091F6098093280A9093290AA09366
:10DEB0002A0AB0932B0A8091F7099091F809A09152
:10DEC000F909B091FA0980932C0A90932D0AA09336
:10DED0002E0AB0932F0A0F9424B76093CD07709346
:10DEE000CE078093CF079093D0070F900F900F909D
:10DEF0000F900F900F90DF91CF911F910F91FF9096
:10DF0000EF90DF90CF90BF90AF900895CF93DF93C5
:10DF10001F92CDB7DEB78C01F8940F94BA45179ACB
:10DF20001092110A169A1092120A149A60E087E46D
:10DF30000F940FB9E2E4FDE08491882341F09091C1
:10DF4000C00095FFFCCF8093C6003196F5CFE3E08B
:10DF5000F1E885919491FC012491222341F03091C4
:10DF6000C00035FFFCCF2093C6000196F4CF80910E
:10DF7000C00085FFFCCF8AE08093C6000115110523
:10DF8000E1F0F8018491F801882349F09091C000F4
:10DF900095FFFCCF8093C60031968491F5CF809198
:10DFA000C00085FFFCCF8AE08093C600BE016F5F92
:10DFB0007F4FC8010F9401650BC0E091530AF0E058
:10DFC000EE0FFF1FED51F048859194910F9475620B
:10DFD000789406E010E00150110951F068EC70E00F
:10DFE00080E090E00F9453B780E00F94CB63F3CFC1
:10DFF000F894FFCF0F94BA458091BB07811142C0BE
:10E0000081E08093BB078091CF099091D009A091C6
:10E01000D109B091D2098093CB099093CC09A093F8
:10E02000CD09B093CE09E2E4FDE08491882341F06C
:10E030009091C00095FFFCCF8093C6003196F5CF3C
:10E04000E9EFF0E885919491FC012491222341F0BD
:10E050003091C00035FFFCCF2093C6000196F4CF6D
:10E060008091C00085FFFCCF8AE08093C600E091DC
:10E07000530AF0E0EE0FFF1FE552F54885919491A9
:10E080000D944A6208958091BB070895CF93DF9362
:10E09000EC0180910C0A8093BC0784E50E942E5EFF
:10E0A000811102C080E084C00E94C95E0F947EC0CE
:10E0B0006093BC076623B1F3ECE3FDE08491882311
:10E0C00041F09091C00095FFFCCF8093C60031963F
:10E0D000F5CFCD36D10509F435C064F4C836D10585
:10E0E000B1F0C936D10509F052C0EBE8FFE7A591C0
:10E0F000B49124C0CA3DD10509F432C0CD3DD1054B
:10E1000009F045C0EFE7FFE7A591B4913DC0EDE808
:10E11000FFE785919491FC012491222309F437C0F3
:10E120003091C00035FFFCCF2093C6000196F3CF9D
:10E130009091C00095FFFCCF8093C6008D91811116
:10E14000F7CF25C0E9E8FFE7A591B4918D91882329
:10E15000F1F09091C00095FFFCCF8093C600F6CF00
:10E16000E1E8FFE7A591B4918D91882381F090912A
:10E17000C00095FFFCCF8093C600F6CF9091C00001
:10E1800095FFFCCF8093C6008D918111F7CF6091F0
:10E19000BC0770E04AE050E080EF96E00E94185D16
:10E1A0008091C00085FFFCCF8AE08093C60081E0AB
:10E1B000DF91CF9108954F925F926F927F928F92ED
:10E1C0009F92AF92BF92CF92DF92EF92FF92CF9346
:10E1D000DF9300D01F92CDB7DEB72B013C0129831E
:10E1E0003A834B835C838DEE9FE00F945DCB8F3F32
:10E1F00001F58EEE9FE00F945DCB8F3FD1F48FEE53
:10E200009FE00F945DCB8F3FA1F480EF9FE00F94D0
:10E210005DCB8F3F71F440E050E0BA018DEE9FE09E
:10E220000F9481CB40E050E0BA0181EF9FE00F9462
:10E2300081CB81EF9FE00F9465CB4B015C018DEEAC
:10E240009FE00F9465CB6B017C0169817A818B81A2
:10E250009C812CE330E040E050E00F94FCC4C20EFF
:10E26000D31EE41EF51EB701A6018DEE9FE00F94AC
:10E2700081CBC301B20128EE33E040E050E00F94BF
:10E28000FCC4BA01A901480D591D6A1D7B1D81EF0F
:10E290009FE00F9481CB10924C0A10924D0A10927D
:10E2A0004E0A10924F0A0F900F900F900F90DF912F
:10E2B000CF91FF90EF90DF90CF90BF90AF909F9065
:10E2C0008F907F906F905F904F9008952F923F9224
:10E2D0004F925F926F927F928F929F92AF92BF9276
:10E2E000CF92DF92EF92FF920F931F93CF93DF9322
:10E2F000CDB7DEB76F970FB6F894DEBF0FBECDBFB8
:10E300008FE590E00E94D25E882309F4A8C4A12C76
:10E3100052EFE52E5BE0F52E6AE0962EBB24B39417
:10E3200079EFC72E70E8D72E809171079091720710
:10E330002091730730917407821B930B8F77992775
:10E34000009709F4C1C08F379105B9F4F7018491A2
:10E35000E2EFFBE0882349F09091C00095FFFCCFED
:10E360008093C60031968491F5CF8091C00085FFDF
:10E37000FCCF9092C600AA24A39480EF96E00E945E
:10E38000255C182F0F9424B76093990A70939A0A0A
:10E3900080939B0A90939C0A0F9424B76093950AEC
:10E3A0007093960A8093970A9093980A17FDBCCFB2
:10E3B0002091D4073091D5071A3031F01D3021F06B
:10E3C0002F3531050CF468C02115310509F40CC254
:10E3D0000091D9071091DA07F901E352F84FE00FE5
:10E3E000F11F11828091D30781113CC00252184F56
:10E3F00060E473E0C8010F94F9C89093D20780934A
:10E40000D107892B09F0A8C26EE470E0C8010F940F
:10E41000C1C89093D2078093D107892B09F0E7C137
:10E420009BC2F801E352F84FB082F3010190002043
:10E43000E9F73197E619F709C80102968E0F9F1F79
:10E440008D3E31E0930709F482C29093DA078093FE
:10E45000D9078091D7079091D80701969093D80754
:10E460008093D7071092D5071092D4078091710737
:10E47000909172072091730730917407821B930B60
:10E480008F779927892B09F4EAC38FE590E00E94E2
:10E49000D25E811149CFE3C31B3311F4B092D3078D
:10E4A0008091D307811140CFE091D907F091DA072D
:10E4B000C90101969093D5078093D407E20FF31F0B
:10E4C000E252F84F108330CF80911D18882309F451
:10E4D00062C00F9424B76093950A7093960A809354
:10E4E000970A9093980A0091990A10919A0A20919C
:10E4F0009B0A30919C0ADC01CB01801B910BA20B83
:10E50000B30B81329340A105B10508F444C0E091FA
:10E51000D407F091D5071E161F060CF03CC0809161
:10E52000D9079091DA07E352F84FE80FF91F1182EB
:10E53000DC01A252B84FFD0101900020E9F73197AC
:10E54000EA1BFB0B02968E0F9F1F9093DA078093B6
:10E55000D9078D3E914021F41092DA071092D90725
:10E560008091D7079091D80701969093D807809310
:10E57000D7071092D5071092D407E4EEFBE0849100
:10E58000882309F46CC39091C00095FFFCCF809361
:10E59000C6003196F4CFAA20A9F02091D40730917B
:10E5A000D5071216130674F48091D9079091DA07F3
:10E5B000821B930B9093DA078093D9071092D507AB
:10E5C0001092D40780919F0A882309F448C3809150
:10E5D000D4079091D507892B09F041C38091D707C3
:10E5E0009091D807892B11F41092760798EE492E56
:10E5F00093E0592E612C712C2CE3822E912CA12CAE
:10E60000B12C8E010F5F1F4F34E0232E312C40912F
:10E610003B0D50913C0D60913D0D70913E0D8091F0
:10E62000330D9091340DA091350DB091360D4817F2
:10E6300059076A077B0708F012C38091760781119A
:10E640000EC380918E0C90918F0CA091900CB09184
:10E65000910C80933B0D90933C0DA0933D0DB09396
:10E660003E0D86E89CE00E9499BB8F8F8A3021F096
:10E67000BF8DBD3009F068C240913B0D50913C0DFB
:10E6800060913D0D70913E0D8091330D9091340D50
:10E69000A091350DB091360D481759076A077B07D1
:10E6A00008F495C0EBEBF0E885919491FC0124917E
:10E6B000211163C28091C00085FFFCCFFAE0F09386
:10E6C000C6000F9424B76093C1077093C20780936C
:10E6D000C3079093C407C090C507D090C607E090C9
:10E6E000C707F090C8076C197D098E099F09C09073
:10E6F0005E0AD0905F0AE090600AF090610A6C199F
:10E700007D098E099F09A30192010F94FCC4690140
:10E710007A0110925E0A10925F0A1092600A1092BB
:10E72000610A60914C0A70914D0A80914E0A909155
:10E730004F0A41DDC701B601A50194010F94FCC445
:10E74000CA01B901A50194010F94FCC47F936F9392
:10E75000C701B60120E13EE040E050E00F94FCC468
:10E760003F932F93A0EDBBE0BF93AF931F930F9305
:10E770000F9441C9ECE3FDE084910FB6F894DEBF3D
:10E780000FBECDBF811101C2F8018191811106C276
:10E790008091C00085FFFCCF3AE03093C600C801ED
:10E7A0000F943D628DE99AE00E9437D361E08DE9D4
:10E7B0009AE00E944ACD80911D18882341F086E09E
:10E7C00090E00F94AD7130922218209221184F8D55
:10E7D000433219F481E080937607E091D407F091F9
:10E7E000D507309709F0E1C11092D30738C26EE423
:10E7F00070E0C8010F94C1C89093D2078093D107ED
:10E80000009709F446C04AE050E060E070E00196ED
:10E810000F94DDC66093D3097093D4098093D50912
:10E820009093D6094090CF095090D0096090D109BB
:10E830007090D209FFEF4F1A5F0A6F0A7F0A0091AA
:10E84000D9071091DA07641575058605970509F44F
:10E85000C2C06DEE7BE0C8018252984F0F946CC825
:10E86000892B09F0B8C040C1E091D107F091D207DF
:10E8700010828091D3099091D409A091D509B091CB
:10E88000D6098093CF099093D009A093D109B09372
:10E89000D2098091D9079091DA0767E470E082523B
:10E8A000984F0F94C1C89093D2078093D1070097D7
:10E8B00009F43AC020919F0A211108C02AE030E0F3
:10E8C00030937B0A20937A0AB092820A2091BB0788
:10E8D000222351F14AE050E060E070E001960F948D
:10E8E000DDC66430710500F5F60185919491FC0157
:10E8F0002491222341F03091C00035FFFCCF2093BA
:10E90000C6000196F4CF8091C00085FFFCCF9092A5
:10E91000C600E091530AF0E0EE0FFF1FE552F54804
:10E92000859194910F944A620091D9071091DA076A
:10E9300098012252384F390166E473E0C9010F94FF
:10E94000CCC8892B09F06DCD80E090E0DFDA109221
:10E95000DA071092D9077DCD6AE270E0C8010F9402
:10E96000C1C8892B09F495CFE2E4FDE084918823A6
:10E9700041F09091C00095FFFCCF8093C600319686
:10E98000F5CFEBEFF0E885919491FC0124912223DF
:10E9900041F03091C00035FFFCCF2093C6000196B6
:10E9A000F4CF4091CF095091D0096091D109709175
:10E9B000D2092AE030E080EF96E00E94E05C80918E
:10E9C000C00085FFFCCF8AE08093C6001092D50777
:10E9D0001092D40744C10252184F6AE270E0C80195
:10E9E0000F94C1C89093D2078093D107009709F084
:10E9F00035C0E2E4FDE08491882341F09091C000AD
:10EA000095FFFCCF8093C6003196F5CFEDEFF0E88F
:10EA100085919491FC012491222341F03091C00012
:10EA200035FFFCCF2093C6000196F4CF4091CF096B
:10EA30005091D0096091D1097091D2092AE030E05B
:10EA400080EF96E00E94E05C8091C00085FFFCCFE3
:10EA50008AE08093C6000E940069B8CFF80110E0F8
:10EA6000E817F90719F021911227FACF4AE050E090
:10EA700060E070E0CF0101960F94DDC6212F30E0F9
:10EA80002617370709F4F0CEE2E4FDE084918823ED
:10EA900041F09091C00095FFFCCF8093C600319665
:10EAA000F5CFE7E0F1E885919491FC0124912223D0
:10EAB00041F03091C00035FFFCCF2093C600019695
:10EAC000F4CF4091CF095091D0096091D109709154
:10EAD000D2092AE030E080EF96E00E94E05C80916D
:10EAE000C00085FFFCCFB4CFE2E4FDE08491882331
:10EAF00041F09091C00095FFFCCF8093C600319605
:10EB0000F5CFE1E0F1E885919491FC012491222375
:10EB100041F03091C00035FFFCCF2093C600019634
:10EB2000F4CF4091CF095091D0096091D1097091F3
:10EB3000D2092AE030E080EF96E00E94E05C80910C
:10EB4000C00085FFFCCF84CFEF8DE33229F4209104
:10EB5000D307211104C090CDFF8DFA33C1F320916A
:10EB6000D4073091D5072F3531050CF085CD8F3F77
:10EB70004FEF940709F058C07FCD3091C00035FFAA
:10EB8000FCCF2093C600019691CD9091C00095FFD7
:10EB9000FCCF8093C60031968491F4CD9091C00053
:10EBA00095FFFCCF8093C600F0CD8091D90790915E
:10EBB000DA07E352F84FE80FF91F1182FC01E35224
:10EBC000F84FA2E0A0832091D7073091D8072F5F9C
:10EBD0003F4F3093D8072093D707DC01A252B84F9C
:10EBE000FD0101900020E9F73197EA1BFB0B02962B
:10EBF0008E0F9F1F8D3EB1E09B0729F09093DA079F
:10EC00008093D90704C01092DA071092D9071092A6
:10EC1000D3071092D5071092D4078FE590E00E9499
:10EC2000D25E8111F4CC1BC0EF8DEB3319F4F1E00F
:10EC3000F093D3074091D3074111E9CCE091D90774
:10EC4000F091DA07A9014F5F5F4F5093D5074093CA
:10EC5000D407E20FF31FE252F84F8083D8CC6F96AF
:10EC60000FB6F894DEBF0FBECDBFDF91CF911F91DD
:10EC70000F91FF90EF90DF90CF90BF90AF909F905B
:10EC80008F907F906F905F904F903F902F9008955E
:10EC9000CF92DF92EF92FF920F931F93CF93C82FE3
:10ECA0008091D7079091D80703970CF40FDB0F944E
:10ECB00024B70091C9071091CA072091CB07309162
:10ECC000CC07C090CD07D090CE07E090CF07F09052
:10ECD000D0076C197D098E099F09061717072807A9
:10ECE000390738F4012B022B032B19F080E090E058
:10ECF0000DD940910702509108026091090270916C
:10ED00000A02452B462B472B19F10F9424B700918B
:10ED1000CD071091CE072091CF073091D007601B0F
:10ED2000710B820B930B0091070210910802209146
:10ED3000090230910A02061717072807390740F41D
:10ED40009091721080917110981302C0CC2349F0F9
:10ED5000CF911F910F91FF90EF90DF90CF900D9486
:10ED60008424179A1092110A169A1092120A149A71
:10ED7000EFCFCF92DF92EF92FF922091300A2223C1
:10ED8000F1F020E030E040E05FE30F940BC36B0153
:10ED90007C0120E030E0A9010F940AC0882379F0BB
:10EDA000A7019601C701B6010F940BC32BED3FE0FD
:10EDB00049E450E40F940BC39B01AC0104C020E074
:10EDC00030E040E85FE360E070E080E89FE30F94AC
:10EDD00011C0FF90EF90DF90CF90089560913D02B9
:10EDE00070913E0280913F0290914002C2DF609399
:10EDF000390270933A0280933B0290933C0208954B
:10EE0000CF93DF93EC010F94224D81E041DF80E04E
:10EE10000F94CB63209799F0C233D10540F062E3A1
:10EE200070E080E090E00F9453B7E297ECCFBE0122
:10EE300080E090E00F9453B7C0E0D0E0E4CFDF91E2
:10EE4000CF9108952F923F924F925F926F927F924F
:10EE50008F929F92AF92BF92CF92DF92EF92FF92EA
:10EE60001F93CF93DF934B015C01CC24CA94DC2C1D
:10EE700076014EEC242E47E0342E58EE452E53E01A
:10EE8000552E612C712C1AE08091FB09811126C14D
:10EE90002FEFC216D206E206F20651F0F7FC1EC1B1
:10EEA0000F9424B76C197D09683B7B4008F016C1AC
:10EEB0000F9424B7681979098A099B09693E734040
:10EEC0008105910508F47FC080911D18811177C0DC
:10EED000E6EDF7E08491882341F09091C00095FF22
:10EEE000FCCF8093C6003196F5CFE091BC0724E0BB
:10EEF000E29FF0011124E65CF84E4081518162816D
:10EF0000738121E030E080EF96E00E940B5EE2ED3D
:10EF1000F7E08491882341F09091C00095FFFCCFE9
:10EF20008093C6003196F5CF6091BC0770E04AE04F
:10EF300050E080EF96E00E94185DF1018491EEECC4
:10EF4000F7E0882349F09091C00095FFFCCF8093B3
:10EF5000C60031968491F5CFF7FE03C0E6E8F6E0EF
:10EF600025C00F9424B74B015C01C701B60168545A
:10EF7000744F8F4F9F4F681979098A099B09A30124
:10EF800092010F94FCC4BA01A9012AE030E080EF9D
:10EF900096E00E94E05C8091C00085FFFCCF0DC030
:10EFA0009091C00095FFFCCF8093C60081918111A4
:10EFB000F7CF8091C00085FFFCCF1093C6000F945F
:10EFC00024B74B015C010F94224D80E061DE80E0AC
:10EFD0000F94CB63FFEFCF16DF06EF06FF0609F0B5
:10EFE00046C08091BA07E091BC07F0E0EF01CC0F7A
:10EFF000DD1FCC0FDD1FC65CD84EEE0FFF1FEE5B92
:10F00000F84E8823D1F080819181BC01882777FD5B
:10F010008095982F0F94ACC020E030E040E85FE38B
:10F020000F9419BF9B01AC01688179818A819B8112
:10F030000F9439C287FF4DC027CF80819181BC01D9
:10F04000882777FD8095982F0F94ACC020E030E0A2
:10F0500040E85FE30F941ABF9B01AC01688179819E
:10F060008A819B810F940AC018169CF50DCFF7FC7E
:10F070000BCFE091BC07F0E0EF01CC0FDD1FCC0F10
:10F08000DD1FC65CD84EEE0FFF1FEE5BF84E808191
:10F090009181BC01882777FD8095982F0F94ACC093
:10F0A0009B01AC01688179818A819B810F9419BF92
:10F0B0000F9479C097FF07C09095809570956195E2
:10F0C0007F4F8F4F9F4F66307105810591050CF47E
:10F0D000DBCE0F9424B76B017C01D6CEDF91CF91AC
:10F0E0001F91FF90EF90DF90CF90BF90AF909F90D7
:10F0F0008F907F906F905F904F903F902F900895EA
:10F10000CF93DF931F921F92CDB7DEB7BE016F5F23
:10F110007F4F88EF9FE00F94716189819A818156BA
:10F12000904F803A9F4020F11A821982E5EAF7E079
:10F130008491882341F09091C00095FFFCCF80938B
:10F14000C6003196F5CF8091C00085FFFCCF8AE0E4
:10F150008093C600BE016F5F7F4F88EF9FE00F94E2
:10F16000606188E697E00F94F56581E00F94C564CF
:10F170000F900F90DF91CF9108950E94536540E961
:10F1800050ED63E070E080EF96E00E94EF5BE4E614
:10F19000FCE08491882341F09091C00095FFFCCF62
:10F1A0008093C6003196F5CF8091C00085FFFCCFDB
:10F1B0008AE08093C6002CE33DE0F9018491882326
:10F1C00041F09091C00095FFFCCF8093C60031962E
:10F1D000F5CF44B740FF17C0E3EDFDE7859194916B
:10F1E000FC015491552341F06091C00065FFFCCFB4
:10F1F0005093C6000196F4CF8091C00085FFFCCFEC
:10F200008AE08093C60041FF17C0E7EFF0E88591E0
:10F210009491FC015491552341F06091C00065FF29
:10F22000FCCF5093C6000196F4CF8091C00085FFBB
:10F23000FCCF8AE08093C60042FF17C0E7EEF1E8FA
:10F2400085919491FC015491552341F06091C00047
:10F2500065FFFCCF5093C6000196F4CF8091C000AB
:10F2600085FFFCCF8AE08093C60043FF17C0E7EF1D
:10F27000F9E785919491FC015491552341F06091F7
:10F28000C00065FFFCCF5093C6000196F4CF80917B
:10F29000C00085FFFCCF8AE08093C60045FF17C001
:10F2A000E1E4FBE785919491FC014491442341F012
:10F2B0005091C00055FFFCCF4093C6000196F4CF9B
:10F2C0008091C00085FFFCCF8AE08093C60014BE09
:10F2D000F9018491ECE3FDE0882349F09091C000AE
:10F2E00095FFFCCF8093C60031968491F5CFE3E87B
:10F2F000F1E885919491FC014491442341F05091AF
:10F30000C00055FFFCCF4093C6000196F4CFEFE458
:10F31000FCE08491882341F09091C00095FFFCCFE0
:10F320008093C6003196F5CFEDE3F3E88591949193
:10F33000FC014491442341F05091C00055FFFCCFA3
:10F340004093C6000196F4CFEEE3FCE0849188235D
:10F3500041F09091C00095FFFCCF8093C60031969C
:10F36000F5CF8091C00085FFFCCF8AE08093C60076
:10F37000E3E3FCE08491882341F09091C00095FF85
:10F38000FCCF8093C6003196F5CFE7E2FCE0849194
:10F39000882341F09091C00095FFFCCF8093C60078
:10F3A0003196F5CF8091C00085FFFCCF8AE0809335
:10F3B000C600F9012491ECE3FDE0222349F080919D
:10F3C000C00085FFFCCF2093C60031962491F5CF75
:10F3D000E3E6F0E885919491FC012491222341F029
:10F3E0003091C00035FFFCCF2093C6000196F4CFCA
:10F3F0000E94C7C14AE050E0BC0180EF96E00E9445
:10F40000185DE3EEFDE785919491FC0124912223A0
:10F4100041F03091C00035FFFCCF2093C60001962B
:10F42000F4CF4AE050E060E575E080EF96E00E949E
:10F43000185D8091C00085FFFCCF8AE08093C600F4
:10F4400080E00F94C5640E9406580E94DEC10F94AC
:10F45000E2440F9449240F945A410E94A5EF0F945F
:10F4600090638091000186FD3BC0FFEF23ED80E3B8
:10F47000F15020408040E1F700C000008091000181
:10F4800086FD37C00F94326189E19CE00F94BE780D
:10F49000809101018460809301019FB7F89480916D
:10F4A00002018460809302019FBF8091000186FF6A
:10F4B000FCCF9FB7F894809102018B7F809302016B
:10F4C0009FBF9FEFE7EAF1E69150E040F040E1F79F
:10F4D00000C000000F94A16660E00E94566509C05C
:10F4E0002FEF83ED90E3215080409040E1F700C082
:10F4F0000000159884EC9FE00F945DCB80931D185D
:10F500006BE178E181EC9FE00F94716120911D180F
:10F5100080911B1890911C182F3F11F4009721F037
:10F520008F3FEFEF9E0711F410921D18019621F402
:10F5300010921C1810921B1880911D18882321F01E
:10F5400088E090E00F94AD718BEB9FE00F945DCB62
:10F5500091E0813009F090E09093630C8DE99AE09E
:10F560000E942FC98CEF9FE00F9465CB6F3F7F4FB8
:10F570008F4F9F4FB9F488EF9FE00F9465CB6F3F9B
:10F580007F4F8F4F9F4F71F484EF9FE00F9465CBB7
:10F590006F3F7F4F8F4F9F4F29F460E08FEF9FE0C9
:10F5A0000F948DCB8EEF9FE00F945DCB8093530A29
:10F5B000873010F00F94479E8FEA9FE00F945DCB49
:10F5C0008F3F41F460E08FEA9FE00F948DCB109263
:10F5D000800A06C091E0811101C090E09093800AFA
:10F5E00086EA9FE00F945DCB8F3F29F460E086EAC6
:10F5F0009FE00F948DCB84DD87EF9FE00F945DCB70
:10F600009FEF980F9E3F70F160E070E088EF9FE001
:10F610000F9489CBE091530AF0E0EE0FFF1FEB59F6
:10F62000FF47859194910F94F56563E87AE087EA46
:10F630009FE00F94716165E87AE089EA9FE00F949A
:10F64000716167E87AE08BEA9FE00F94716169E885
:10F650007AE08DEA9FE00F94716181E00F94C564B8
:10F660000D9495B6863E41F4E091530AF0E0EE0F1A
:10F67000FF1FEF5EFC4711C08130B9F48091800A12
:10F68000882399F20E94BE628111CFCFE091530A84
:10F69000F0E0EE0FFF1FED50F248859194910F942A
:10F6A000F56581E00F94C564C0CF803F09F0BDCF00
:10F6B000B1CF8F929F92AF92BF92CF92DF92EF9293
:10F6C000FF920F931F93CF93DF9381E08093470ABC
:10F6D00085E090E09093450A8093440A89E790E0A2
:10F6E0009093430A8093420A82E00F94CB63E091A7
:10F6F0000C0A84E0E89FF0011124E65CF84E20E05B
:10F7000030E042E053E460817181828193810F9403
:10F7100039C21816B4F420E030E040E85FE36091AD
:10F720002C0A70912D0A80912E0A90912F0A0F9425
:10F7300019BF60932C0A70932D0A80932E0A909320
:10F740002F0AE090280AF090290A00912A0A1091C5
:10F750002B0A2091240A3091250A4091260A5091C3
:10F76000270A6091200A7091210A8091220A9091C3
:10F77000230ACCE0DAE0DF93CF93812C912CB8EC14
:10F78000AB2EB3E4BB2EECE2CE2EEAE0DE2E0F94DD
:10F79000152680E090E0ACE8B2E48093200A9093D4
:10F7A000210AA093220AB093230A80E090E0A0E40B
:10F7B000B0EC8093240A9093250AA093260AB09374
:10F7C000270A80E090E0A0E8BFE38093280A9093A6
:10F7D000290AA0932A0AB0932B0ADF93CF93812C96
:10F7E000912CF8E4AF2EF2E4BF2EE12CF12C00E8CE
:10F7F0001FE320E030E040E450EC60E070E08CE893
:10F8000092E40F9415260F94B93E0F900F900F902D
:10F810000F906091401770914117882777FD809570
:10F82000982F0F94ACC09B01AC016091341770917C
:10F83000351780913617909137170F9419BF9F771E
:10F8400020E030E040E85FE30F9439C2181624F45A
:10F8500088EE93E0D5DADDCFC8E7D0E088EE93E01C
:10F86000CFDAD093430AC093420AC336D10519F0C8
:10F87000C930D10511F482E001C081E00F94CB635F
:10F88000219761F71092450A1092440A1092430A98
:10F890001092420A1092470ADF91CF911F910F9167
:10F8A000FF90EF90DF90CF90BF90AF909F908F90A0
:10F8B00008952F923F924F925F926F927F928F9214
:10F8C0009F92AF92BF92CF92DF92EF92FF920F93EF
:10F8D0001F93CF93DF93CDB7DEB7CA58D2400FB690
:10F8E000F894DEBF0FBECDBFC958DD4F6883798362
:10F8F0008A839B83C757D240FE01E75FFD4F88E2B2
:10F90000DF011D928A95E9F7E850F24080E991E025
:10F91000DF019C011D9221503040E1F7C75ADD4FB5
:10F9200019821882C955D240CE01875A9D4F5C0179
:10F930004E019FE6891A9EEF990ADE01AF51BE4F34
:10F940003D0190EBC92E9FE0D92E22E3E22EF12C4F
:10F9500000E010E0C359DD4F8882CD56D240CD582B
:10F96000DD4F9882C357D240B701882777FD809535
:10F97000982F0F94ACC0D3016D937D938D939D937D
:10F980003D01F501619171915F01882777FD8095B7
:10F99000982F0F94ACC0D4016D937D938D939D935C
:10F9A0004D010F5F1F4F0630110559F0B501C6011B
:10F9B0000F947161BAE0EB0EF11CE2E0CE0ED11CA7
:10F9C000D3CFCF51DE4F288139814A815B81C15E1F
:10F9D000D140C958DD4F688179818A819B81C757A1
:10F9E000D2400F940AC087FD2BC3FE01EF51FE4F9A
:10F9F0007F016E01FFE2CF1AFEEFDF0A3E012BEB23
:10FA0000621A2DEF720AC359DD4F0881CD56D240DC
:10FA1000CD58DD4F1881C357D24085E090E0CF58D4
:10FA2000DD4F99838883C157D240CF58DD4FA881DD
:10FA3000B981C157D2401197CF58DD4FB983A88300
:10FA4000C157D240F701208931894289538964899D
:10FA50007589868997890F9419BF4B015C01D8017C
:10FA600050962D913D914D915C91539754966D9187
:10FA70007D918D919C9157970F9419BFA501940189
:10FA80000F9411C0F60192938293729362936F0167
:10FA9000D301BE92AE929E928E923D010450110906
:10FAA000B4E0EB1AF108CF58DD4FE881F981C15776
:10FAB000D240EF2B09F0B9CF6E01FFECCF1AFDEF6A
:10FAC000DF0A3E0127E4621A2EEF720A2E013DE39F
:10FAD000430E511CCE0101967C0101E010E0D601DD
:10FAE0008D909D90AD90BC90139714962D913D9163
:10FAF0004D915C911797C501B4010F941ABF9B01FA
:10FB0000AC010F941ABFF70164A775A786A797A742
:10FB10000130110541F080A691A6A2A6B3A6848269
:10FB20009582A682B7820F5F1F4FD30114962D9145
:10FB30003D914D915C91179718966D917D918D91A6
:10FB40009C911B970F9419BF20E030E040EC50E4EB
:10FB50000F940BC3F2016083718382839383F4E07B
:10FB6000CF0ED11C2CE2E20EF11C34E0630E711CAE
:10FB700088E2480E511C0530110509F0B0CF8E0106
:10FB80000B5A1F4F6E0191E5C90ED11C22242394FC
:10FB9000312C2C0E3D1EA8ED2A0E311CF801B89711
:10FBA0002081318142815381F8016081718182819C
:10FBB00093810F9411C04B015C01E12CF12C3601B3
:10FBC000F8E26F1A710826014E0C5F1CF301EE0D6E
:10FBD000FF1D2481358146815781C501B4010F94F1
:10FBE0000BC39B01AC01D20114966D917D918D9157
:10FBF0009C9117970F9419BFF201648375838683D4
:10FC00009783F4E0EF0EF11C24E1E216F104D9F63B
:10FC1000045D1F4F38E2C30ED11C0215130509F015
:10FC2000BDCF1E0185EB280E311C6E0191EBC90E74
:10FC3000D11C3E01A7EE6A1AADEF7A0AB4E0EB2EB2
:10FC4000F12C270100E010E0812C912CA12CB12C8B
:10FC5000F601E00FF11FD301A00FB11F2D913D91CF
:10FC60004D915C9160817181828193810F940BC36E
:10FC70009B01AC01B401C5010F941ABF4B015C019B
:10FC8000BFEF4B1A5B0A0C5F1F4FE5E04E165104A5
:10FC9000F9F69B01AC01D1016D917D918D919C9103
:10FCA0000F9419BFF60120813181428153810F9455
:10FCB00011C0D3016D937D938D939C931397B1E005
:10FCC000EB1AF108E8E22E1A3108FCE2CF1AD1084B
:10FCD00024E0621A7108E114F10409F0B2CFCB50AC
:10FCE000DE4F88819981AA81BB81C55FD140C95708
:10FCF000DD4F88839983AA83BB83C758D2408E0186
:10FD0000075F1D4FDE01AF5CBD4FC558DD4FB983A6
:10FD1000A883CB57D240C359DD4F2880CD56D2405F
:10FD2000CD58DD4F3880C357D240FE01EF51FE4F12
:10FD3000C358DD4FF983E883CD57D240C358DD4F18
:10FD4000A881B981CD57D240CD90DD90ED90FD9046
:10FD5000C358DD4FB983A883CD57D240C958DD4F72
:10FD6000288139814A815B81C757D240C701B601DA
:10FD70000F940AC01816B4F0C358DD4FE881F9811A
:10FD8000CD57D2402081318142815381C958DD4F06
:10FD9000688179818A819B81C757D2400F940AC0BC
:10FDA0001816FCF4CF58DD4F28813981C157D24055
:10FDB0002430310509F01FC1C957DD4F2881398131
:10FDC0004A815B81C758D240C958DD4F688179812B
:10FDD0008A819B81C757D2400F9439C218160CF004
:10FDE0000AC1D80114968D919D910D90BC91A02DC2
:10FDF000C158DD4F88839983AA83BB83CF57D240F4
:10FE0000F8014080518062807380C558DD4FA88121
:10FE1000B981CB57D2408D919D910D90BC91A02D71
:10FE2000C359DD4F88839983AA83BB83CD56D240C3
:10FE3000D1018D919D910D90BC91A02DCD57DD4F9D
:10FE400088839983AA83BB83C358D240A7019601B4
:10FE5000C958DD4F688179818A819B81C757D2401B
:10FE60000F9419BFCD58DD4F688379838A839B83B4
:10FE7000C357D24020E030E040E450E40F946EC31A
:10FE80006B017C01A3019201C158DD4F688179812A
:10FE90008A819B81CF57D2400F9419BF4B015C01DF
:10FEA00020E030E040EC50E4C359DD4F68817981B7
:10FEB0008A819B81CD56D2400F940BC39B01AC012C
:10FEC000C501B4010F9411C0A70196010F940BC393
:10FED0006B017C0120E030E040E05FE3C301B20150
:10FEE0000F940BC34B015C01CD58DD4F2881398144
:10FEF0004A815B81C357D240CA01B9010F940BC339
:10FF00009B01AC01C501B4010F940BC39B01AC0173
:10FF1000C701B6010F941ABF6B017C01CD57DD4FAD
:10FF2000288139814A815B81C358D240F1016481C3
:10FF30007581868197810F9419BFC359DD4F288140
:10FF400039814A815B81CD56D2400F9411C04B015B
:10FF50005C01C359DD4F288139814A815B81CD56CF
:10FF6000D240CA01B9010F941ABFA30192010F94A4
:10FF70000BC32B013C01C359DD4F288139814A81D4
:10FF80005B81CD56D240C158DD4F688179818A812D
:10FF90009B81CF57D2400F940BC39B01AC01C3018F
:10FFA000B2010F941ABF20E030E040EC50E40F940F
:10FFB00011C09B01AC01C501B4010F9419BFCD580C
:10FFC000DD4F288139814A815B81C357D2400F942C
:10FFD0000BC39B01AC01C701B6010F941ABFCD57EB
:10FFE000DD4F288139814A815B81C358D2400F940B
:10FFF0001ABF4B015C01CF58DD4F28813981C157B1
:020000021000EC
:10000000D2402F5F3F4FCF58DD4F39832883C157F0
:10001000D2400C5F1F4FC558DD4F88819981CB5767
:10002000D2400496C558DD4F99838883CB57D24080
:1000300094E0290E311C2530310509F07FCE04C033
:10004000812C912CA12CB12CB401C501C657DD4FD8
:100050000FB6F894DEBF0FBECDBFDF91CF911F91D9
:100060000F91FF90EF90DF90CF90BF90AF909F9057
:100070008F907F906F905F904F903F902F9008955A
:100080008F929F92AF92BF92CF92DF92EF92FF92A8
:100090000F931F93CF93DF931F921F92CDB7DEB7BD
:1000A0001A82198287EF9FE00F945DCB813009F0AF
:1000B0009DC02091401730914117EAE0F0E0C9015E
:1000C000BF010F94E9C4892BD9F4C901CC978932B7
:1000D0009105B0F4BF010F94E9C4CB018852984F49
:1000E000BE016F5F7F4F880F991F0F947161698107
:1000F0007A81882777FD8095982F0F94ACC008C02F
:10010000B901882777FD8095982F0F94ACC0D1DB7B
:100110002091361630913716409138165091391685
:100120000F9411C06B017C01E6E6F7E0849188230F
:1001300041F09091C00095FFFCCF8093C6003196AE
:10014000F5CFE5E5F7E08491882341F09091C00078
:1001500095FFFCCF8093C6003196F5CF22E030E0CA
:10016000B701A60180EF96E00E940B5E20E030E030
:1001700040E252E460915102709152028091530228
:10018000909154020F9411C04B015C01A70196019C
:100190006091280A7091290A80912A0A90912B0A6D
:1001A0000F9419BF7B018C012091240A3091250AFC
:1001B0004091260A5091270A6091200A7091210AE5
:1001C0008091220A9091230AECE0FAE0FF93EF93EA
:1001D000ECE2CE2EEAE0DE2E0F9415260F94B93E07
:1001E00088E29AE00F9421340F900F900F900F90B7
:1001F000DF91CF911F910F91FF90EF90DF90CF9003
:10020000BF90AF909F908F9008954F925F926F92A2
:100210007F928F929F92AF92BF92CF92DF92EF9296
:10022000FF920F931F93CF93DF93CDB7DEB728973D
:100230000FB6F894DEBF0FBECDBF0F94B93E8091CC
:1002400047029091480290938C0A80938B0AE09128
:100250000C0AF0E0EE0FFF1FEE5BF84E608171813B
:10026000882777FD8095982F0F94ACC06093740A0F
:100270007093750A8093760A9093770A80910A0AA0
:1002800090910B0A9093730A8093720A0F9424B78B
:1002900060935A0A70935B0A80935C0A90935D0A9C
:1002A0008091200A9091210AA091220AB091230AFC
:1002B00089839A83AB83BC838093620A9093630A99
:1002C000A093640AB093650A4090240A5090250ACE
:1002D0006090260A7090270A4092660A5092670A38
:1002E0006092680A7092690A8091280A9091290A9E
:1002F000A0912A0AB0912B0A8D839E83AF83B88781
:1003000080936A0A90936B0AA0936C0AB0936D0A6B
:1003100060912C0A70912D0A80912E0A90912F0ADB
:1003200060936E0A70936F0A8093700A9093710ABB
:1003300020E030E040E85FE30F9419BF60932C0A9F
:1003400070932D0A80932E0A90932F0A8CE09AE0E6
:100350009F938F93812C912CB8ECAB2EB3E4BB2EE2
:100360001CE2C12E1AE0D12EED80FE800F8118858F
:10037000A301920169817A818B819C810F9415265A
:1003800020E030E040EA51E46091280A7091290AA7
:1003900080912A0A90912B0A0F941ABF2B013C01DD
:1003A0000F900F9020E030E042E553E40F9439C203
:1003B00018164CF04092280A5092290A60922A0A94
:1003C00070922B0A0CC080E090E0A2E5B3E4809329
:1003D000280A9093290AA0932A0AB0932B0AE09046
:1003E000280AF090290A00912A0A10912B0A2091DC
:1003F000240A3091250A4091260A5091270A6091DB
:10040000200A7091210A8091220A9091230AACE07F
:100410006A2EAAE07A2E7F926F92812C912CB0E7FF
:10042000AB2EB1E4BB2EECE2CE2EEAE0DE2E0F9432
:1004300015261092431710924217109245171092EA
:100440004417109247171092461780E090E0A8E4F6
:10045000B2E48093200A9093210AA093220AB093D9
:10046000230A80E090E0AEE3B3E48093240A909303
:10047000250AA093260AB093270AE090280AF09054
:10048000290A00912A0A10912B0A7F926F92812CDF
:10049000912CF8E4AF2EF2E4BF2E9C01AD01C50112
:1004A000B4010F94152610920B0A10920A0A0F90AD
:1004B0000F900F900F9028960FB6F894DEBF0FBEE6
:1004C000CDBFDF91CF911F910F91FF90EF90DF9003
:1004D000CF90BF90AF909F908F907F906F905F90E4
:1004E0004F900D94B93EE0910C0A84E0E89FF00132
:1004F0001124E65CF84E4081518162817381E2E50E
:10050000F7E08491882341F09091C00095FFFCCFE3
:100510008093C6003196F5CF22E030E080EF96E080
:100520000E940B5EEEE4F7E08491882341F0909105
:10053000C00095FFFCCF8093C6003196F5CF609147
:100540000C0A70E04AE050E080EF96E00E94185DEF
:10055000EAE4F7E08491882341F09091C00095FF90
:10056000FCCF8093C6003196F5CF4091341750915F
:100570003517609136177091371721E030E080EF22
:1005800096E00E940B5E8091C00085FFFCCF8AE060
:100590008093C60008958091890C882349F040918A
:1005A0003B0D50913C0D60913D0D70913E0D03C08F
:1005B00040E050E0BA018AE99FE00D9481CB2F9290
:1005C0003F924F925F926F927F928F929F92AF92E3
:1005D000BF92CF92DF92EF92FF920F931F93CF9330
:1005E000DF93CDB7DEB7C655D1090FB6F894DEBF9D
:1005F0000FBECDBF50988BE493E00E941A5E882313
:10060000A1F00091D1071091D2070B5F1F4F6AE252
:1006100070E0C8010F94C1C8009711F0DC011C9272
:10062000C8010F943D620C9437AB80E493E00E94C4
:100630001A5E882309F42BC180E593E00E941A5EBC
:10064000882391F080911D18882311F40C9437AB06
:100650000F9424B76093910A7093920A8093930A3F
:100660009093940A0C9437AB85E593E00E941A5E50
:10067000882361F06091500A7091510A4AE050E07D
:1006800080EF96E00E946A5D0C9437AB89E593E0B9
:100690000E941A5E8823C1F080911D18882361F0A2
:1006A00060911B1870911C184AE050E080EF96E0B2
:1006B0000E941F5D0C9437AB6CE573E080EF96E011
:1006C0000E940B5D0C9437AB8EE693E00E941A5E9D
:1006D000882379F16091D1077091D2076D5F7F4FC8
:1006E00021E041E08DE99AE00E94B2CE80918E0C2B
:1006F00090918F0CA091900CB091910C80933B0D38
:1007000090933C0DA0933D0DB0933E0D86E89CE088
:100710000E9499BB2091C00025FFFCCF8093C600AA
:100720000A9721F760E08DE99AE00E9442CE0C948E
:1007300037AB81E793E00E941A5E882399F00E940C
:10074000136881E08093520A6091D1077091D207BB
:100750006C5F7F4F21E040E08DE99AE00E94B2CECD
:100760000C9437AB85E793E00E941A5E8823A9F0CA
:10077000E9E7F3E08191882339F09091C00095FF7B
:10078000FCCF8093C600F6CF8091C00085FFFCCFE0
:100790008AE08093C6000C9437AB84E893E00E9413
:1007A0001A5E8823A9F0E8E8F3E08191882339F004
:1007B0009091C00095FFFCCF8093C600F6CF80914A
:1007C000C00085FFFCCF8AE08093C6000C9437AB55
:1007D00086EA93E00E941A5E882321F00F94DB6181
:1007E0000C9437AB8BEA93E00E941A5E882341F0A9
:1007F00060E070E088EF9FE00F9460610C9437AB8D
:100800008EEA93E00E941A5E882359F06EEA73E044
:1008100080EF96E00E940B5D40E950ED63E070E0F0
:1008200010C089EB93E00E941A5E882381F069EB87
:1008300073E080EF96E00E940B5D40EA55E266E2CD
:1008400070E080EF96E00E94EF5B0C9424B385EC9F
:1008500093E00E941A5E882361F00F9424B760939E
:100860007C0A70937D0A80937E0A90937F0A0C9491
:1008700037AB8AEC93E00E941A5E882311F40C9443
:1008800037AB61E080E00E9456650C9437AB8EE593
:100890000E942E5E81110C9437AB87E40E942E5E7D
:1008A000882311F40C94AE900E94C95E0F9479C015
:1008B0006B34710509F406C70CF050C06430710543
:1008C00009F4FFC354F46230710509F4E2C30CF07B
:1008D000ECC377FF92C00C9437AB6B30710509F411
:1008E00046C45CF46A30710511F00C9437AB60E0DB
:1008F00081E00E94F96C0C9437AB6C31710509F4FE
:100900003CC46E31710511F00C9437AB0F94B93EB5
:1009100081E00E944F5E8091510290915202A0911D
:100920005302B091540280930B0290930C02A09357
:100930000D02B0930E0220E030E043E060E070E092
:1009400080E291EC0E94DEF2E091530AF0E0EE0FBB
:10095000FF1FED5FFC47859194914EC66735710589
:1009600011F40C942E90DCF46035710511F40C94A4
:10097000168F34F46C34710509F4D1C60C9437AB7E
:100980006135710511F40C94758F6635710511F0A0
:100990000C9437AB86EE0E94B8620C9437AB6C3582
:1009A000710511F40C9437907CF46A35710511F4DB
:1009B0000C9433906B35710511F00C9437AB81E0DA
:1009C0008093CA090C9437AB6236710511F40C940C
:1009D00099906336710511F00C9437AB10921D1885
:1009E0000F94E06160911D1884EC9FE00F946FCB31
:1009F00082E00F94CB630C9437AB8091BB078111DD
:100A00000C9437AB489BDAC2809147029091480220
:100A100090934202809341022091200A3091210A52
:100A20004091220A5091230A28AF39AF4AAF5BAFF9
:100A30002F8F38A349A35AA34090240A5090250A27
:100A40006090260A7090270A4BA25CA26DA27EA23B
:100A50008091280A9091290AA0912A0AB0912B0A24
:100A60008CAF9DAFAEAFBFAF8FA398A7A9A7BAA712
:100A700060912C0A70912D0A80912E0A90912F0A74
:100A800029833A834B835C834D825E826F827886B2
:100A90002CAD3DAD4EAD5FAD29873A874B875C8766
:100AA0006D877E878F87988B20E030E040E050E4B0
:100AB0000F9419BF6BA77CA78DA79EA71CE0212EC2
:100AC0001AE0312E3F922F92812C912C08ECA02E0F
:100AD00003E4B02EAE01455D5F4F6A01ECACFDACA6
:100AE0000EAD1FADA301920168AD79AD8AAD9BAD8E
:100AF0000F94152620E030E040EA51E46FA178A57C
:100B000089A59AA50F941ABF7B018C016FA378A7C2
:100B100089A79AA72BA13CA14DA15EA16F8D78A1B9
:100B200089A19AA13F922F92812C912CE6E9AE2EB9
:100B3000E3E4BE2E0F9415261F8E18A219A21AA246
:100B40008DEC9CECACE0B0EC8BA39CA3ADA3BEA35E
:100B5000EFA0F8A409A51AA53F922F92812C912C01
:100B6000FCE8AF2EF2E4BF2E9C01AD0160E070E026
:100B7000CB010F94152620E030E040EA52E46BA54B
:100B80007CA58DA59EA50F9419BF6BA77CA78DA7EB
:100B90009EA7EFA0F8A409A51AA52BA13CA14DA1E1
:100BA0005EA16F8D78A189A19AA13F922F92812C8D
:100BB000912CA0EAAA2EA1E4BA2E0F9415260F9428
:100BC000B93E149A64E670E080E090E00F9453B769
:100BD0000F94C78A0FB6F894DEBF0FBECDBF00E0FA
:100BE00010E0F12C0F94EC6581112AC0F3940F945E
:100BF000224D81E00E944876F110F4CF043FF1E0ED
:100C00001F0711F400E010E08091010184608093DF
:100C100001010115110531F49FB7F894809102018B
:100C2000846008C00431110541F49FB7F8948091A5
:100C300002018B7F809302019FBF0F5F1F4FD2CFB6
:100C40009FB7F894809102018B7F809302019FBF30
:100C500020E030E04CE852E46BA57CA58DA59EA574
:100C60000F941ABF6BA77CA78DA79EA7EFA0F8A42F
:100C700009A51AA52BA13CA14DA15EA16F8D78A15C
:100C800089A19AA1FCE06F2EFAE07F2E7F926F92ED
:100C9000812C912CA0EAAA2EA1E4BA2EDE019B960B
:100CA0006D010F94152620E030E048E452E46BA576
:100CB0007CA58DA59EA50F941ABF6BA77CA78DA7B9
:100CC0009EA7EFA0F8A409A51AA52BA13CA14DA1B0
:100CD0005EA16F8D78A189A19AA17F926F92812CDC
:100CE000912CA12CB0E4BB2E0F9415261092790AFA
:100CF0001092780A0F94488B0F900F900F900F90DE
:100D00008091780A9091790A019709F489C010922C
:100D1000790A1092780A0F94928B8091780A9091B8
:100D2000790A8230910571F1039709F076C020E0CD
:100D300030E048E452E46BA57CA58DA59EA50F94F8
:100D40001ABF6BA77CA78DA79EA7EFA0F8A409A543
:100D50001AA52BA13CA14DA15EA16F8D78A189A1FF
:100D60009AA17F926F92812C912CA12CA0E4BA2E93
:100D7000DE019B966D010F9415260F94FE8A0F904D
:100D80000F90BECF20E030E04CE852E46BA57CA58C
:100D90008DA59EA50F941ABF6BA77CA78DA79EA7B4
:100DA000EFA0F8A409A51AA52BA13CA14DA15EA115
:100DB0006F8D78A189A19AA17F926F92812C912C3D
:100DC000B0EAAB2EB1E4BB2EDE019B966D010F9411
:100DD000152620E030E048E452E46BA57CA58DA503
:100DE0009EA50F941ABF6BA77CA78DA79EA7EFA007
:100DF000F8A409A51AA52BA13CA14DA15EA16F8D58
:100E000078A189A19AA17F926F92812C912CA12C1B
:100E1000E0E4BE2E0F9415266DCF0F94EB8A70CFB1
:100E200020E030E040EA50E46BA57CA58DA59EA5AE
:100E30000F941ABF6BA77CA78DA79EA7EFA0F8A45D
:100E400009A51AA52BA13CA14DA15EA16F8D78A18A
:100E500089A19AA1ECE06E2EEAE07E2E7F926F923D
:100E6000812C912CA12CF0E4BF2EFE01BB966F01CA
:100E70000F941526A50194016BA57CA58DA59EA5B3
:100E80000F9419BF6BA77CA78DA79EA7EFA0F8A40E
:100E900009A51AA52BA13CA14DA15EA16F8D78A13A
:100EA00089A19AA17F926F92812C912CA8ECAA2EF5
:100EB000A3E4BA2E0F941526EFA0F8A409A51AA54D
:100EC0002BA13CA14DA15EA16F8D78A189A19AA112
:100ED0007F926F92812C912CBCE8AB2EB2E4BB2E9A
:100EE0000F941526EFA0F8A409A51AA52D813E811F
:100EF0004F81588569817A818B819C817F926F9225
:100F00000F941526E984FA840B851C852D813E817A
:100F10004F81588569817A818B819C817F926F9204
:100F2000812C912CE8E4AE2EE3E4BE2E0F9415261E
:100F300020E030E040E050E46BA57CA58DA59EA5A7
:100F40000F941ABF6BA77CA78DA79EA7E984FA848C
:100F50000B851C852D813E814F81588569817A8161
:100F60008B819C817F926F92812C912CF0EAAF2E25
:100F7000F0E4BF2E0F941526CE010D960F94443445
:100F800080914102909142028093470290934802DF
:100F90009F938F9387EC9BE09F938F938E01015DCE
:100FA0001F4F1F930F930F9441C960E0C8010E9427
:100FB000B5630FB6F894DEBF0FBECDBF0E942E6999
:100FC00060914C0A70914D0A80914E0A90914F0A9F
:100FD0000F94AAC04B015C01C0902C0AD0902D0A3E
:100FE000E0902E0AF0902F0A4090F7095090F809EF
:100FF0006090F9097090FA09A3019201C701B60146
:101000000F9419BF20E030E048EC52E40F940BC37A
:101010009B01AC01C501B4010F9439C21816E4F468
:10102000A7019601C301B2010F9419BF20E030E07F
:1010300048EC52E40F940BC39B01AC01C501B40111
:101040000F941ABF0F947EC060934C0A70934D0AA0
:1010500080934E0A90934F0A8091090A8823A9F041
:1010600088E50E942E5E811110C089E50E942E5EE7
:1010700081110BC08AE50E942E5E811106C085E4B5
:101080000E942E5E81110C943AAB0E94F66B0C9478
:1010900037AB8091BB0781110C9437AB0E94B169CB
:1010A00081E00E94D46E0C9437AB8091BB07811114
:1010B0000C9437AB0E94B16980E00E94D46E0C940E
:1010C00037AB80E50E942E5E882339F00E94C95E0E
:1010D0000F947EC04B015C0103C0812C912C540104
:1010E00083E50E942E5E882361F00E94C95E20E0A5
:1010F00030E04AE754E40F940BC30F947EC04B01D9
:101100005C0181149104A104B10459F0E091530AE7
:10111000F0E0EE0FFF1FE15EFE47859194910F9482
:101120004A620F94B93E0F9424B72B013C01480C3E
:10113000591C6A1C7B1C0F9424B76093CD077093D5
:10114000CE078093CF079093D0070F9424B76415F0
:1011500075058605970510F00C9437AB0F94224D5A
:1011600080E00E94487680E00F94CB63EECF60E091
:1011700080E00E94F96C0C9437AB11E01093810A67
:101180001092930F0E94DEEF0F94EF1880910B02E4
:1011900090910C02A0910D02B0910E028093D7099C
:1011A0009093D809A093D909B093DA0980914702A6
:1011B0009091480290938C0A80938B0A84E690E089
:1011C00090934802809347020F9424B76093CD0711
:1011D0007093CE078093CF079093D00781E00F9450
:1011E0007C358091200A9091210AA091220AB09129
:1011F000230A8093EB099093EC09A093ED09B09337
:10120000EE094091240A5091250A6091260A7091B6
:10121000270A4093EF095093F0096093F109709306
:10122000F2094091280A5091290A60912A0A709186
:101230002B0A4093F3095093F4096093F5097093D6
:10124000F60940912C0A50912D0A60912E0A709156
:101250002F0A4093F7095093F8096093F9097093A6
:10126000FA0910920B0210920C0210920D021092C9
:101270000E0288E50E942E5E882311F080E009C0EE
:1012800089E50E942E5E8111F9CF8AE50E942E5ECB
:10129000812780930F0281110C9469AB88E50E942D
:1012A0002E5E81110C9469AB80910F0281110C9418
:1012B0006FAB89E50E942E5E81110C946FAB88E5BF
:1012C0000E942E5E882341F00E94445E672B682BAB
:1012D000692B11F00C9475AB89E50E942E5E882372
:1012E00041F00E94445E672B682B692B11F00C942F
:1012F0008BAB80910F02811106C08AE50E942E5EA1
:10130000882309F4EDC08091110A882311F40C940C
:10131000A1AB8091120A882311F40C94A1AB0E9416
:1013200033F0EAE4FEE885919591A591B491898323
:101330009A83AB83BC83E6E4FEE885919591A59101
:10134000B4918F8F98A3A9A3BAA32FEE39E04BEEE7
:1013500059E0BE016F5F7F4FCE014F960E94E7605C
:101360000E94A5EF2DEC3CEC4CE050EC6091EF09B5
:101370007091F0098091F1099091F2090F940AC0DF
:1013800087FF0CC08DEC9CECACE0B0EC8093EF09D7
:101390009093F009A093F109B093F20980E090E0F6
:1013A000A0EAB0E48093F3099093F409A093F509BF
:1013B000B093F60920E030E040E251E46091510240
:1013C0007091520280915302909154020F9411C077
:1013D00060930B0270930C0280930D0290930E02A7
:1013E0001092280A1092290A10922A0A10922B0AA7
:1013F00080E00F947C35E090280AF090290A009153
:101400002A0A10912B0A2091240A3091250A409132
:10141000260A5091270A6091200A7091210A809132
:10142000220A9091230AFCE2CF2EFAE0DF2E0F94DD
:10143000C03280900B0290900C02A0900D02B090F0
:101440000E02E090F309F090F4090091F509109173
:10145000F6092091EF093091F0094091F10950917E
:10146000F2096091EB097091EC098091ED0990917E
:10147000EE09ECE0FAE0FF93EF93A7EFCA2EA9E0A4
:10148000DA2E0F9415260F94B93E8091EB099091B6
:10149000EC09A091ED09B091EE098093200A909398
:1014A000210AA093220AB093230A8091EF09909118
:1014B000F009A091F109B091F2098093240A909368
:1014C000250AA093260AB093270A81E00F947C3561
:1014D0000F94643582E090E00E94175F0F900F90A8
:1014E0008AE50E942E5E8823D1F00E94445E672B1D
:1014F000682B692BA1F00E94C95E20911C0A3091D3
:101500001D0A40911E0A50911F0A0F941ABF609342
:10151000280A7093290A80932A0A90932B0AE09054
:10152000280AF090290A00912A0A10912B0A20918A
:10153000240A3091250A4091260A5091270A609189
:10154000200A7091210A8091220A9091230AECE2EC
:10155000CE2EEAE0DE2E0F94C03280E00F947C3570
:101560008091D7099091D809A091D909B091DA0951
:1015700080930B0290930C02A0930D02B0930E0285
:1015800080918B0A90918C0A909348028093470235
:101590000F9424B76093CD077093CE078093CF0745
:1015A0009093D0070F9464350E9433F00E944FF25D
:1015B00088E50E942E5E81110C94ABAB89E50E94F8
:1015C0002E5E81110C94ABAB87E50E942E5E8111DB
:1015D0000C94ABAB8AE50E942E5E81110C94ABABF0
:1015E0000F94B93E1092810A21C43091C00035FF9A
:1015F000FCCF2093C6000196FC0124912111F5CF68
:10160000E2ECFBE08491882341F09091C00095FFCB
:10161000FCCF8093C6003196F5CF4091200A5091BF
:10162000210A6091220A7091230A25E030E080EFC0
:1016300096E00E940B5EEDEBFBE08491882341F085
:101640009091C00095FFFCCF8093C6003196F5CFF6
:101650004091240A5091250A6091260A7091270A28
:1016600025E030E080EF96E00E940B5EE8EBFBE0C7
:101670008491882341F09091C00095FFFCCF809326
:10168000C6003196F5CF4091280A5091290A609101
:101690002A0A70912B0A25E030E080EF96E00E9444
:1016A0000B5EE6EBFBE08491882341F09091C00053
:1016B00095FFFCCF8093C6003196F5CF0E947D5EEA
:1016C0000C9437AB08E210E04AE050E0B80180EF3C
:1016D00096E00E94185DEAE7F6E08191882339F0F0
:1016E0009091C00095FFFCCF8093C600F6CFB80163
:1016F000882777FD8095982F0F94ACC00E94597C65
:10170000AB01BC0122E030E080EF96E00E940C5E6D
:101710000F5F1F4F0F361105B9F60C9437AB82E3FC
:1017200090E090934117809340171A82198280911C
:10173000110A882341F08091120A882321F08091B8
:10174000130A81110AC081E08093D60761E08FEA15
:101750009BE00E9492640C9437ABE1E9FBE084913A
:10176000882341F09091C00095FFFCCF8093C60084
:101770003196F5CF8091C00085FFFCCF8AE0809341
:10178000C60084E090E09093450A8093440A81E08B
:1017900090E09093430A8093420AE091530AF0E06C
:1017A000EE0FFF1FED55F5488591949121E0892BAF
:1017B00009F420E02093470A80E090E0ACE8B2E42E
:1017C0008093200A9093210AA093220AB093230ABF
:1017D00080E090E0A0E4B0EC8093240A9093250A86
:1017E000A093260AB093270A80E090E0A0E8BFE328
:1017F0008093280A9093290AA0932A0AB0932B0A6F
:101800008CE09AE09F938F93812C912C18E4A12E69
:1018100012E4B12E0CE2C02E0AE0D02EE12CF12C05
:1018200000E81FE320E030E040E450EC60E070E0CE
:101830008CE892E40F9415260F94B93E0F900F9008
:1018400020E030E048E452E460913417709135179D
:1018500080913617909137170F9419BF4B015C0197
:1018600020E030E0A9010F9439C218168CF420E072
:1018700030E040E85FE3C501B4010F9439C21816A7
:101880008CF488EE93E00E9400770E947382D8CF98
:1018900020E030E040E85FEBC501B4010F940AC0DE
:1018A00087FDEFCF08E710E088EE93E00E94007715
:1018B0000E94738201501109B9F760E086EA9FE047
:1018C0000F946FCB80E090E0A0EAB0E48093280A08
:1018D0009093290AA0932A0AB0932B0A2091240AF4
:1018E0003091250A4091260A5091270A6091200ADA
:1018F0007091210A8091220A9091230AECE0FAE08B
:10190000FF93EF93812C912CE8E4AE2EE2E4BE2EFF
:10191000FCE2CF2EFAE0DF2EE12CF12C00EA10E4FD
:101920000F941526E6E4FEE885919591A591B49172
:101930008093200A9093210AA093220AB093230A4D
:10194000EAE4FEE825913591459154912093240ACB
:101950003093250A4093260A5093270AE090280ADC
:10196000F090290A00912A0A10912B0A6091200A0E
:101970007091210A8091220A9091230AECE0FAE00A
:10198000FF93EF93812C912CB8E4AB2EB2E4BB2EE5
:101990000F9415260F94B93E20E030E043E060E05C
:1019A00070E080E89FEB0E94DEF22091280A3091DF
:1019B000290A40912A0A50912B0A28AF39AF4AAF21
:1019C0005BAFE0E9FBE084910F900F900F900F90D8
:1019D0004091280A5091290A60912A0A70912B0A95
:1019E000882349F09091C00095FFFCCF8093C600FA
:1019F00031968491F5CF8091C00085FFFCCF8AE0BD
:101A00008093C600E9E8FBE08491882341F090913F
:101A1000C00095FFFCCF8093C6003196F5CF22E041
:101A200030E080EF96E00E940B5EE8E8FBE08491F6
:101A3000882341F09091C00095FFFCCF8093C600B1
:101A40003196F5CF8091C00085FFFCCF8AE080936E
:101A5000C60012E0412E512C0CE3602E712C80EB5D
:101A6000282E8FE0382EE1E8FBE08491882341F0B6
:101A70009091C00095FFFCCF8093C6003196F5CFC2
:101A80004AE050E0B20180EF96E00E94185DEEE778
:101A9000FBE08491882341F09091C00095FFFCCF3A
:101AA0008093C6003196F5CF8091C00085FFFCCFB2
:101AB0008AE08093C6005092430A4092420AB301E2
:101AC000882777FD8095982F0F94ACC06CAF7DAFC1
:101AD0008EAF9FAF709241176092401720E030E0C8
:101AE0004CE852E42093200A3093210A4093220AC2
:101AF0005093230A80E090E0A0E4B0EC8093240AA5
:101B00009093250AA093260AB093270A20E030E09C
:101B100040E85FE32093280A3093290A40932A0A79
:101B200050932B0AACE0BAE0BF93AF93812C912C79
:101B3000A8E4AA2EA2E4BA2EBCE2CB2EBAE0DB2E99
:101B400079018A0120E030E040E450EC60E070E090
:101B50008CE892E40F9415260F94B93E0F900F90E5
:101B60002CAD3DAD4EAD5FAD609134177091351722
:101B700080913617909137170F940AC087FF07C0DE
:101B800088EE93E00E9400770E947382E9CF08E715
:101B900010E088EE93E00E9400770E94738201506B
:101BA0001109B9F720E030E040EA50E42093280A18
:101BB0003093290A40932A0A50932B0A2091240A31
:101BC0003091250A4091260A5091270A6091200AF7
:101BD0007091210A8091220A9091230AACE0BAE028
:101BE000BF93AF93812C912C18E4A12E12E4B12E57
:101BF0000CE2C02E0AE0D02EE12CF12C00EA10E419
:101C00000F941526E6E4FEE885919591A591B4918F
